 openloop_DE_sfun

 Timestamp is 523061f5 (Wed Sep 11 08:28:37 2013)

 Preferred load address is 0000000180000000

 Start         Length     Name                   Class
 0001:00000000 00036a14H .text                   CODE
 0001:00036a20 00000092H .text$x                 CODE
 0002:00000000 00000478H .idata$5                DATA
 0002:00000478 00000008H .CRT$XCA                DATA
 0002:00000480 00000008H .CRT$XCZ                DATA
 0002:00000488 00000008H .CRT$XIA                DATA
 0002:00000490 00000008H .CRT$XIAA               DATA
 0002:00000498 00000008H .CRT$XIZ                DATA
 0002:000004a0 00004b0cH .rdata                  DATA
 0002:00004fb0 00000008H .rtc$IAA                DATA
 0002:00004fb8 00000008H .rtc$IZZ                DATA
 0002:00004fc0 00000008H .rtc$TAA                DATA
 0002:00004fc8 00000008H .rtc$TZZ                DATA
 0002:00004fd0 00003f94H .xdata                  DATA
 0002:00008f64 0000008cH .idata$2                DATA
 0002:00008ff0 00000014H .idata$3                DATA
 0002:00009008 00000478H .idata$4                DATA
 0002:00009480 00000a5cH .idata$6                DATA
 0002:00009ee0 00000056H .edata                  DATA
 0003:00000000 000018e8H .data                   DATA
 0003:00001900 000026d8H .bss                    DATA
 0004:00000000 00003084H .pdata                  DATA

  Address         Publics by Value              Rva+Base               Lib:Object

 0000:00000000       ___safe_se_handler_table   0000000000000000     <absolute>
 0000:00000000       ___safe_se_handler_count   0000000000000000     <absolute>
 0000:00000000       __ImageBase                0000000180000000     <linker-defined>
 0001:00000000       sf_c2_openloop_DE_get_eml_resolved_functions_info 0000000180001000 f   c2_openloop_DE.obj
 0001:000004e0       sf_c2_openloop_DE_get_check_sum 00000001800014e0 f   c2_openloop_DE.obj
 0001:00000560       sf_c2_openloop_DE_get_autoinheritance_info 0000000180001560 f   c2_openloop_DE.obj
 0001:00000ef0       sf_internal_get_sim_state_c2_openloop_DE 0000000180001ef0 f   c2_openloop_DE.obj
 0001:00001240       sf_internal_set_sim_state_c2_openloop_DE 0000000180002240 f   c2_openloop_DE.obj
 0001:00001640       c2_openloop_DE_method_dispatcher 0000000180002640 f   c2_openloop_DE.obj
 0001:00004450       sf_process_check_sum_call  0000000180005450 f   openloop_DE_sfun_registry.obj
 0001:000044a0       sf_process_autoinheritance_call 00000001800054a0 f   openloop_DE_sfun_registry.obj
 0001:00004640       sf_process_get_eml_resolved_functions_info_call 0000000180005640 f   openloop_DE_sfun_registry.obj
 0001:000047c0       sf_mex_unlock_call         00000001800057c0 f   openloop_DE_sfun_registry.obj
 0001:00004870       sf_machine_global_initializer_called 0000000180005870 f   openloop_DE_sfun_registry.obj
 0001:000048a0       sf_machine_global_method_dispatcher 00000001800058a0 f   openloop_DE_sfun_registry.obj
 0001:00004900       sf_machine_global_terminator 0000000180005900 f   openloop_DE_sfun_registry.obj
 0001:00004940       sf_register_machine_exported_symbols 0000000180005940 f   openloop_DE_sfun_registry.obj
 0001:00004960       callCustomFcn              0000000180005960 f   openloop_DE_sfun_registry.obj
 0001:00004970       sf_machine_global_initializer 0000000180005970 f   openloop_DE_sfun_registry.obj
 0001:000049e0       _ssSetStateAbsTol          00000001800059e0 f   openloop_DE_sfun_registry.obj
 0001:00004ac0       _ssGetAbsTol               0000000180005ac0 f   openloop_DE_sfun_registry.obj
 0001:00004b30       _ssSetInputPortMatrixDimensions 0000000180005b30 f   openloop_DE_sfun_registry.obj
 0001:00004c40       _ssSetOutputPortMatrixDimensions 0000000180005c40 f   openloop_DE_sfun_registry.obj
 0001:00004d50       _ssSetInputPortVectorDimension 0000000180005d50 f   openloop_DE_sfun_registry.obj
 0001:00004e20       _ssSetOutputPortVectorDimension 0000000180005e20 f   openloop_DE_sfun_registry.obj
 0001:00004ef0       ssIsRunTimeParamTunable    0000000180005ef0 f   openloop_DE_sfun_registry.obj
 0001:00004f60       ssGetSFuncBlockHandle      0000000180005f60 f   openloop_DE_sfun_registry.obj
 0001:00004fd0       _ssGetCurrentInputPortWidth 0000000180005fd0 f   openloop_DE_sfun_registry.obj
 0001:000050f0       _ssGetCurrentOutputPortWidth 00000001800060f0 f   openloop_DE_sfun_registry.obj
 0001:00005210       _ssGetCallSystemNumFcnCallDestinations 0000000180006210 f   openloop_DE_sfun_registry.obj
 0001:00005280       ssWarning                  0000000180006280 f   openloop_DE_sfun_registry.obj
 0001:00005390       ssGetIsZeroCrossControlDisabled 0000000180006390 f   openloop_DE_sfun_registry.obj
 0001:00005400       ssSetIsInputPortUsedForContZcSignal 0000000180006400 f   openloop_DE_sfun_registry.obj
 0001:00005470       ssSetZcSignalIsZcElementDisc 0000000180006470 f   openloop_DE_sfun_registry.obj
 0001:00005520       ssSetZcSignalName          0000000180006520 f   openloop_DE_sfun_registry.obj
 0001:00005590       ssSetZcSignalWidth         0000000180006590 f   openloop_DE_sfun_registry.obj
 0001:00005600       ssSetZcSignalZcEventType   0000000180006600 f   openloop_DE_sfun_registry.obj
 0001:00005670       ssSetZcSignalType          0000000180006670 f   openloop_DE_sfun_registry.obj
 0001:000056e0       ssSetZcSignalZcTol         00000001800066e0 f   openloop_DE_sfun_registry.obj
 0001:00005750       ssSetZcSignalNeedsEventNotification 0000000180006750 f   openloop_DE_sfun_registry.obj
 0001:000057c0       ssCreateAndAddZcSignalInfo 00000001800067c0 f   openloop_DE_sfun_registry.obj
 0001:00005830       ssCloneAndAddZcSignalInfo  0000000180006830 f   openloop_DE_sfun_registry.obj
 0001:000058a0       ssGetNumZcSignals          00000001800068a0 f   openloop_DE_sfun_registry.obj
 0001:00005910       ssGetZcSignalVector        0000000180006910 f   openloop_DE_sfun_registry.obj
 0001:00005980       ssGetZcSignalZcEvents      0000000180006980 f   openloop_DE_sfun_registry.obj
 0001:000059f0       ssGetZcSignalName          00000001800069f0 f   openloop_DE_sfun_registry.obj
 0001:00005a60       ssGetZcSignalWidth         0000000180006a60 f   openloop_DE_sfun_registry.obj
 0001:00005ad0       ssGetZcSignalZcEventType   0000000180006ad0 f   openloop_DE_sfun_registry.obj
 0001:00005b40       ssGetZcSignalType          0000000180006b40 f   openloop_DE_sfun_registry.obj
 0001:00005bb0       ssGetZcSignalZcTol         0000000180006bb0 f   openloop_DE_sfun_registry.obj
 0001:00005c30       ssGetZcSignalNeedsEventNotification 0000000180006c30 f   openloop_DE_sfun_registry.obj
 0001:00005ca0       ssGetZcSignalIsZcElementDisc 0000000180006ca0 f   openloop_DE_sfun_registry.obj
 0001:00005d40       ssGetIsInputPortElementContinuous 0000000180006d40 f   openloop_DE_sfun_registry.obj
 0001:00005de0       _ssGetInputPortSignalPtrsFcn 0000000180006de0 f   openloop_DE_sfun_registry.obj
 0001:000060a0       _ssGetInputPortSignalFcn   00000001800070a0 f   openloop_DE_sfun_registry.obj
 0001:000062c0       _ssSetInputPortDirectFeedThroughFcn 00000001800072c0 f   openloop_DE_sfun_registry.obj
 0001:00006420       _ssSetInputPortReusableFcn 0000000180007420 f   openloop_DE_sfun_registry.obj
 0001:00006510       _ssSetOutputPortReusableFcn 0000000180007510 f   openloop_DE_sfun_registry.obj
 0001:000065f0       ssGetDTypeIdFromMxArray    00000001800075f0 f   openloop_DE_sfun_registry.obj
 0001:00006710       ssWriteRTWStr              0000000180007710 f   openloop_DE_sfun_registry.obj
 0001:00006770       ssWriteRTWMxVectParam      0000000180007770 f   openloop_DE_sfun_registry.obj
 0001:000067d0       ssWriteRTWMx2dMatParam     00000001800077d0 f   openloop_DE_sfun_registry.obj
 0001:00006850       ssWriteRTWNameValuePair    0000000180007850 f   openloop_DE_sfun_registry.obj
 0001:00006d40       ssWriteRTWParameters       0000000180007d40 f   openloop_DE_sfun_registry.obj
 0001:00007340       ssWriteRTWParamSettings    0000000180008340 f   openloop_DE_sfun_registry.obj
 0001:00007a10       ssWriteRTWWorkVect         0000000180008a10 f   openloop_DE_sfun_registry.obj
 0001:00007f10       mexFunction                0000000180008f10 f   openloop_DE_sfun_registry.obj
 0001:00009bd0       ProcessMexSfunctionEveryCall 000000018000abd0 f   openloop_DE_sfun_registry.obj
 0001:00009d40       openloop_DE_initializer    000000018000ad40 f   openloop_DE_sfun.obj
 0001:00009d50       openloop_DE_terminator     000000018000ad50 f   openloop_DE_sfun.obj
 0001:00009d60       sf_openloop_DE_method_dispatcher 000000018000ad60 f   openloop_DE_sfun.obj
 0001:00009db0       sf_openloop_DE_process_check_sum_call 000000018000adb0 f   openloop_DE_sfun.obj
 0001:0000a1c0       sf_openloop_DE_autoinheritance_info 000000018000b1c0 f   openloop_DE_sfun.obj
 0001:0000a330       sf_openloop_DE_get_eml_resolved_functions_info 000000018000b330 f   openloop_DE_sfun.obj
 0001:0000a460       openloop_DE_debug_initialize 000000018000b460 f   openloop_DE_sfun.obj
 0001:0000a4d0       openloop_DE_register_exported_symbols 000000018000b4d0 f   openloop_DE_sfun.obj
 0001:0000a4e0       load_openloop_DE_optimization_info 000000018000b4e0 f   openloop_DE_sfun.obj
 0001:0000a530       unload_openloop_DE_optimization_info 000000018000b530 f   openloop_DE_sfun.obj
 0001:0000a650       sf_mex_mx_is_numeric       000000018000b650 f   sfc_mex:sfc_mex.obj
 0001:0000a690       strcmp_ignore_ws           000000018000b690 f   sfc_mex:sfc_mex.obj
 0001:0000a7d0       sf_mex_duplicatearraysafe  000000018000b7d0 f   sfc_mex:sfc_mex.obj
 0001:0000a930       sf_set_error_debugger_context_message_fcn 000000018000b930 f   sfc_mex:sfc_mex.obj
 0001:0000a940       sf_set_debugger_matlab_error_fcn 000000018000b940 f   sfc_mex:sfc_mex.obj
 0001:0000a970       sf_set_error_prefix_string 000000018000b970 f   sfc_mex:sfc_mex.obj
 0001:0000a9a0       sf_get_error_prefix_string 000000018000b9a0 f   sfc_mex:sfc_mex.obj
 0001:0000a9b0       sf_mex_enter_parallel_region 000000018000b9b0 f   sfc_mex:sfc_mex.obj
 0001:0000a9c0       sf_mex_exit_parallel_region 000000018000b9c0 f   sfc_mex:sfc_mex.obj
 0001:0000a9d0       sf_get_current_jmp_buf_ptr 000000018000b9d0 f   sfc_mex:sfc_mex.obj
 0001:0000a9e0       sf_set_current_jmp_buf_ptr 000000018000b9e0 f   sfc_mex:sfc_mex.obj
 0001:0000a9f0       sf_mex_set_halt_simulation 000000018000b9f0 f   sfc_mex:sfc_mex.obj
 0001:0000aa00       sf_mex_get_halt_simulation 000000018000ba00 f   sfc_mex:sfc_mex.obj
 0001:0000aa10       sf_mex_clear_error_message 000000018000ba10 f   sfc_mex:sfc_mex.obj
 0001:0000aa30       sf_mex_get_error_message_for_read 000000018000ba30 f   sfc_mex:sfc_mex.obj
 0001:0000aa40       sf_mex_get_error_message_buffer_length 000000018000ba40 f   sfc_mex:sfc_mex.obj
 0001:0000ab20       sf_mex_warning_message     000000018000bb20 f   sfc_mex:sfc_mex.obj
 0001:0000ab90       sf_mex_v_errbuf_createf    000000018000bb90 f   sfc_mex:sfc_mex.obj
 0001:0000aba0       sf_mex_errbuf_createf      000000018000bba0 f   sfc_mex:sfc_mex.obj
 0001:0000abd0       sf_mex_v_errbuf_catf       000000018000bbd0 f   sfc_mex:sfc_mex.obj
 0001:0000ac10       sf_mex_errbuf_catf         000000018000bc10 f   sfc_mex:sfc_mex.obj
 0001:0000ac60       sf_mex_errbuf_copy         000000018000bc60 f   sfc_mex:sfc_mex.obj
 0001:0000ac70       sf_mex_errbuf_clear        000000018000bc70 f   sfc_mex:sfc_mex.obj
 0001:0000ac80       sf_mex_errbuf_isempty      000000018000bc80 f   sfc_mex:sfc_mex.obj
 0001:0000ad90       sf_mex_set_error_status    000000018000bd90 f   sfc_mex:sfc_mex.obj
 0001:0000ade0       sf_mex_error_direct_call   000000018000bde0 f   sfc_mex:sfc_mex.obj
 0001:0000ae00       sf_mex_error_message_no_long_jump 000000018000be00 f   sfc_mex:sfc_mex.obj
 0001:0000ae20       sf_mex_long_jump_on_error  000000018000be20 f   sfc_mex:sfc_mex.obj
 0001:0000ae50       sf_mex_call_matlab         000000018000be50 f   sfc_mex:sfc_mex.obj
 0001:0000af70       sf_mex_check_builtin       000000018000bf70 f   sfc_mex:sfc_mex.obj
 0001:0000b010       sf_mex_check_builtin_vs    000000018000c010 f   sfc_mex:sfc_mex.obj
 0001:0000b0d0       sf_mex_check_enum          000000018000c0d0 f   sfc_mex:sfc_mex.obj
 0001:0000b150       sf_mex_create_enum         000000018000c150 f   sfc_mex:sfc_mex.obj
 0001:0000b1c0       sf_mex_get_enum_element    000000018000c1c0 f   sfc_mex:sfc_mex.obj
 0001:0000b1d0       sf_mex_createcellarray     000000018000c1d0 f   sfc_mex:sfc_mex.obj
 0001:0000b1e0       sf_mex_setcell             000000018000c1e0 f   sfc_mex:sfc_mex.obj
 0001:0000b1f0       sf_mex_getcell             000000018000c1f0 f   sfc_mex:sfc_mex.obj
 0001:0000b200       sf_mex_dup                 000000018000c200 f   sfc_mex:sfc_mex.obj
 0001:0000b220       sf_mex_assign              000000018000c220 f   sfc_mex:sfc_mex.obj
 0001:0000b2a0       sf_mex_destroy             000000018000c2a0 f   sfc_mex:sfc_mex.obj
 0001:0000b2d0       mx_array_has_fi_type       000000018000c2d0 f   sfc_mex:sfc_mex.obj
 0001:0000b300       sf_mex_convert_from_fi     000000018000c300 f   sfc_mex:sfc_mex.obj
 0001:0000b430       sf_mex_convert_to_double   000000018000c430 f   sfc_mex:sfc_mex.obj
 0001:0000b550       sf_mex_import_fi_vs        000000018000c550 f   sfc_mex:sfc_mex.obj
 0001:0000b710       sf_matrix_matrix_index_ok  000000018000c710 f   sfc_mex:sfc_mex.obj
 0001:0000b7a0       sf_vector_vector_index_ok  000000018000c7a0 f   sfc_mex:sfc_mex.obj
 0001:0000b7d0       ssGetCurrentInputPortDimensions_wrapper 000000018000c7d0 f   sfc_mex:sfc_mex.obj
 0001:0000b7f0       ssGetCurrentOutputPortDimensions_wrapper 000000018000c7f0 f   sfc_mex:sfc_mex.obj
 0001:0000b810       sf_mex_emlrt_context_is_debug_mode 000000018000c810 f   sfc_mex:sfc_mex.obj
 0001:0000b820       sf_mex_emlrt_context_set_debug_mode 000000018000c820 f   sfc_mex:sfc_mex.obj
 0001:0000b830       sf_mex_emlrtNameCapturePostProcessR2012a 000000018000c830 f   sfc_mex:sfc_mex.obj
 0001:0000b8a0       sf_clear_error_manager_info 000000018000c8a0 f   sfc_mex:sfc_mex.obj
 0001:0000b900       sf_mex_stop_simulation_abruptly_wo_error 000000018000c900 f   sfc_mex:sfc_mex.obj
 0001:0000b940       sf_mex_error_message       000000018000c940 f   sfc_mex:sfc_mex.obj
 0001:0000b9a0       sf_react_to_error_in_matlab_call 000000018000c9a0 f   sfc_mex:sfc_mex.obj
 0001:0000b9d0       sf_mex_addfield            000000018000c9d0 f   sfc_mex:sfc_mex.obj
 0001:0000ba70       sf_mex_getfield            000000018000ca70 f   sfc_mex:sfc_mex.obj
 0001:0000bd70       sf_mex_check_class         000000018000cd70 f   sfc_mex:sfc_mex.obj
 0001:0000be10       sf_mex_is_real             000000018000ce10 f   sfc_mex:sfc_mex.obj
 0001:0000c280       sf_mex_decode_encoded_mx_struct_array 000000018000d280 f   sfc_mex:sfc_mex.obj
 0001:0000c560       sf_mex_lw_bounds_check     000000018000d560 f   sfc_mex:sfc_mex.obj
 0001:0000c590       sf_mex_lw_size_eq_check_1d 000000018000d590 f   sfc_mex:sfc_mex.obj
 0001:0000c5b0       sf_mex_lw_size_eq_check_nd 000000018000d5b0 f   sfc_mex:sfc_mex.obj
 0001:0000c790       sf_mex_lw_dim_size_eq_check 000000018000d790 f   sfc_mex:sfc_mex.obj
 0001:0000c7c0       sf_mex_lw_dim_size_geq_check 000000018000d7c0 f   sfc_mex:sfc_mex.obj
 0001:0000c7f0       sf_mex_lw_sub_assign_size_check_nd 000000018000d7f0 f   sfc_mex:sfc_mex.obj
 0001:0000ca20       sf_mex_lw_runtime_error_msgid 000000018000da20 f   sfc_mex:sfc_mex.obj
 0001:0000cb10       sf_mex_lw_matrix_matrix_index_check 000000018000db10 f   sfc_mex:sfc_mex.obj
 0001:0000cb30       sf_mex_lw_vector_vector_index_check 000000018000db30 f   sfc_mex:sfc_mex.obj
 0001:0000cb70       sf_mex_lw_for_loop_vector_check 000000018000db70 f   sfc_mex:sfc_mex.obj
 0001:0000cc00       sf_mex_lw_non_negative_check 000000018000dc00 f   sfc_mex:sfc_mex.obj
 0001:0000cc40       sf_mex_overflow_error      000000018000dc40 f   sfc_mex:sfc_mex.obj
 0001:0000cc50       sf_mex_dividebyzero_error  000000018000dc50 f   sfc_mex:sfc_mex.obj
 0001:0000cc60       sf_mex_unsafe_enum_error   000000018000dc60 f   sfc_mex:sfc_mex.obj
 0001:0000cc70       sf_emlrtErrHandler         000000018000dc70 f   sfc_mex:sfc_mex.obj
 0001:0000cd50       sf_mex_size_one_check      000000018000dd50 f   sfc_mex:sfc_mex.obj
 0001:0000cd70       sf_mex_printf              000000018000dd70 f   sfc_mex:sfc_mex.obj
 0001:0000cf40       sf_mex_check_size          000000018000df40 f   sfc_mex:sfc_mex.obj
 0001:0000d210       sf_mex_check_struct        000000018000e210 f   sfc_mex:sfc_mex.obj
 0001:0000d470       sf_mex_check_struct_vs     000000018000e470 f   sfc_mex:sfc_mex.obj
 0001:0000d500       sf_mex_check_fi            000000018000e500 f   sfc_mex:sfc_mex.obj
 0001:0000d600       sf_mex_check_fi_vs         000000018000e600 f   sfc_mex:sfc_mex.obj
 0001:0000d6a0       sf_echo_expression         000000018000e6a0 f   sfc_mex:sfc_mex.obj
 0001:0000d700       sf_assertion_failed        000000018000e700 f   sfc_mex:sfc_mex.obj
 0001:0000d9e0       sf_mex_evalin              000000018000e9e0 f   sfc_mex:sfc_mex.obj
 0001:0000dc50       sf_mex_export              000000018000ec50 f   sfc_mex:sfc_mex.obj
 0001:0000dd10       sf_mex_get_ml_var_no_error 000000018000ed10 f   sfc_mex:sfc_mex.obj
 0001:0000deb0       sf_mex_get_ml_var          000000018000eeb0 f   sfc_mex:sfc_mex.obj
 0001:0000e350       ml_set_element_value_in_array 000000018000f350 f   sfc_mex:sfc_mex.obj
 0001:0000fa20       sf_mex_call_impl           0000000180010a20 f   sfc_mex:sfc_mex.obj
 0001:0000ff50       sf_mex_call_debug          0000000180010f50 f   sfc_mex:sfc_mex.obj
 0001:0000ff80       sf_mex_call                0000000180010f80 f   sfc_mex:sfc_mex.obj
 0001:000105d0       sf_mex_createstruct        00000001800115d0 f   sfc_mex:sfc_mex.obj
 0001:000106c0       sf_mex_createstructarray   00000001800116c0 f   sfc_mex:sfc_mex.obj
 0001:00010740       sf_mex_get_mx_datatype_from_sf_datatype 0000000180011740 f   sfc_mex:sfc_mex.obj
 0001:00010a50       sf_mex_ml_var_sub          0000000180011a50 f   sfc_mex:sfc_mex.obj
 0001:00010c20       sf_mex_ml_var_subsasgn     0000000180011c20 f   sfc_mex:sfc_mex.obj
 0001:00011010       sf_mex_sub                 0000000180012010 f   sfc_mex:sfc_mex.obj
 0001:00011210       sf_mex_subsasgn            0000000180012210 f   sfc_mex:sfc_mex.obj
 0001:000116f0       sf_mex_create              00000001800126f0 f   sfc_mex:sfc_mex.obj
 0001:00012140       sf_mex_import_named        0000000180013140 f   sfc_mex:sfc_mex.obj
 0001:000121a0       sf_mex_import              00000001800131a0 f   sfc_mex:sfc_mex.obj
 0001:000121f0       sf_mex_import_vs           00000001800131f0 f   sfc_mex:sfc_mex.obj
 0001:00012300       sf_mex_lower_fixpt_mx_array 0000000180013300 f   sfc_mex:sfc_mex.obj
 0001:000125f0       sf_send_message_wrapper    00000001800135f0 f   sfc_mex:sfc_sf.obj
 0001:00012620       sf_receive_message_wrapper 0000000180013620 f   sfc_mex:sfc_sf.obj
 0001:00012660       sf_check_out_message_wrapper 0000000180013660 f   sfc_mex:sfc_sf.obj
 0001:000126a0       sf_check_in_message_wrapper 00000001800136a0 f   sfc_mex:sfc_sf.obj
 0001:000126e0       sf_no_message_wrapper      00000001800136e0 f   sfc_mex:sfc_sf.obj
 0001:00012a70       sim_mode_is_rtw_gen        0000000180013a70 f   sfc_mex:sfc_sf.obj
 0001:00012aa0       sim_mode_is_external       0000000180013aa0 f   sfc_mex:sfc_sf.obj
 0001:00012ab0       sim_mode_is_modelref_sim   0000000180013ab0 f   sfc_mex:sfc_sf.obj
 0001:00012ad0       mdlInitializeSizes         0000000180013ad0 f   sfc_mex:sfc_sf.obj
 0001:00012af0       mdlInitializeSampleTimes   0000000180013af0 f   sfc_mex:sfc_sf.obj
 0001:00012b30       mdlZeroCrossings           0000000180013b30 f   sfc_mex:sfc_sf.obj
 0001:00012c10       mdlDerivatives             0000000180013c10 f   sfc_mex:sfc_sf.obj
 0001:00012cc0       mdl_initialize_conditions_processing 0000000180013cc0 f   sfc_mex:sfc_sf.obj
 0001:00012cf0       mdlInitializeConditions    0000000180013cf0 f   sfc_mex:sfc_sf.obj
 0001:00012db0       mdlGetSimState             0000000180013db0 f   sfc_mex:sfc_sf.obj
 0001:00012dc0       mdlSetSimState             0000000180013dc0 f   sfc_mex:sfc_sf.obj
 0001:00012dd0       mdl_ext_mode_exec_processing 0000000180013dd0 f   sfc_mex:sfc_sf.obj
 0001:00012df0       mdlExtModeExec             0000000180013df0 f   sfc_mex:sfc_sf.obj
 0001:00012f80       mdlTerminate               0000000180013f80 f   sfc_mex:sfc_sf.obj
 0001:00012ff0       mdlRTW                     0000000180013ff0 f   sfc_mex:sfc_sf.obj
 0001:00013020       mdlSetWorkWidths           0000000180014020 f   sfc_mex:sfc_sf.obj
 0001:00013030       mdlProcessParameters       0000000180014030 f   sfc_mex:sfc_sf.obj
 0001:00013040       mdl_start_processing       0000000180014040 f   sfc_mex:sfc_sf.obj
 0001:000130a0       mdlStart                   00000001800140a0 f   sfc_mex:sfc_sf.obj
 0001:000131b0       mdlEnable                  00000001800141b0 f   sfc_mex:sfc_sf.obj
 0001:00013280       mdlDisable                 0000000180014280 f   sfc_mex:sfc_sf.obj
 0001:00013330       sf_get_chart_instance_ptr  0000000180014330 f   sfc_mex:sfc_sf.obj
 0001:00013350       sf_load_rtw_optimization_info 0000000180014350 f   sfc_mex:sfc_sf.obj
 0001:00013420       sf_rtw_info_uint_prop      0000000180014420 f   sfc_mex:sfc_sf.obj
 0001:00013560       sf_is_chart_inlinable      0000000180014560 f   sfc_mex:sfc_sf.obj
 0001:00013580       sf_mark_output_events_with_multiple_callers 0000000180014580 f   sfc_mex:sfc_sf.obj
 0001:00013710       sf_mark_chart_reusable_outputs 0000000180014710 f   sfc_mex:sfc_sf.obj
 0001:00013970       sf_mark_chart_expressionable_inputs 0000000180014970 f   sfc_mex:sfc_sf.obj
 0001:00013bd0       sf_get_subchart_simstruct  0000000180014bd0 f   sfc_mex:sfc_sf.obj
 0001:00013c20       sf_get_fixpt_data_type_id  0000000180014c20 f   sfc_mex:sfc_sf.obj
 0001:00013c60       sf_get_enum_data_type_id   0000000180014c60 f   sfc_mex:sfc_sf.obj
 0001:00013ca0       sf_get_param_data_type_id  0000000180014ca0 f   sfc_mex:sfc_sf.obj
 0001:00013cd0       sf_mex_listen_for_ctrl_c_force 0000000180014cd0 f   sfc_mex:sfc_sf.obj
 0001:00013de0       sf_mex_draw_now            0000000180014de0 f   sfc_mex:sfc_sf.obj
 0001:00013e20       sf_mex_set_debugger_sim_status_listener_fcn 0000000180014e20 f   sfc_mex:sfc_sf.obj
 0001:00013e30       sf_mex_listen_for_ctrl_c   0000000180014e30 f   sfc_mex:sfc_sf.obj
 0001:00013ec0       sf_mex_get_sfun_param      0000000180014ec0 f   sfc_mex:sfc_sf.obj
 0001:00013f10       sf_get_runtime_param_data  0000000180014f10 f   sfc_mex:sfc_sf.obj
 0001:00013f50       sf_call_output_fcn_call    0000000180014f50 f   sfc_mex:sfc_sf.obj
 0001:00014090       sf_call_output_fcn_enable  0000000180015090 f   sfc_mex:sfc_sf.obj
 0001:00014120       sf_call_output_fcn_disable 0000000180015120 f   sfc_mex:sfc_sf.obj
 0001:000141b0       sf_clear_rtw_identifier    00000001800151b0 f   sfc_mex:sfc_sf.obj
 0001:000149a0       sf_set_encoded_dwork_info  00000001800159a0 f   sfc_mex:sfc_sf.obj
 0001:000149f0       sf_get_dwork_info_from_mat_file 00000001800159f0 f   sfc_mex:sfc_sf.obj
 0001:00014bb0       sf_set_rtw_dwork_info      0000000180015bb0 f   sfc_mex:sfc_sf.obj
 0001:00014d20       mdlOutputs                 0000000180015d20 f   sfc_mex:sfc_sf.obj
 0001:00014ec0       sf_debug_disp              0000000180015ec0 f   sfc_debug:sfcdebug.obj
 0001:00015120       sf_debug_data_runtime_size_mismatch_error_check 0000000180016120 f   sfc_debug:sfcdebug.obj
 0001:000151c0       sf_debug_try_loading_machine 00000001800161c0 f   sfc_debug:sfcdebug.obj
 0001:000152c0       sf_debug_reset_current_state_configuration 00000001800162c0 f   sfc_debug:sfcdebug.obj
 0001:00015350       sf_debug_store_current_state_configuration 0000000180016350 f   sfc_debug:sfcdebug.obj
 0001:000153e0       sf_debug_restore_previous_state_configuration 00000001800163e0 f   sfc_debug:sfcdebug.obj
 0001:00015470       sf_debug_restore_previous_state_configuration2 0000000180016470 f   sfc_debug:sfcdebug.obj
 0001:00015500       sf_debug_get_event_scope   0000000180016500 f   sfc_debug:sfcdebug.obj
 0001:00015670       use_debugger_step_animation 0000000180016670 f   sfc_debug:sfcdebug.obj
 0001:00015690       sf_debug_get_script_id     0000000180016690 f   sfc_debug:sfcdebug.obj
 0001:00015720       sf_debug_set_script_translation 0000000180016720 f   sfc_debug:sfcdebug.obj
 0001:000158a0       sf_debug_extract_message_post_receive_info 00000001800168a0 f   sfc_debug:sfcdebug.obj
 0001:000159a0       sf_debug_get_current_machine_id 00000001800169a0 f   sfc_debug:sfcdebug.obj
 0001:000159c0       sf_debug_get_current_optional_integer 00000001800169c0 f   sfc_debug:sfcdebug.obj
 0001:000159d0       sf_debug_get_current_machine_number 00000001800169d0 f   sfc_debug:sfcdebug.obj
 0001:000159f0       sf_debug_get_current_machine_name 00000001800169f0 f   sfc_debug:sfcdebug.obj
 0001:00015a10       sf_debug_get_current_chart_id 0000000180016a10 f   sfc_debug:sfcdebug.obj
 0001:00015a60       sf_debug_get_current_chart_number 0000000180016a60 f   sfc_debug:sfcdebug.obj
 0001:00015a70       sf_debug_get_current_instance_number 0000000180016a70 f   sfc_debug:sfcdebug.obj
 0001:00015a80       sf_debug_get_current_is_minor_time_step 0000000180016a80 f   sfc_debug:sfcdebug.obj
 0001:00015b00       sf_debug_get_current_object_type 0000000180016b00 f   sfc_debug:sfcdebug.obj
 0001:00015b10       sf_debug_get_current_instance_handle 0000000180016b10 f   sfc_debug:sfcdebug.obj
 0001:00015b70       sf_debug_get_current_event_type 0000000180016b70 f   sfc_debug:sfcdebug.obj
 0001:00015b80       sf_debug_get_current_object_id 0000000180016b80 f   sfc_debug:sfcdebug.obj
 0001:00015bc0       sf_debug_get_current_active_event_type 0000000180016bc0 f   sfc_debug:sfcdebug.obj
 0001:00015bd0       sf_debug_get_current_active_event_id 0000000180016bd0 f   sfc_debug:sfcdebug.obj
 0001:00015c10       sf_debug_get_current_tag_type 0000000180016c10 f   sfc_debug:sfcdebug.obj
 0001:00015c20       sf_debug_get_current_simulation_time 0000000180016c20 f   sfc_debug:sfcdebug.obj
 0001:00015c30       sf_debug_get_current_coverage_percentage 0000000180016c30 f   sfc_debug:sfcdebug.obj
 0001:00015c40       sf_debug_current_statement_context 0000000180016c40 f   sfc_debug:sfcdebug.obj
 0001:00015cd0       sf_debug_get_current_statement_info 0000000180016cd0 f   sfc_debug:sfcdebug.obj
 0001:00015e50       sf_debug_terminate_instance 0000000180016e50 f   sfc_debug:sfcdebug.obj
 0001:00016190       sf_debug_assertion_failed  0000000180017190 f   sfc_debug:sfcdebug.obj
 0001:000163f0       sf_debug_set_number_of_data_with_change_event_for_machine 00000001800173f0 f   sfc_debug:sfcdebug.obj
 0001:00016430       sf_debug_set_machine_event_thresholds 0000000180017430 f   sfc_debug:sfcdebug.obj
 0001:00016450       sf_debug_set_machine_event_scope 0000000180017450 f   sfc_debug:sfcdebug.obj
 0001:00016490       sf_debug_set_machine_data_thresholds 0000000180017490 f   sfc_debug:sfcdebug.obj
 0001:000164d0       sf_debug_set_machine_data_scope 00000001800174d0 f   sfc_debug:sfcdebug.obj
 0001:00016560       sf_debug_set_machine_data_name 0000000180017560 f   sfc_debug:sfcdebug.obj
 0001:00016600       sf_debug_set_machine_data_size 0000000180017600 f   sfc_debug:sfcdebug.obj
 0001:00016740       sf_debug_set_machine_data_type 0000000180017740 f   sfc_debug:sfcdebug.obj
 0001:000168b0       sf_debug_get_chart_data_number 00000001800178b0 f   sfc_debug:sfcdebug.obj
 0001:000168d0       sf_debug_get_chart_event_number 00000001800178d0 f   sfc_debug:sfcdebug.obj
 0001:000168f0       sf_debug_set_chart_state_info 00000001800178f0 f   sfc_debug:sfcdebug.obj
 0001:00016970       sf_debug_set_chart_decomposition 0000000180017970 f   sfc_debug:sfcdebug.obj
 0001:000169e0       sf_debug_set_chart_substate_count 00000001800179e0 f   sfc_debug:sfcdebug.obj
 0001:00016ac0       sf_debug_set_chart_substate_index 0000000180017ac0 f   sfc_debug:sfcdebug.obj
 0001:00016b30       sf_debug_set_chart_state_substate_count 0000000180017b30 f   sfc_debug:sfcdebug.obj
 0001:00016c40       sf_debug_set_chart_state_substate_index 0000000180017c40 f   sfc_debug:sfcdebug.obj
 0001:00016cc0       sf_debug_set_number_of_data_with_change_event_for_chart 0000000180017cc0 f   sfc_debug:sfcdebug.obj
 0001:00016d40       sf_debug_set_number_of_states_with_entry_event_for_chart 0000000180017d40 f   sfc_debug:sfcdebug.obj
 0001:00016db0       sf_debug_set_number_of_states_with_exit_event_for_chart 0000000180017db0 f   sfc_debug:sfcdebug.obj
 0001:00016e20       sf_debug_set_chart_disable_implicit_casting 0000000180017e20 f   sfc_debug:sfcdebug.obj
 0001:00016e90       sf_debug_set_chart_event_thresholds 0000000180017e90 f   sfc_debug:sfcdebug.obj
 0001:00016f00       sf_debug_set_chart_data_compiled_props 0000000180017f00 f   sfc_debug:sfcdebug.obj
 0001:00017250       sf_debug_set_chart_data_props 0000000180018250 f   sfc_debug:sfcdebug.obj
 0001:00017570       sf_debug_check_fi_license  0000000180018570 f   sfc_debug:sfcdebug.obj
 0001:00017760       sf_debug_symbol_scope_push 0000000180018760 f   sfc_debug:sfcdebug.obj
 0001:000177a0       sf_debug_symbol_scope_push_eml 00000001800187a0 f   sfc_debug:sfcdebug.obj
 0001:000177f0       sf_debug_symbol_scope_pop  00000001800187f0 f   sfc_debug:sfcdebug.obj
 0001:00017830       sf_debug_symbol_scope_add_importable 0000000180018830 f   sfc_debug:sfcdebug.obj
 0001:000178b0       sf_debug_symbol_scope_add  00000001800188b0 f   sfc_debug:sfcdebug.obj
 0001:00017930       sf_debug_symbol_scope_add_dyn_importable 0000000180018930 f   sfc_debug:sfcdebug.obj
 0001:000179f0       sf_debug_symbol_scope_add_dyn 00000001800189f0 f   sfc_debug:sfcdebug.obj
 0001:00017a20       sf_debug_symbol_scope_add_eml_importable 0000000180018a20 f   sfc_debug:sfcdebug.obj
 0001:00017a60       sf_debug_symbol_scope_add_eml 0000000180018a60 f   sfc_debug:sfcdebug.obj
 0001:00017aa0       sf_debug_symbol_scope_add_eml_dyn_importable 0000000180018aa0 f   sfc_debug:sfcdebug.obj
 0001:00017b10       sf_debug_symbol_scope_add_eml_dyn 0000000180018b10 f   sfc_debug:sfcdebug.obj
 0001:00017b70       sf_debug_symbol_switch     0000000180018b70 f   sfc_debug:sfcdebug.obj
 0001:00017b90       sf_debug_symbol_scope_add_verbose 0000000180018b90 f   sfc_debug:sfcdebug.obj
 0001:00017c60       sf_debug_set_machine_data_value_ptr 0000000180018c60 f   sfc_debug:sfcdebug.obj
 0001:00017ca0       sf_debug_set_instance_data_value_ptr 0000000180018ca0 f   sfc_debug:sfcdebug.obj
 0001:00017d60       sf_debug_unset_instance_data_value_ptr 0000000180018d60 f   sfc_debug:sfcdebug.obj
 0001:00017e10       sf_debug_set_chart_event_scope 0000000180018e10 f   sfc_debug:sfcdebug.obj
 0001:00017e90       sf_debug_set_chart_transition_coverage_maps 0000000180018e90 f   sfc_debug:sfcdebug.obj
 0001:00017fa0       sf_debug_set_chart_state_coverage_maps 0000000180018fa0 f   sfc_debug:sfcdebug.obj
 0001:00018080       sf_debug_set_instance_transition_coverage_weights 0000000180019080 f   sfc_debug:sfcdebug.obj
 0001:00018120       sf_debug_set_instance_state_coverage_weights 0000000180019120 f   sfc_debug:sfcdebug.obj
 0001:00018370       sf_debug_unload_machine    0000000180019370 f   sfc_debug:sfcdebug.obj
 0001:000183c0       sf_debug_load_machine      00000001800193c0 f   sfc_debug:sfcdebug.obj
 0001:000184c0       sf_debug_set_active_instance_in_data_dictionary 00000001800194c0 f   sfc_debug:sfcdebug.obj
 0001:000186a0       sf_debug_set_active_instance 00000001800196a0 f   sfc_debug:sfcdebug.obj
 0001:00018800       sf_debug_chart_visiblity_change 0000000180019800 f   sfc_debug:sfcdebug.obj
 0001:00018900       sf_debug_select_chart      0000000180019900 f   sfc_debug:sfcdebug.obj
 0001:00018a70       sf_debug_set_instance_cv_ids 0000000180019a70 f   sfc_debug:sfcdebug.obj
 0001:00018d80       sf_debug_select_charts     0000000180019d80 f   sfc_debug:sfcdebug.obj
 0001:00018f10       sf_debug_initialized       0000000180019f10 f   sfc_debug:sfcdebug.obj
 0001:00018f20       sf_debug_is_uninterruptible 0000000180019f20 f   sfc_debug:sfcdebug.obj
 0001:00018f50       sf_debug_initialize_debugger_gui 0000000180019f50 f   sfc_debug:sfcdebug.obj
 0001:00019340       sf_debug_resume            000000018001a340 f   sfc_debug:sfcdebug.obj
 0001:00019360       sf_debug_go                000000018001a360 f   sfc_debug:sfcdebug.obj
 0001:00019370       sf_debug_break             000000018001a370 f   sfc_debug:sfcdebug.obj
 0001:00019380       sf_debug_step_over         000000018001a380 f   sfc_debug:sfcdebug.obj
 0001:00019390       sf_debug_step_out          000000018001a390 f   sfc_debug:sfcdebug.obj
 0001:000193a0       sf_debug_set_disable_all_breakpoints 000000018001a3a0 f   sfc_debug:sfcdebug.obj
 0001:000193b0       sf_debug_disable_all_breakpoints_and_go 000000018001a3b0 f   sfc_debug:sfcdebug.obj
 0001:000193c0       sf_debug_break_on_chart_entry 000000018001a3c0 f   sfc_debug:sfcdebug.obj
 0001:000193d0       sf_debug_break_on_event_broadcast 000000018001a3d0 f   sfc_debug:sfcdebug.obj
 0001:000193e0       sf_debug_break_on_state_entry 000000018001a3e0 f   sfc_debug:sfcdebug.obj
 0001:000193f0       sf_debug_break_between_times 000000018001a3f0 f   sfc_debug:sfcdebug.obj
 0001:00019410       sf_debug_browse_data       000000018001a410 f   sfc_debug:sfcdebug.obj
 0001:00019430       sf_debug_watch_data        000000018001a430 f   sfc_debug:sfcdebug.obj
 0001:00019450       sf_debug_assign_data       000000018001a450 f   sfc_debug:sfcdebug.obj
 0001:00019470       sf_debug_whos              000000018001a470 f   sfc_debug:sfcdebug.obj
 0001:00019490       sf_debug_get_consistency_info 000000018001a490 f   sfc_debug:sfcdebug.obj
 0001:000194a0       sf_debug_browse_trace      000000018001a4a0 f   sfc_debug:sfcdebug.obj
 0001:000194b0       sf_debug_set_breakpoints   000000018001a4b0 f   sfc_debug:sfcdebug.obj
 0001:00019610       sf_debug_set_eml_breakpoints 000000018001a610 f   sfc_debug:sfcdebug.obj
 0001:00019770       sf_debug_set_script_breakpoints 000000018001a770 f   sfc_debug:sfcdebug.obj
 0001:000197f0       sf_debug_add_script_breakpoints 000000018001a7f0 f   sfc_debug:sfcdebug.obj
 0001:00019860       sf_debug_clear_script_breakpoints 000000018001a860 f   sfc_debug:sfcdebug.obj
 0001:000198d0       sf_debug_query_script_breakpoints 000000018001a8d0 f   sfc_debug:sfcdebug.obj
 0001:00019990       sf_debug_get_eml_script_id 000000018001a990 f   sfc_debug:sfcdebug.obj
 0001:000199e0       sf_debug_set_watch         000000018001a9e0 f   sfc_debug:sfcdebug.obj
 0001:00019c10       sf_debug_get_instance_handle 000000018001ac10 f   sfc_debug:sfcdebug.obj
 0001:00019ca0       sf_debug_get_active_states 000000018001aca0 f   sfc_debug:sfcdebug.obj
 0001:00019cb0       sf_debug_get_animation     000000018001acb0 f   sfc_debug:sfcdebug.obj
 0001:00019cc0       sf_debug_set_animation     000000018001acc0 f   sfc_debug:sfcdebug.obj
 0001:00019cd0       sf_debug_animate           000000018001acd0 f   sfc_debug:sfcdebug.obj
 0001:00019d00       sf_debug_cycle_detection_check 000000018001ad00 f   sfc_debug:sfcdebug.obj
 0001:00019d10       sf_debug_data_range_check  000000018001ad10 f   sfc_debug:sfcdebug.obj
 0001:00019d20       sf_debug_transition_conflict_check 000000018001ad20 f   sfc_debug:sfcdebug.obj
 0001:00019d30       sf_debug_state_consistency_check 000000018001ad30 f   sfc_debug:sfcdebug.obj
 0001:00019d40       sf_debug_data_range_check_enabled 000000018001ad40 f   sfc_debug:sfcdebug.obj
 0001:00019d60       sf_debug_transition_conflict_check_enabled 000000018001ad60 f   sfc_debug:sfcdebug.obj
 0001:00019d80       sf_debug_transition_conflict_check_begin 000000018001ad80 f   sfc_debug:sfcdebug.obj
 0001:00019da0       sf_debug_transition_conflict_check_end 000000018001ada0 f   sfc_debug:sfcdebug.obj
 0001:00019dc0       sf_debug_stop_debugging    000000018001adc0 f   sfc_debug:sfcdebug.obj
 0001:00019df0       sf_debug_is_cycle_detected 000000018001adf0 f   sfc_debug:sfcdebug.obj
 0001:00019e00       sf_debug_is_array_bounds_detected 000000018001ae00 f   sfc_debug:sfcdebug.obj
 0001:00019e10       sf_debug_get_state_vectors_data_size 000000018001ae10 f   sfc_debug:sfcdebug.obj
 0001:00019e50       sf_debug_get_state_vectors_data 000000018001ae50 f   sfc_debug:sfcdebug.obj
 0001:00019f50       sf_debug_set_state_vectors_data 000000018001af50 f   sfc_debug:sfcdebug.obj
 0001:0001a210       sf_debug_get_script_index  000000018001b210 f   sfc_debug:sfcdebug.obj
 0001:0001a3a0       sf_debug_add_script        000000018001b3a0 f   sfc_debug:sfcdebug.obj
 0001:0001a530       cv_eval_point              000000018001b530 f   sfc_debug:sfcdebug.obj
 0001:0001a6a0       cv_eval_testobjective      000000018001b6a0 f   sfc_debug:sfcdebug.obj
 0001:0001a7c0       sf_debug_cv_init_state     000000018001b7c0 f   sfc_debug:sfcdebug.obj
 0001:0001a8e0       sf_debug_cv_init_chart     000000018001b8e0 f   sfc_debug:sfcdebug.obj
 0001:0001a9c0       sf_debug_cv_init_trans     000000018001b9c0 f   sfc_debug:sfcdebug.obj
 0001:0001aac0       sf_debug_cv_init_testobjectives 000000018001bac0 f   sfc_debug:sfcdebug.obj
 0001:0001aca0       cv_eml_init_script         000000018001bca0 f   sfc_debug:sfcdebug.obj
 0001:0001adb0       cv_eml_init_fcn            000000018001bdb0 f   sfc_debug:sfcdebug.obj
 0001:0001ae60       cv_eml_init_testobjective  000000018001be60 f   sfc_debug:sfcdebug.obj
 0001:0001af30       cv_eml_init_saturation     000000018001bf30 f   sfc_debug:sfcdebug.obj
 0001:0001aff0       cv_eml_init_if             000000018001bff0 f   sfc_debug:sfcdebug.obj
 0001:0001b0c0       cv_eml_init_for            000000018001c0c0 f   sfc_debug:sfcdebug.obj
 0001:0001b180       cv_eml_init_while          000000018001c180 f   sfc_debug:sfcdebug.obj
 0001:0001b240       cv_eml_init_mcdc           000000018001c240 f   sfc_debug:sfcdebug.obj
 0001:0001b350       cv_eml_init_switch         000000018001c350 f   sfc_debug:sfcdebug.obj
 0001:0001b440       cv_eml_eval                000000018001c440 f   sfc_debug:sfcdebug.obj
 0001:0001b520       sf_debug_bm_is_a_eml_breakpoint 000000018001c520 f   sfc_debug:sfcdebug.obj
 0001:0001b670       sf_debug_temporal_threshold 000000018001c670 f   sfc_debug:sfcdebug.obj
 0001:0001b9d0       sf_debug_transition_conflict_error 000000018001c9d0 f   sfc_debug:sfcdebug.obj
 0001:0001bd50       sf_debug_state_inconsistency_error 000000018001cd50 f   sfc_debug:sfcdebug.obj
 0001:0001be70       sf_debug_check_for_state_inconsistency 000000018001ce70 f   sfc_debug:sfcdebug.obj
 0001:0001bea0       sf_debug_cycle_detecton_error 000000018001cea0 f   sfc_debug:sfcdebug.obj
 0001:0001c670       sf_debug_size_eq_check_1d  000000018001d670 f   sfc_debug:sfcdebug.obj
 0001:0001c690       sf_debug_size_eq_check_nd  000000018001d690 f   sfc_debug:sfcdebug.obj
 0001:0001c870       sf_debug_dim_size_eq_check 000000018001d870 f   sfc_debug:sfcdebug.obj
 0001:0001c8a0       sf_debug_dim_size_geq_check 000000018001d8a0 f   sfc_debug:sfcdebug.obj
 0001:0001c8d0       sf_debug_sub_assign_size_check_nd 000000018001d8d0 f   sfc_debug:sfcdebug.obj
 0001:0001cb10       sf_debug_matrix_matrix_index_check 000000018001db10 f   sfc_debug:sfcdebug.obj
 0001:0001cb40       sf_debug_vector_vector_index_check 000000018001db40 f   sfc_debug:sfcdebug.obj
 0001:0001cb70       sf_debug_for_loop_vector_check 000000018001db70 f   sfc_debug:sfcdebug.obj
 0001:0001cc00       sf_debug_runtime_error_msgid 000000018001dc00 f   sfc_debug:sfcdebug.obj
 0001:0001cc90       sf_debug_data_array_bounds_error_check 000000018001dc90 f   sfc_debug:sfcdebug.obj
 0001:0001cda0       sf_debug_eml_data_array_bounds_error_check 000000018001dda0 f   sfc_debug:sfcdebug.obj
 0001:0001d280       sf_debug_integer_check     000000018001e280 f   sfc_debug:sfcdebug.obj
 0001:0001d360       sf_debug_not_nan_check     000000018001e360 f   sfc_debug:sfcdebug.obj
 0001:0001d420       sf_debug_non_negative_check 000000018001e420 f   sfc_debug:sfcdebug.obj
 0001:0001d4e0       sf_debug_overflow_detection 000000018001e4e0 f   sfc_debug:sfcdebug.obj
 0001:0001dbd0       sf_debug_cast_to_real32_T  000000018001ebd0 f   sfc_debug:sfcdebug.obj
 0001:0001dc90       sf_debug_cast_to_int8_T    000000018001ec90 f   sfc_debug:sfcdebug.obj
 0001:0001dd50       sf_debug_cast_to_uint8_T   000000018001ed50 f   sfc_debug:sfcdebug.obj
 0001:0001de10       sf_debug_cast_to_int16_T   000000018001ee10 f   sfc_debug:sfcdebug.obj
 0001:0001ded0       sf_debug_cast_to_uint16_T  000000018001eed0 f   sfc_debug:sfcdebug.obj
 0001:0001df90       sf_debug_cast_to_int32_T   000000018001ef90 f   sfc_debug:sfcdebug.obj
 0001:0001e050       sf_debug_cast_to_uint32_T  000000018001f050 f   sfc_debug:sfcdebug.obj
 0001:0001e110       sf_debug_data_range_error  000000018001f110 f   sfc_debug:sfcdebug.obj
 0001:0001e460       sf_debug_read_before_write_check 000000018001f460 f   sfc_debug:sfcdebug.obj
 0001:0001e8c0       sf_debug_data_range_error_wrapper_min_max 000000018001f8c0 f   sfc_debug:sfcdebug.obj
 0001:0001e9b0       sf_debug_data_range_error_wrapper_min 000000018001f9b0 f   sfc_debug:sfcdebug.obj
 0001:0001ea90       sf_debug_data_range_error_wrapper_max 000000018001fa90 f   sfc_debug:sfcdebug.obj
 0001:0001eb70       sf_debug_data_range_wrapper 000000018001fb70 f   sfc_debug:sfcdebug.obj
 0001:0001ec20       sf_debug_set_current_status_info 000000018001fc20 f   sfc_debug:sfcdebug.obj
 0001:0001efd0       sf_debug_register_message_post_receive_info 000000018001ffd0 f   sfc_debug:sfcdebug.obj
 0001:0001f240       sf_debug_call              0000000180020240 f   sfc_debug:sfcdebug.obj
 0001:0001fea0       sf_debug_initialize_machine 0000000180020ea0 f   sfc_debug:sfcdebug.obj
 0001:000201b0       sf_debug_initialize_chart  00000001800211b0 f   sfc_debug:sfcdebug.obj
 0001:00020600       sf_debug_ensure_script     0000000180021600 f   sfc_debug:sfcdebug.obj
 0001:000206c0       cv_script_init_script      00000001800216c0 f   sfc_debug:sfcdebug.obj
 0001:000207b0       cv_script_init_fcn         00000001800217b0 f   sfc_debug:sfcdebug.obj
 0001:00020860       cv_script_init_testobjective 0000000180021860 f   sfc_debug:sfcdebug.obj
 0001:00020910       cv_script_init_if          0000000180021910 f   sfc_debug:sfcdebug.obj
 0001:000209c0       cv_script_init_for         00000001800219c0 f   sfc_debug:sfcdebug.obj
 0001:00020a70       cv_script_init_while       0000000180021a70 f   sfc_debug:sfcdebug.obj
 0001:00020b20       cv_script_init_mcdc        0000000180021b20 f   sfc_debug:sfcdebug.obj
 0001:00020c20       cv_script_init_switch      0000000180021c20 f   sfc_debug:sfcdebug.obj
 0001:00020d00       cv_script_eval             0000000180021d00 f   sfc_debug:sfcdebug.obj
 0001:00020de0       eml_debug_line_call        0000000180021de0 f   sfc_debug:sfcdebug.obj
 0001:00020f90       sf_debug_terminate         0000000180021f90 f   sfc_debug:sfcdebug.obj
 0001:00021100       sf_debug_set_script_cv_ids 0000000180022100 f   sfc_debug:sfcdebug.obj
 0001:00021230       sf_debug_api               0000000180022230 f   sfc_debug:sfc_api.obj
 0001:000228e0       sf_debug_sm_terminate      00000001800238e0 f   sfc_debug:sfdb_animation.obj
 0001:00022aa0       sf_debug_reset_path_objects 0000000180023aa0 f   sfc_debug:sfdb_animation.obj
 0001:00022b20       sf_debug_sm_reset_object_selection_status 0000000180023b20 f   sfc_debug:sfdb_animation.obj
 0001:00022bc0       sf_debug_sm_reset_state_buffer 0000000180023bc0 f   sfc_debug:sfdb_animation.obj
 0001:00022c90       sf_debug_sm_store_state_buffer 0000000180023c90 f   sfc_debug:sfdb_animation.obj
 0001:00022d10       sf_debug_sm_restore_state_buffer1 0000000180023d10 f   sfc_debug:sfdb_animation.obj
 0001:00022d80       sf_debug_sm_restore_state_buffer2 0000000180023d80 f   sfc_debug:sfdb_animation.obj
 0001:00022df0       sf_debug_sm_chart_active   0000000180023df0 f   sfc_debug:sfdb_animation.obj
 0001:00022e40       sf_debug_sm_select_active_objects 0000000180023e40 f   sfc_debug:sfdb_animation.obj
 0001:00023330       sf_debug_sm_is_chart_active 0000000180024330 f   sfc_debug:sfdb_animation.obj
 0001:00023370       sf_debug_sm_is_state_active 0000000180024370 f   sfc_debug:sfdb_animation.obj
 0001:000235b0       sf_debug_sm_get_active_states 00000001800245b0 f   sfc_debug:sfdb_animation.obj
 0001:00023b70       sf_debug_sm_initialize_instance 0000000180024b70 f   sfc_debug:sfdb_animation.obj
 0001:00023d90       sf_debug_sm_change_object_selection_status 0000000180024d90 f   sfc_debug:sfdb_animation.obj
 0001:000240a0       cv_create_interface        00000001800250a0 f   sfc_debug:cv_sfinterface.obj
 0001:00024400       cv_init_trans              0000000180025400 f   sfc_debug:cv_sfinterface.obj
 0001:00024450       cv_init_testobjective      0000000180025450 f   sfc_debug:cv_sfinterface.obj
 0001:00024490       cv_init_state              0000000180025490 f   sfc_debug:cv_sfinterface.obj
 0001:00024500       cv_init_chart              0000000180025500 f   sfc_debug:cv_sfinterface.obj
 0001:00024550       cv_dec_update_call         0000000180025550 f   sfc_debug:cv_sfinterface.obj
 0001:00024590       cv_cond_update_call        0000000180025590 f   sfc_debug:cv_sfinterface.obj
 0001:000245d0       cv_testobjective_update_call 00000001800255d0 f   sfc_debug:cv_sfinterface.obj
 0001:00024610       cv_sigrange_update         0000000180025610 f   sfc_debug:cv_sfinterface.obj
 0001:00024650       cvsf_eml_eval              0000000180025650 f   sfc_debug:cv_sfinterface.obj
 0001:00024740       cvsf_eml_init_script       0000000180025740 f   sfc_debug:cv_sfinterface.obj
 0001:000247d0       cvsf_eml_init_fcn          00000001800257d0 f   sfc_debug:cv_sfinterface.obj
 0001:00024830       cvsf_eml_init_testobjective 0000000180025830 f   sfc_debug:cv_sfinterface.obj
 0001:00024890       cvsf_eml_init_saturation   0000000180025890 f   sfc_debug:cv_sfinterface.obj
 0001:000248e0       cvsf_eml_init_if           00000001800258e0 f   sfc_debug:cv_sfinterface.obj
 0001:00024940       cvsf_eml_init_for          0000000180025940 f   sfc_debug:cv_sfinterface.obj
 0001:00024990       cvsf_eml_init_while        0000000180025990 f   sfc_debug:cv_sfinterface.obj
 0001:000249e0       cvsf_eml_init_mcdc         00000001800259e0 f   sfc_debug:cv_sfinterface.obj
 0001:00024a70       cvsf_eml_init_switch       0000000180025a70 f   sfc_debug:cv_sfinterface.obj
 0001:00024ae0       cvsf_script_eval           0000000180025ae0 f   sfc_debug:cv_sfinterface.obj
 0001:00024bd0       cvsf_script_init_script    0000000180025bd0 f   sfc_debug:cv_sfinterface.obj
 0001:00024c60       cvsf_script_init_fcn       0000000180025c60 f   sfc_debug:cv_sfinterface.obj
 0001:00024cc0       cvsf_script_init_testobjective 0000000180025cc0 f   sfc_debug:cv_sfinterface.obj
 0001:00024d20       cvsf_script_init_saturation 0000000180025d20 f   sfc_debug:cv_sfinterface.obj
 0001:00024d70       cvsf_script_init_if        0000000180025d70 f   sfc_debug:cv_sfinterface.obj
 0001:00024dd0       cvsf_script_init_for       0000000180025dd0 f   sfc_debug:cv_sfinterface.obj
 0001:00024e20       cvsf_script_init_while     0000000180025e20 f   sfc_debug:cv_sfinterface.obj
 0001:00024e70       cvsf_script_init_mcdc      0000000180025e70 f   sfc_debug:cv_sfinterface.obj
 0001:00024f00       cvsf_script_init_switch    0000000180025f00 f   sfc_debug:cv_sfinterface.obj
 0001:00024f70       cv_destroy_interface       0000000180025f70 f   sfc_debug:cv_sfinterface.obj
 0001:00024f90       cv_create_instance_objects 0000000180025f90 f   sfc_debug:cv_sfinterface.obj
 0001:00025440       cv_is_enabled              0000000180026440 f   sfc_debug:cv_sfinterface.obj
 0001:00025450       sf_debug_cv_initialize_script 0000000180026450 f   sfc_debug:cv_sfinterface.obj
 0001:00025600       sf_debug_cv_initialize_instance 0000000180026600 f   sfc_debug:cv_sfinterface.obj
 0001:000259a0       sf_debug_cv_terminate_chart 00000001800269a0 f   sfc_debug:cv_sfinterface.obj
 0001:00025ae0       cv_call_trans_test         0000000180026ae0 f   sfc_debug:cv_sfinterface.obj
 0001:00025af0       cv_call_sub_cond_test      0000000180026af0 f   sfc_debug:cv_sfinterface.obj
 0001:00025b30       sf_debug_st_initialize_machine 0000000180026b30 f   sfc_debug:sfdb_data_browse.obj
 0001:00025bf0       sf_debug_st_initialize_instance 0000000180026bf0 f   sfc_debug:sfdb_data_browse.obj
 0001:00025e20       sf_debug_st_terminate      0000000180026e20 f   sfc_debug:sfdb_data_browse.obj
 0001:000261c0       sf_debug_st_set_data_value_ptr_in_machine 00000001800271c0 f   sfc_debug:sfdb_data_browse.obj
 0001:00026250       sf_debug_st_set_data_value_ptr_in_instance 0000000180027250 f   sfc_debug:sfdb_data_browse.obj
 0001:00026330       sf_debug_st_unset_data_value_ptr_in_machine 0000000180027330 f   sfc_debug:sfdb_data_browse.obj
 0001:000263a0       sf_debug_st_unset_data_value_ptr_in_instance 00000001800273a0 f   sfc_debug:sfdb_data_browse.obj
 0001:000266b0       sf_debug_mx_value          00000001800276b0 f   sfc_debug:sfdb_data_browse.obj
 0001:00026710       sf_debug_mx_packed_vector  0000000180027710 f   sfc_debug:sfdb_data_browse.obj
 0001:000267f0       sf_debug_mx_uint_vector    00000001800277f0 f   sfc_debug:sfdb_data_browse.obj
 0001:000268b0       sf_debug_st_get_double_value_from_void_ptr_vector 00000001800278b0 f   sfc_debug:sfdb_data_browse.obj
 0001:000273a0       sf_debug_st_browse_data    00000001800283a0 f   sfc_debug:sfdb_data_browse.obj
 0001:00027c30       sf_debug_hm_initialize_instance 0000000180028c30 f   sfc_debug:sfdb_handle_management.obj
 0001:00028160       sf_debug_hm_get_object_id  0000000180029160 f   sfc_debug:sfdb_handle_management.obj
 0001:00028d10       sf_debug_hm_update_chart_visibility 0000000180029d10 f   sfc_debug:sfdb_handle_management.obj
 0001:00029ff0       sf_debug_object_is_eml_function 000000018002aff0 f   sfc_debug:sfdb_handle_management.obj
 0001:0002a060       sf_debug_hm_initialize_ids_in_machine 000000018002b060 f   sfc_debug:sfdb_handle_management.obj
 0001:0002a1d0       sf_debug_hm_initialize_ids_in_chart 000000018002b1d0 f   sfc_debug:sfdb_handle_management.obj
 0001:0002a2d0       sf_debug_hm_initialize_chart 000000018002b2d0 f   sfc_debug:sfdb_handle_management.obj
 0001:0002aa70       sf_debug_hm_terminate      000000018002ba70 f   sfc_debug:sfdb_handle_management.obj
 0001:0002aad0       sf_debug_hm_initialize_machine 000000018002bad0 f   sfc_debug:sfdb_handle_management.obj
 0001:0002b280       sf_debug_ss_initialize     000000018002c280 f   sfc_debug:sfdb_symbol_scope.obj
 0001:0002b2a0       sf_debug_ss_terminate      000000018002c2a0 f   sfc_debug:sfdb_symbol_scope.obj
 0001:0002b330       sf_debug_ss_push_symbol_scope 000000018002c330 f   sfc_debug:sfdb_symbol_scope.obj
 0001:0002b430       sf_debug_ss_push_symbol_scope_eml 000000018002c430 f   sfc_debug:sfdb_symbol_scope.obj
 0001:0002b490       sf_debug_ss_pop_symbol_scope 000000018002c490 f   sfc_debug:sfdb_symbol_scope.obj
 0001:0002b540       sf_debug_ss_add_symbol     000000018002c540 f   sfc_debug:sfdb_symbol_scope.obj
 0001:0002b6a0       sf_debug_ss_add_symbol_eml 000000018002c6a0 f   sfc_debug:sfdb_symbol_scope.obj
 0001:0002c3c0       sf_debug_ss_set_data_value 000000018002d3c0 f   sfc_debug:sfdb_symbol_scope.obj
 0001:0002c890       getInstanceNumber          000000018002d890 f   sfc_debug:sfdb_symbol_scope.obj
 0001:0002c960       sf_debug_ss_watch_data     000000018002d960 f   sfc_debug:sfdb_symbol_scope.obj
 0001:0002cb00       sf_debug_ss_assign_data    000000018002db00 f   sfc_debug:sfdb_symbol_scope.obj
 0001:0002d520       get_data_entry_name        000000018002e520 f   sfc_debug:sfdb_symbol_scope.obj
 0001:0002d570       sf_debug_ss_whos           000000018002e570 f   sfc_debug:sfdb_symbol_scope.obj
 0001:0002dc90       sf_debug_cc_initialize_chart 000000018002ec90 f   sfc_debug:sfdb_coverage.obj
 0001:0002e680       sf_debug_cc_initialize_instance 000000018002f680 f   sfc_debug:sfdb_coverage.obj
 0001:0002f490       sf_debug_cc_terminate      0000000180030490 f   sfc_debug:sfdb_coverage.obj
 0001:0002f580       sf_debug_cc_set_transition_maps 0000000180030580 f   sfc_debug:sfdb_coverage.obj
 0001:0002f6b0       sf_debug_cc_set_state_maps 00000001800306b0 f   sfc_debug:sfdb_coverage.obj
 0001:0002f790       sf_debug_cc_set_transition_weights 0000000180030790 f   sfc_debug:sfdb_coverage.obj
 0001:0002fa60       sf_debug_cc_set_state_weights 0000000180030a60 f   sfc_debug:sfdb_coverage.obj
 0001:0002fd30       sf_debug_cc_mark_transition_guard 0000000180030d30 f   sfc_debug:sfdb_coverage.obj
 0001:0002fdc0       sf_debug_cc_mark_transition_trigger 0000000180030dc0 f   sfc_debug:sfdb_coverage.obj
 0001:0002fe50       sf_debug_cc_mark_transition_decision 0000000180030e50 f   sfc_debug:sfdb_coverage.obj
 0001:0002fec0       sf_debug_cc_mark_transition_condition_action 0000000180030ec0 f   sfc_debug:sfdb_coverage.obj
 0001:0002ff10       sf_debug_cc_mark_transition_transition_action 0000000180030f10 f   sfc_debug:sfdb_coverage.obj
 0001:0002ff60       sf_debug_cc_mark_state_entry 0000000180030f60 f   sfc_debug:sfdb_coverage.obj
 0001:0002ffb0       sf_debug_cc_mark_state_during 0000000180030fb0 f   sfc_debug:sfdb_coverage.obj
 0001:00030000       sf_debug_cc_mark_state_exit 0000000180031000 f   sfc_debug:sfdb_coverage.obj
 0001:00030050       sf_debug_bm_clear_script_breakpoints 0000000180031050 f   sfc_debug:sfdb_breakpoints.obj
 0001:00030080       sf_debug_bm_set_script_breakpoint 0000000180031080 f   sfc_debug:sfdb_breakpoints.obj
 0001:00030100       sf_debug_bm_clear_single_script_breakpoint 0000000180031100 f   sfc_debug:sfdb_breakpoints.obj
 0001:00030180       sf_debug_bm_query_script_breakpoint 0000000180031180 f   sfc_debug:sfdb_breakpoints.obj
 0001:000301d0       sf_debug_bm_initialize_scripts 00000001800311d0 f   sfc_debug:sfdb_breakpoints.obj
 0001:000308f0       sf_debug_bm_terminate      00000001800318f0 f   sfc_debug:sfdb_breakpoints.obj
 0001:00030be0       sf_debug_bm_remove_all_breakpoints_in_machine 0000000180031be0 f   sfc_debug:sfdb_breakpoints.obj
 0001:00030c50       sf_debug_bm_remove_all_breakpoints_in_chart 0000000180031c50 f   sfc_debug:sfdb_breakpoints.obj
 0001:00030da0       sf_debug_bm_initialize_global_breakpoints 0000000180031da0 f   sfc_debug:sfdb_breakpoints.obj
 0001:00030f20       sf_debug_bm_set_breakpoint 0000000180031f20 f   sfc_debug:sfdb_breakpoints.obj
 0001:00031520       sf_debug_bm_set_eml_breakpoint 0000000180032520 f   sfc_debug:sfdb_breakpoints.obj
 0001:000315c0       sf_debug_bm_initialize_machine_breakpoint_map 00000001800325c0 f   sfc_debug:sfdb_breakpoints.obj
 0001:000319e0       sf_debug_bm_is_a_breakpoint 00000001800329e0 f   sfc_debug:sfdb_breakpoints.obj
 0001:00031fc0       sf_debug_bm_get_all_breakpoints_in_machine 0000000180032fc0 f   sfc_debug:sfdb_breakpoints.obj
 0001:000322c0       sf_debug_bm_get_all_breakpoints_in_chart 00000001800332c0 f   sfc_debug:sfdb_breakpoints.obj
 0001:00032f80       sf_debug_bm_initialize_machine 0000000180033f80 f   sfc_debug:sfdb_breakpoints.obj
 0001:00033050       sf_debug_bm_initialize_chart 0000000180034050 f   sfc_debug:sfdb_breakpoints.obj
 0001:00033470       sf_debug_sc_terminate      0000000180034470 f   sfc_debug:sfdb_state_consistency.obj
 0001:000337a0       sf_debug_sc_is_chart_consistent 00000001800347a0 f   sfc_debug:sfdb_state_consistency.obj
 0001:00033a50       sf_debug_sc_get_consistency_error_info 0000000180034a50 f   sfc_debug:sfdb_state_consistency.obj
 0001:00033ea0       sf_debug_tm_terminate      0000000180034ea0 f   sfc_debug:sfdb_call_stack.obj
 0001:00033f60       sf_debug_tm_push_chart_instance 0000000180034f60 f   sfc_debug:sfdb_call_stack.obj
 0001:000340b0       sf_debug_tm_pop_chart_instance 00000001800350b0 f   sfc_debug:sfdb_call_stack.obj
 0001:00034110       sf_debug_tm_push_trace_node 0000000180035110 f   sfc_debug:sfdb_call_stack.obj
 0001:000342a0       sf_debug_tm_pop_trace_node 00000001800352a0 f   sfc_debug:sfdb_call_stack.obj
 0001:00034320       sf_debug_tm_get_current_global_trace_index 0000000180035320 f   sfc_debug:sfdb_call_stack.obj
 0001:00034330       sf_debug_tm_get_current_local_trace_index 0000000180035330 f   sfc_debug:sfdb_call_stack.obj
 0001:00034360       sf_debug_tm_set_cycle_detected_flag 0000000180035360 f   sfc_debug:sfdb_call_stack.obj
 0001:000343a0       sf_debug_tm_set_cycle_started_flag 00000001800353a0 f   sfc_debug:sfdb_call_stack.obj
 0001:000343e0       sf_debug_tm_get_chart_number_from_stack 00000001800353e0 f   sfc_debug:sfdb_call_stack.obj
 0001:000345e0       sf_debug_tm_browse_trace   00000001800355e0 f   sfc_debug:sfdb_call_stack.obj
 0001:00034920       sf_debug_cd_initialize_instance 0000000180035920 f   sfc_debug:sfdb_cycle_detection.obj
 0001:00034bd0       sf_debug_cd_mark_processed_transition_in_instance 0000000180035bd0 f   sfc_debug:sfdb_cycle_detection.obj
 0001:00034c70       sf_debug_cd_checksum_push  0000000180035c70 f   sfc_debug:sfdb_cycle_detection.obj
 0001:00034f30       sf_debug_cd_checksum_pop   0000000180035f30 f   sfc_debug:sfdb_cycle_detection.obj
 0001:00034fa0       sf_debug_cd_turn_off_cycle_detection 0000000180035fa0 f   sfc_debug:sfdb_cycle_detection.obj
 0001:00034ff0       sf_debug_cd_terminate      0000000180035ff0 f   sfc_debug:sfdb_cycle_detection.obj
 0001:00035230       md5_initialize_state       0000000180036230 f   sfc_debug:ckmd5.obj
 0001:00035ca0       md5_update_state           0000000180036ca0 f   sfc_debug:ckmd5.obj
 0001:00035cc0       md5_get_hash               0000000180036cc0 f   sfc_debug:ckmd5.obj
 0001:00035cf0       md5_get_hash_for_a_single_string 0000000180036cf0 f   sfc_debug:ckmd5.obj
 0001:00035d54       mxGetPr                    0000000180036d54 f   libmx:libmx.dll
 0001:00035d5a       mxCreateDoubleScalar       0000000180036d5a f   libmx:libmx.dll
 0001:00035d60       mxCreateDoubleMatrix_730   0000000180036d60 f   libmx:libmx.dll
 0001:00035d66       mxSetField_730             0000000180036d66 f   libmx:libmx.dll
 0001:00035d6c       mxCreateString             0000000180036d6c f   libmx:libmx.dll
 0001:00035d72       mxCreateStructMatrix_730   0000000180036d72 f   libmx:libmx.dll
 0001:00035d78       mxDestroyArray             0000000180036d78 f   libmx:libmx.dll
 0001:00035d7e       mxDuplicateArray           0000000180036d7e f   libmx:libmx.dll
 0001:00035d84       mxGetString_730            0000000180036d84 f   libmx:libmx.dll
 0001:00035d8a       mxIsChar                   0000000180036d8a f   libmx:libmx.dll
 0001:00035d90       mxGetClassID               0000000180036d90 f   libmx:libmx.dll
 0001:00035d96       mxIsNumeric                0000000180036d96 f   libmx:libmx.dll
 0001:00035d9c       mxIsComplex                0000000180036d9c f   libmx:libmx.dll
 0001:00035da2       mxGetN                     0000000180036da2 f   libmx:libmx.dll
 0001:00035da8       mxGetM                     0000000180036da8 f   libmx:libmx.dll
 0001:00035dae       mxCalloc                   0000000180036dae f   libmx:libmx.dll
 0001:00035db4       mxGetScalar                0000000180036db4 f   libmx:libmx.dll
 0001:00035dba       mxIsLogical                0000000180036dba f   libmx:libmx.dll
 0001:00035dc0       mxCreateDoubleMatrix_700   0000000180036dc0 f   libmx:libmx.dll
 0001:00035dc6       mxFree                     0000000180036dc6 f   libmx:libmx.dll
 0001:00035dcc       mxArrayToString            0000000180036dcc f   libmx:libmx.dll
 0001:00035dd2       mxCreateCellMatrix_700     0000000180036dd2 f   libmx:libmx.dll
 0001:00035dd8       mxSetCell_700              0000000180036dd8 f   libmx:libmx.dll
 0001:00035dde       mxGetCell_700              0000000180036dde f   libmx:libmx.dll
 0001:00035de4       mxGetClassName             0000000180036de4 f   libmx:libmx.dll
 0001:00035dea       mxSetField_700             0000000180036dea f   libmx:libmx.dll
 0001:00035df0       mxAddField                 0000000180036df0 f   libmx:libmx.dll
 0001:00035df6       mxGetField_700             0000000180036df6 f   libmx:libmx.dll
 0001:00035dfc       mxGetNumberOfElements      0000000180036dfc f   libmx:libmx.dll
 0001:00035e02       mxIsStruct                 0000000180036e02 f   libmx:libmx.dll
 0001:00035e08       mxIsA                      0000000180036e08 f   libmx:libmx.dll
 0001:00035e0e       mxIsClass                  0000000180036e0e f   libmx:libmx.dll
 0001:00035e14       mxGetLogicals              0000000180036e14 f   libmx:libmx.dll
 0001:00035e1a       mxIsSparse                 0000000180036e1a f   libmx:libmx.dll
 0001:00035e20       mxSetFieldByNumber_700     0000000180036e20 f   libmx:libmx.dll
 0001:00035e26       mxGetFieldByNumber_700     0000000180036e26 f   libmx:libmx.dll
 0001:00035e2c       mxGetFieldNameByNumber     0000000180036e2c f   libmx:libmx.dll
 0001:00035e32       mxGetNumberOfFields        0000000180036e32 f   libmx:libmx.dll
 0001:00035e38       mxCreateStructMatrix_700   0000000180036e38 f   libmx:libmx.dll
 0001:00035e3e       mxGetFieldNumber           0000000180036e3e f   libmx:libmx.dll
 0001:00035e44       mxIsNaN                    0000000180036e44 f   libmx:libmx.dll
 0001:00035e4a       mxIsEmpty                  0000000180036e4a f   libmx:libmx.dll
 0001:00035e50       mxGetData                  0000000180036e50 f   libmx:libmx.dll
 0001:00035e56       mxGetImagData              0000000180036e56 f   libmx:libmx.dll
 0001:00035e5c       mxArrayClassIDName         0000000180036e5c f   libmx:libmx.dll
 0001:00035e62       mxCreateNumericMatrix_700  0000000180036e62 f   libmx:libmx.dll
 0001:00035e68       mxCreateStructArray_700    0000000180036e68 f   libmx:libmx.dll
 0001:00035e6e       mxCalcSingleSubscript_700  0000000180036e6e f   libmx:libmx.dll
 0001:00035e74       mxGetDimensions_700        0000000180036e74 f   libmx:libmx.dll
 0001:00035e7a       mxGetNumberOfDimensions_700 0000000180036e7a f   libmx:libmx.dll
 0001:00035e80       mxCreateNumericArray_700   0000000180036e80 f   libmx:libmx.dll
 0001:00035e86       mxGetElementSize           0000000180036e86 f   libmx:libmx.dll
 0001:00035e8c       mxCreateStringFromNChars_700 0000000180036e8c f   libmx:libmx.dll
 0001:00035e92       mxGetString_700            0000000180036e92 f   libmx:libmx.dll
 0001:00035e98       mxIsLogicalScalarTrue      0000000180036e98 f   libmx:libmx.dll
 0001:00035e9e       mxCreateLogicalScalar      0000000180036e9e f   libmx:libmx.dll
 0001:00035ea4       mexUnlock                  0000000180036ea4 f   libmex:libmex.dll
 0001:00035eaa       mexIsLocked                0000000180036eaa f   libmex:libmex.dll
 0001:00035eb0       mexWarnMsgTxt              0000000180036eb0 f   libmex:libmex.dll
 0001:00035eb6       mexCallMATLAB              0000000180036eb6 f   libmex:libmex.dll
 0001:00035ebc       mexErrMsgTxt               0000000180036ebc f   libmex:libmex.dll
 0001:00035ec2       mexMakeArrayPersistent     0000000180036ec2 f   libmex:libmex.dll
 0001:00035ec8       mexSetTrapFlag             0000000180036ec8 f   libmex:libmex.dll
 0001:00035ece       mexPutVariable             0000000180036ece f   libmex:libmex.dll
 0001:00035ed4       mexGetVariable             0000000180036ed4 f   libmex:libmex.dll
 0001:00035eda       mexLock                    0000000180036eda f   libmex:libmex.dll
 0001:00035ee0       mexMakeMemoryPersistent    0000000180036ee0 f   libmex:libmex.dll
 0001:00035ee6       mexFunctionName            0000000180036ee6 f   libmex:libmex.dll
 0001:00035eec       ssRegisterDataTypeFxpFSlopeFixExpBias 0000000180036eec f   libfixedpoint:libfixedpoint.dll
 0001:00035ef2       utVSNprintf                0000000180036ef2 f   libut:libut.dll
 0001:00035ef8       utCPUtime                  0000000180036ef8 f   libut:libut.dll
 0001:00035efe       utFree                     0000000180036efe f   libut:libut.dll
 0001:00035f04       utMalloc                   0000000180036f04 f   libut:libut.dll
 0001:00035f0a       emlrtCreateRootTLS         0000000180036f0a f   libemlrt:libemlrt.dll
 0001:00035f10       emlrtDestroyRootTLS        0000000180036f10 f   libemlrt:libemlrt.dll
 0001:00035f16       emlrtCheckBuiltInR2012b    0000000180036f16 f   libemlrt:libemlrt.dll
 0001:00035f1c       emlrtCheckVsBuiltInR2012b  0000000180036f1c f   libemlrt:libemlrt.dll
 0001:00035f22       emlrtCheckEnumR2012b       0000000180036f22 f   libemlrt:libemlrt.dll
 0001:00035f28       emlrtCreateEnumR2012b      0000000180036f28 f   libemlrt:libemlrt.dll
 0001:00035f2e       emlrtGetEnumElementR2009a  0000000180036f2e f   libemlrt:libemlrt.dll
 0001:00035f34       emlrtCreateReference       0000000180036f34 f   libemlrt:libemlrt.dll
 0001:00035f3a       emlrtImportVsFiArrayR2009b 0000000180036f3a f   libemlrt:libemlrt.dll
 0001:00035f40       emlrtNameCapturePostProcessR2012a 0000000180036f40 f   libemlrt:libemlrt.dll
 0001:00035f46       emlrtExtractMessageId      0000000180036f46 f   libemlrt:libemlrt.dll
 0001:00035f4c       emlrtTranslateMessageIDtoLCPstring 0000000180036f4c f   libemlrt:libemlrt.dll
 0001:00035f52       emlrtForLoopVectorIsValidR2011b 0000000180036f52 f   libemlrt:libemlrt.dll
 0001:00035f58       emlrtTranslateUTF16MessagetoLCPstring 0000000180036f58 f   libemlrt:libemlrt.dll
 0001:00035f5e       emlrtGetEnumUnderlyingArrayR2009a 0000000180036f5e f   libemlrt:libemlrt.dll
 0001:00035f64       emlrtIsEnumR2009a          0000000180036f64 f   libemlrt:libemlrt.dll
 0001:00035f6a       strlen                     0000000180036f6a f   MSVCRT:MSVCR100.dll
 0001:00035f70       memset                     0000000180036f70 f   MSVCRT:MSVCR100.dll
 0001:00035f76       malloc                     0000000180036f76 f   MSVCRT:MSVCR100.dll
 0001:00035f7c       __GSHandlerCheckCommon     0000000180036f7c f   MSVCRT:gshandler.obj
 0001:00035fe0       __GSHandlerCheck           0000000180036fe0 f   MSVCRT:gshandler.obj
 0001:00036010       __security_check_cookie    0000000180037010 f   MSVCRT:amdsecgs.obj
 0001:00036030       free                       0000000180037030 f   MSVCRT:MSVCR100.dll
 0001:00036036       strcmp                     0000000180037036 f   MSVCRT:MSVCR100.dll
 0001:0003603c       sprintf                    000000018003703c f   MSVCRT:MSVCR100.dll
 0001:00036042       strcat                     0000000180037042 f   MSVCRT:MSVCR100.dll
 0001:00036048       memcpy                     0000000180037048 f   MSVCRT:MSVCR100.dll
 0001:00036050       NtCurrentTeb               0000000180037050 f i MSVCRT:crtdll.obj
 0001:000360bc       _CRT_INIT                  00000001800370bc f   MSVCRT:crtdll.obj
 0001:00036454       _DllMainCRTStartup         0000000180037454 f   MSVCRT:crtdll.obj
 0001:00036492       strncpy                    0000000180037492 f   MSVCRT:MSVCR100.dll
 0001:000364b0       _alloca_probe              00000001800374b0     MSVCRT:chkstk.obj
 0001:000364b0       __chkstk                   00000001800374b0 f   MSVCRT:chkstk.obj
 0001:000364fe       longjmp                    00000001800374fe f   MSVCRT:MSVCR100.dll
 0001:00036504       strncmp                    0000000180037504 f   MSVCRT:MSVCR100.dll
 0001:0003650a       ceil                       000000018003750a f   MSVCRT:MSVCR100.dll
 0001:00036510       strrchr                    0000000180037510 f   MSVCRT:MSVCR100.dll
 0001:00036516       _setjmp                    0000000180037516 f   MSVCRT:MSVCR100.dll
 0001:0003651c       calloc                     000000018003751c f   MSVCRT:MSVCR100.dll
 0001:00036522       realloc                    0000000180037522 f   MSVCRT:MSVCR100.dll
 0001:00036528       ldexp                      0000000180037528 f   MSVCRT:MSVCR100.dll
 0001:00036530       __report_gsfailure         0000000180037530 f   MSVCRT:gs_report.obj
 0001:0003667c       __clean_type_info_names    000000018003767c f   MSVCRT:tncleanup.obj
 0001:00036688       _onexit                    0000000180037688 f   MSVCRT:atonexit.obj
 0001:00036738       atexit                     0000000180037738 f   MSVCRT:atonexit.obj
 0001:00036750       _RTC_Initialize            0000000180037750 f   MSVCRT:_initsect_.obj
 0001:00036788       _RTC_Terminate             0000000180037788 f   MSVCRT:_initsect_.obj
 0001:000367c0       _malloc_crt                00000001800377c0 f   MSVCRT:MSVCR100.dll
 0001:000367d0       _ValidateImageBase         00000001800377d0 f   MSVCRT:pesect.obj
 0001:00036800       _FindPESection             0000000180037800 f   MSVCRT:pesect.obj
 0001:00036850       _IsNonwritableInCurrentImage 0000000180037850 f   MSVCRT:pesect.obj
 0001:00036892       _initterm                  0000000180037892 f   MSVCRT:MSVCR100.dll
 0001:00036898       _initterm_e                0000000180037898 f   MSVCRT:MSVCR100.dll
 0001:0003689e       _encoded_null              000000018003789e f   MSVCRT:MSVCR100.dll
 0001:000368a4       _amsg_exit                 00000001800378a4 f   MSVCRT:MSVCR100.dll
 0001:000368aa       __C_specific_handler       00000001800378aa f   MSVCRT:MSVCR100.dll
 0001:000368b0       __CppXcptFilter            00000001800378b0 f   MSVCRT:MSVCR100.dll
 0001:000368b8       DllMain                    00000001800378b8 f   MSVCRT:dllmain.obj
 0001:000368dc       __security_init_cookie     00000001800378dc f   MSVCRT:gs_support.obj
 0001:00036990       __crt_debugger_hook        0000000180037990 f   MSVCRT:MSVCR100.dll
 0001:00036996       __clean_type_info_names_internal 0000000180037996 f   MSVCRT:MSVCR100.dll
 0001:0003699c       _unlock                    000000018003799c f   MSVCRT:MSVCR100.dll
 0001:000369a2       __dllonexit                00000001800379a2 f   MSVCRT:MSVCR100.dll
 0001:000369a8       _lock                      00000001800379a8 f   MSVCRT:MSVCR100.dll
 0001:000369ae       EncodePointer              00000001800379ae f   kernel32:KERNEL32.dll
 0001:000369b4       DecodePointer              00000001800379b4 f   kernel32:KERNEL32.dll
 0001:000369ba       Sleep                      00000001800379ba f   kernel32:KERNEL32.dll
 0001:000369c0       TerminateProcess           00000001800379c0 f   kernel32:KERNEL32.dll
 0001:000369c6       GetCurrentProcess          00000001800379c6 f   kernel32:KERNEL32.dll
 0001:000369cc       UnhandledExceptionFilter   00000001800379cc f   kernel32:KERNEL32.dll
 0001:000369d2       SetUnhandledExceptionFilter 00000001800379d2 f   kernel32:KERNEL32.dll
 0001:000369d8       IsDebuggerPresent          00000001800379d8 f   kernel32:KERNEL32.dll
 0001:000369de       RtlVirtualUnwind           00000001800379de f   kernel32:KERNEL32.dll
 0001:000369e4       RtlLookupFunctionEntry     00000001800379e4 f   kernel32:KERNEL32.dll
 0001:000369ea       RtlCaptureContext          00000001800379ea f   kernel32:KERNEL32.dll
 0001:000369f0       DisableThreadLibraryCalls  00000001800379f0 f   kernel32:KERNEL32.dll
 0001:000369f6       QueryPerformanceCounter    00000001800379f6 f   kernel32:KERNEL32.dll
 0001:000369fc       GetTickCount               00000001800379fc f   kernel32:KERNEL32.dll
 0001:00036a02       GetCurrentThreadId         0000000180037a02 f   kernel32:KERNEL32.dll
 0001:00036a08       GetCurrentProcessId        0000000180037a08 f   kernel32:KERNEL32.dll
 0001:00036a0e       GetSystemTimeAsFileTime    0000000180037a0e f   kernel32:KERNEL32.dll
 0002:00000000       __imp_GetSystemTimeAsFileTime 0000000180038000     kernel32:KERNEL32.dll
 0002:00000008       __imp_GetCurrentProcessId  0000000180038008     kernel32:KERNEL32.dll
 0002:00000010       __imp_GetCurrentThreadId   0000000180038010     kernel32:KERNEL32.dll
 0002:00000018       __imp_GetTickCount         0000000180038018     kernel32:KERNEL32.dll
 0002:00000020       __imp_QueryPerformanceCounter 0000000180038020     kernel32:KERNEL32.dll
 0002:00000028       __imp_DisableThreadLibraryCalls 0000000180038028     kernel32:KERNEL32.dll
 0002:00000030       __imp_RtlCaptureContext    0000000180038030     kernel32:KERNEL32.dll
 0002:00000038       __imp_RtlLookupFunctionEntry 0000000180038038     kernel32:KERNEL32.dll
 0002:00000040       __imp_RtlVirtualUnwind     0000000180038040     kernel32:KERNEL32.dll
 0002:00000048       __imp_IsDebuggerPresent    0000000180038048     kernel32:KERNEL32.dll
 0002:00000050       __imp_SetUnhandledExceptionFilter 0000000180038050     kernel32:KERNEL32.dll
 0002:00000058       __imp_UnhandledExceptionFilter 0000000180038058     kernel32:KERNEL32.dll
 0002:00000060       __imp_GetCurrentProcess    0000000180038060     kernel32:KERNEL32.dll
 0002:00000068       __imp_TerminateProcess     0000000180038068     kernel32:KERNEL32.dll
 0002:00000070       __imp_Sleep                0000000180038070     kernel32:KERNEL32.dll
 0002:00000078       __imp_DecodePointer        0000000180038078     kernel32:KERNEL32.dll
 0002:00000080       __imp_EncodePointer        0000000180038080     kernel32:KERNEL32.dll
 0002:00000088       \177KERNEL32_NULL_THUNK_DATA 0000000180038088     kernel32:KERNEL32.dll
 0002:00000090       __imp__onexit              0000000180038090     MSVCRT:MSVCR100.dll
 0002:00000098       __imp__lock                0000000180038098     MSVCRT:MSVCR100.dll
 0002:000000a0       __imp___dllonexit          00000001800380a0     MSVCRT:MSVCR100.dll
 0002:000000a8       __imp__unlock              00000001800380a8     MSVCRT:MSVCR100.dll
 0002:000000b0       __imp___clean_type_info_names_internal 00000001800380b0     MSVCRT:MSVCR100.dll
 0002:000000b8       __imp___crt_debugger_hook  00000001800380b8     MSVCRT:MSVCR100.dll
 0002:000000c0       __imp___CppXcptFilter      00000001800380c0     MSVCRT:MSVCR100.dll
 0002:000000c8       __imp___C_specific_handler 00000001800380c8     MSVCRT:MSVCR100.dll
 0002:000000d0       __imp__amsg_exit           00000001800380d0     MSVCRT:MSVCR100.dll
 0002:000000d8       __imp__encoded_null        00000001800380d8     MSVCRT:MSVCR100.dll
 0002:000000e0       __imp__initterm_e          00000001800380e0     MSVCRT:MSVCR100.dll
 0002:000000e8       __imp__initterm            00000001800380e8     MSVCRT:MSVCR100.dll
 0002:000000f0       __imp__malloc_crt          00000001800380f0     MSVCRT:MSVCR100.dll
 0002:000000f8       __imp_ldexp                00000001800380f8     MSVCRT:MSVCR100.dll
 0002:00000100       __imp_realloc              0000000180038100     MSVCRT:MSVCR100.dll
 0002:00000108       __imp_calloc               0000000180038108     MSVCRT:MSVCR100.dll
 0002:00000110       __imp__setjmp              0000000180038110     MSVCRT:MSVCR100.dll
 0002:00000118       __imp_strrchr              0000000180038118     MSVCRT:MSVCR100.dll
 0002:00000120       __imp_ceil                 0000000180038120     MSVCRT:MSVCR100.dll
 0002:00000128       __imp_strncmp              0000000180038128     MSVCRT:MSVCR100.dll
 0002:00000130       __imp_longjmp              0000000180038130     MSVCRT:MSVCR100.dll
 0002:00000138       __imp_strncpy              0000000180038138     MSVCRT:MSVCR100.dll
 0002:00000140       __imp_memcpy               0000000180038140     MSVCRT:MSVCR100.dll
 0002:00000148       __imp_strcat               0000000180038148     MSVCRT:MSVCR100.dll
 0002:00000150       __imp_sprintf              0000000180038150     MSVCRT:MSVCR100.dll
 0002:00000158       __imp_strcmp               0000000180038158     MSVCRT:MSVCR100.dll
 0002:00000160       __imp_free                 0000000180038160     MSVCRT:MSVCR100.dll
 0002:00000168       __imp_malloc               0000000180038168     MSVCRT:MSVCR100.dll
 0002:00000170       __imp_memset               0000000180038170     MSVCRT:MSVCR100.dll
 0002:00000178       __imp_strlen               0000000180038178     MSVCRT:MSVCR100.dll
 0002:00000180       \177MSVCR100_NULL_THUNK_DATA 0000000180038180     MSVCRT:MSVCR100.dll
 0002:00000188       __imp_emlrtIsEnumR2009a    0000000180038188     libemlrt:libemlrt.dll
 0002:00000190       __imp_emlrtGetEnumUnderlyingArrayR2009a 0000000180038190     libemlrt:libemlrt.dll
 0002:00000198       __imp_emlrtTranslateUTF16MessagetoLCPstring 0000000180038198     libemlrt:libemlrt.dll
 0002:000001a0       __imp_emlrtForLoopVectorIsValidR2011b 00000001800381a0     libemlrt:libemlrt.dll
 0002:000001a8       __imp_emlrtTranslateMessageIDtoLCPstring 00000001800381a8     libemlrt:libemlrt.dll
 0002:000001b0       __imp_emlrtExtractMessageId 00000001800381b0     libemlrt:libemlrt.dll
 0002:000001b8       __imp_emlrtNameCapturePostProcessR2012a 00000001800381b8     libemlrt:libemlrt.dll
 0002:000001c0       __imp_emlrtImportVsFiArrayR2009b 00000001800381c0     libemlrt:libemlrt.dll
 0002:000001c8       __imp_emlrtCreateReference 00000001800381c8     libemlrt:libemlrt.dll
 0002:000001d0       __imp_emlrtGetEnumElementR2009a 00000001800381d0     libemlrt:libemlrt.dll
 0002:000001d8       __imp_emlrtCreateEnumR2012b 00000001800381d8     libemlrt:libemlrt.dll
 0002:000001e0       __imp_emlrtCheckEnumR2012b 00000001800381e0     libemlrt:libemlrt.dll
 0002:000001e8       __imp_emlrtCheckVsBuiltInR2012b 00000001800381e8     libemlrt:libemlrt.dll
 0002:000001f0       __imp_emlrtCheckBuiltInR2012b 00000001800381f0     libemlrt:libemlrt.dll
 0002:000001f8       __imp_emlrtDestroyRootTLS  00000001800381f8     libemlrt:libemlrt.dll
 0002:00000200       __imp_emlrtCreateRootTLS   0000000180038200     libemlrt:libemlrt.dll
 0002:00000208       \177libemlrt_NULL_THUNK_DATA 0000000180038208     libemlrt:libemlrt.dll
 0002:00000210       __imp_ssRegisterDataTypeFxpFSlopeFixExpBias 0000000180038210     libfixedpoint:libfixedpoint.dll
 0002:00000218       \177libfixedpoint_NULL_THUNK_DATA 0000000180038218     libfixedpoint:libfixedpoint.dll
 0002:00000220       __imp_mexFunctionName      0000000180038220     libmex:libmex.dll
 0002:00000228       __imp_mexMakeMemoryPersistent 0000000180038228     libmex:libmex.dll
 0002:00000230       __imp_mexLock              0000000180038230     libmex:libmex.dll
 0002:00000238       __imp_mexIsLocked          0000000180038238     libmex:libmex.dll
 0002:00000240       __imp_mexWarnMsgTxt        0000000180038240     libmex:libmex.dll
 0002:00000248       __imp_mexCallMATLAB        0000000180038248     libmex:libmex.dll
 0002:00000250       __imp_mexErrMsgTxt         0000000180038250     libmex:libmex.dll
 0002:00000258       __imp_mexMakeArrayPersistent 0000000180038258     libmex:libmex.dll
 0002:00000260       __imp_mexGetVariable       0000000180038260     libmex:libmex.dll
 0002:00000268       __imp_mexPutVariable       0000000180038268     libmex:libmex.dll
 0002:00000270       __imp_mexSetTrapFlag       0000000180038270     libmex:libmex.dll
 0002:00000278       __imp_mexUnlock            0000000180038278     libmex:libmex.dll
 0002:00000280       \177libmex_NULL_THUNK_DATA 0000000180038280     libmex:libmex.dll
 0002:00000288       __imp_mxSetField_730       0000000180038288     libmx:libmx.dll
 0002:00000290       __imp_mxCreateDoubleMatrix_730 0000000180038290     libmx:libmx.dll
 0002:00000298       __imp_mxCreateDoubleScalar 0000000180038298     libmx:libmx.dll
 0002:000002a0       __imp_mxCreateString       00000001800382a0     libmx:libmx.dll
 0002:000002a8       __imp_mxCreateStructMatrix_730 00000001800382a8     libmx:libmx.dll
 0002:000002b0       __imp_mxCreateLogicalScalar 00000001800382b0     libmx:libmx.dll
 0002:000002b8       __imp_mxIsLogicalScalarTrue 00000001800382b8     libmx:libmx.dll
 0002:000002c0       __imp_mxGetString_700      00000001800382c0     libmx:libmx.dll
 0002:000002c8       __imp_mxCreateStringFromNChars_700 00000001800382c8     libmx:libmx.dll
 0002:000002d0       __imp_mxGetElementSize     00000001800382d0     libmx:libmx.dll
 0002:000002d8       __imp_mxCreateNumericArray_700 00000001800382d8     libmx:libmx.dll
 0002:000002e0       __imp_mxGetNumberOfDimensions_700 00000001800382e0     libmx:libmx.dll
 0002:000002e8       __imp_mxGetDimensions_700  00000001800382e8     libmx:libmx.dll
 0002:000002f0       __imp_mxCalcSingleSubscript_700 00000001800382f0     libmx:libmx.dll
 0002:000002f8       __imp_mxCreateStructArray_700 00000001800382f8     libmx:libmx.dll
 0002:00000300       __imp_mxCreateNumericMatrix_700 0000000180038300     libmx:libmx.dll
 0002:00000308       __imp_mxArrayClassIDName   0000000180038308     libmx:libmx.dll
 0002:00000310       __imp_mxGetImagData        0000000180038310     libmx:libmx.dll
 0002:00000318       __imp_mxGetData            0000000180038318     libmx:libmx.dll
 0002:00000320       __imp_mxIsEmpty            0000000180038320     libmx:libmx.dll
 0002:00000328       __imp_mxIsNaN              0000000180038328     libmx:libmx.dll
 0002:00000330       __imp_mxGetFieldNumber     0000000180038330     libmx:libmx.dll
 0002:00000338       __imp_mxCreateStructMatrix_700 0000000180038338     libmx:libmx.dll
 0002:00000340       __imp_mxGetNumberOfFields  0000000180038340     libmx:libmx.dll
 0002:00000348       __imp_mxGetFieldNameByNumber 0000000180038348     libmx:libmx.dll
 0002:00000350       __imp_mxGetFieldByNumber_700 0000000180038350     libmx:libmx.dll
 0002:00000358       __imp_mxSetFieldByNumber_700 0000000180038358     libmx:libmx.dll
 0002:00000360       __imp_mxIsSparse           0000000180038360     libmx:libmx.dll
 0002:00000368       __imp_mxGetLogicals        0000000180038368     libmx:libmx.dll
 0002:00000370       __imp_mxIsClass            0000000180038370     libmx:libmx.dll
 0002:00000378       __imp_mxIsA                0000000180038378     libmx:libmx.dll
 0002:00000380       __imp_mxIsStruct           0000000180038380     libmx:libmx.dll
 0002:00000388       __imp_mxGetNumberOfElements 0000000180038388     libmx:libmx.dll
 0002:00000390       __imp_mxGetField_700       0000000180038390     libmx:libmx.dll
 0002:00000398       __imp_mxAddField           0000000180038398     libmx:libmx.dll
 0002:000003a0       __imp_mxSetField_700       00000001800383a0     libmx:libmx.dll
 0002:000003a8       __imp_mxGetClassName       00000001800383a8     libmx:libmx.dll
 0002:000003b0       __imp_mxGetCell_700        00000001800383b0     libmx:libmx.dll
 0002:000003b8       __imp_mxSetCell_700        00000001800383b8     libmx:libmx.dll
 0002:000003c0       __imp_mxCreateCellMatrix_700 00000001800383c0     libmx:libmx.dll
 0002:000003c8       __imp_mxArrayToString      00000001800383c8     libmx:libmx.dll
 0002:000003d0       __imp_mxFree               00000001800383d0     libmx:libmx.dll
 0002:000003d8       __imp_mxCreateDoubleMatrix_700 00000001800383d8     libmx:libmx.dll
 0002:000003e0       __imp_mxIsLogical          00000001800383e0     libmx:libmx.dll
 0002:000003e8       __imp_mxGetScalar          00000001800383e8     libmx:libmx.dll
 0002:000003f0       __imp_mxCalloc             00000001800383f0     libmx:libmx.dll
 0002:000003f8       __imp_mxGetM               00000001800383f8     libmx:libmx.dll
 0002:00000400       __imp_mxGetN               0000000180038400     libmx:libmx.dll
 0002:00000408       __imp_mxIsComplex          0000000180038408     libmx:libmx.dll
 0002:00000410       __imp_mxIsNumeric          0000000180038410     libmx:libmx.dll
 0002:00000418       __imp_mxGetClassID         0000000180038418     libmx:libmx.dll
 0002:00000420       __imp_mxIsChar             0000000180038420     libmx:libmx.dll
 0002:00000428       __imp_mxGetString_730      0000000180038428     libmx:libmx.dll
 0002:00000430       __imp_mxDuplicateArray     0000000180038430     libmx:libmx.dll
 0002:00000438       __imp_mxDestroyArray       0000000180038438     libmx:libmx.dll
 0002:00000440       __imp_mxGetPr              0000000180038440     libmx:libmx.dll
 0002:00000448       \177libmx_NULL_THUNK_DATA  0000000180038448     libmx:libmx.dll
 0002:00000450       __imp_utFree               0000000180038450     libut:libut.dll
 0002:00000458       __imp_utCPUtime            0000000180038458     libut:libut.dll
 0002:00000460       __imp_utVSNprintf          0000000180038460     libut:libut.dll
 0002:00000468       __imp_utMalloc             0000000180038468     libut:libut.dll
 0002:00000470       \177libut_NULL_THUNK_DATA  0000000180038470     libut:libut.dll
 0002:00000478       __xc_a                     0000000180038478     MSVCRT:cinitexe.obj
 0002:00000480       __xc_z                     0000000180038480     MSVCRT:cinitexe.obj
 0002:00000488       __xi_a                     0000000180038488     MSVCRT:cinitexe.obj
 0002:00000498       __xi_z                     0000000180038498     MSVCRT:cinitexe.obj
 0002:000004a0       __real@41e8ede630e00000    00000001800384a0     c2_openloop_DE.obj
 0002:000004a8       __real@41e5aa1daa400000    00000001800384a8     c2_openloop_DE.obj
 0002:000004b0       __real@41e056cc42c00000    00000001800384b0     c2_openloop_DE.obj
 0002:000004b8       __real@41e76f8962400000    00000001800384b8     c2_openloop_DE.obj
 0002:000004c0       __real@4000000000000000    00000001800384c0     c2_openloop_DE.obj
 0002:000004c8       __real@4024000000000000    00000001800384c8     c2_openloop_DE.obj
 0002:000004d0       __real@3ff0000000000000    00000001800384d0     c2_openloop_DE.obj
 0002:000004d8       __real@bff0000000000000    00000001800384d8     c2_openloop_DE.obj
 0002:000004e0       __real@4014000000000000    00000001800384e0     c2_openloop_DE.obj
 0002:000004f0       DYNAMIC_DIMENSION_DEF      00000001800384f0     openloop_DE_sfun_registry.obj
 0002:00000510       _ssBadLevel2InputAccessMsg 0000000180038510     openloop_DE_sfun_registry.obj
 0002:000006a0       _ssBadLevel2DirectFeedMsg  00000001800386a0     openloop_DE_sfun_registry.obj
 0002:000007e0       _ssBadLevel2DirectFeedSolutionMsg 00000001800387e0     openloop_DE_sfun_registry.obj
 0002:00000850       _ssBadLevel2ZeroDirectFeedMsg 0000000180038850     openloop_DE_sfun_registry.obj
 0002:00000990       _ssBadLevel2ZeroDirectFeedMsg2 0000000180038990     openloop_DE_sfun_registry.obj
 0002:00000a78       __real@0000000000000000    0000000180038a78     openloop_DE_sfun_registry.obj
 0002:00000a80       __real@41602cbca0000000    0000000180038a80     openloop_DE_sfun_registry.obj
 0002:00000a88       __real@41e60de268200000    0000000180038a88     openloop_DE_sfun.obj
 0002:00000a90       __real@41a4abfc1a000000    0000000180038a90     openloop_DE_sfun.obj
 0002:00000a98       __real@41e7e1815f200000    0000000180038a98     openloop_DE_sfun.obj
 0002:00000aa0       __real@41d131cd66800000    0000000180038aa0     openloop_DE_sfun.obj
 0002:00000aa8       __real@41ed08af7be00000    0000000180038aa8     openloop_DE_sfun.obj
 0002:00000ab0       __real@41d03fc151000000    0000000180038ab0     openloop_DE_sfun.obj
 0002:00000ab8       __real@41c439d4aa000000    0000000180038ab8     openloop_DE_sfun.obj
 0002:00000ac0       __real@41ea8f1e72e00000    0000000180038ac0     openloop_DE_sfun.obj
 0002:00000ac8       __real@41e4b64c6dc00000    0000000180038ac8     openloop_DE_sfun.obj
 0002:00000ad0       __real@41e306d027a00000    0000000180038ad0     openloop_DE_sfun.obj
 0002:00000ad8       __real@41d677980a000000    0000000180038ad8     openloop_DE_sfun.obj
 0002:00000ae0       __real@41cf03578f000000    0000000180038ae0     openloop_DE_sfun.obj
 0002:00000ae8       __real@41e96d1d79200000    0000000180038ae8     openloop_DE_sfun.obj
 0002:00000af0       __real@41efc3bcdca00000    0000000180038af0     openloop_DE_sfun.obj
 0002:00000af8       __real@41e6c7a2a1200000    0000000180038af8     openloop_DE_sfun.obj
 0002:00000b00       __real@41de089c12800000    0000000180038b00     openloop_DE_sfun.obj
 0002:00000b08       ??_C@_00CNPNBAHC@?$AA@     0000000180038b08     sfc_mex:sfc_mex.obj
 0002:00000b0c       ??_C@_05DGLCPCBN@?$CFsx?$CFd?$AA@ 0000000180038b0c     sfc_mex:sfc_mex.obj
 0002:00000b14       ??_C@_02DPKJAMEF@?$CFd?$AA@ 0000000180038b14     sfc_mex:sfc_mex.obj
 0002:00000b18       ??_C@_0CC@DJOAOECF@Unknown?5MATLAB?5error?5encountered@ 0000000180038b18     sfc_mex:sfc_mex.obj
 0002:00000b40       ??_C@_0CJ@DAIIKGLI@?$CFs?5in?5?$CFs?5should?5never?5be?5called?5@ 0000000180038b40     sfc_mex:sfc_mex.obj
 0002:00000b70       ??_C@_0CE@ICKLNELB@Error?5calling?5MATLAB?5function?5?8?$CF@ 0000000180038b70     sfc_mex:sfc_mex.obj
 0002:00000b94       ??_C@_02DKCKIIND@?$CFs?$AA@ 0000000180038b94     sfc_mex:sfc_mex.obj
 0002:00000b98       ??_C@_07PHDIELCI@lasterr?$AA@ 0000000180038b98     sfc_mex:sfc_mex.obj
 0002:00000ba0       ??_C@_09HKCBALOK@embedded?4?$AA@ 0000000180038ba0     sfc_mex:sfc_mex.obj
 0002:00000bac       ??_C@_06BNJCAIGJ@double?$AA@ 0000000180038bac     sfc_mex:sfc_mex.obj
 0002:00000bb4       ??_C@_06EJFMBPJF@single?$AA@ 0000000180038bb4     sfc_mex:sfc_mex.obj
 0002:00000bbc       ??_C@_06KKKLBFKN@uint64?$AA@ 0000000180038bbc     sfc_mex:sfc_mex.obj
 0002:00000bc4       ??_C@_05DIFFJEPM@int64?$AA@ 0000000180038bc4     sfc_mex:sfc_mex.obj
 0002:00000bcc       ??_C@_06PKDKHAMA@uint32?$AA@ 0000000180038bcc     sfc_mex:sfc_mex.obj
 0002:00000bd4       ??_C@_05GIMEPBJB@int32?$AA@ 0000000180038bd4     sfc_mex:sfc_mex.obj
 0002:00000bdc       ??_C@_06JNNCGBKK@uint16?$AA@ 0000000180038bdc     sfc_mex:sfc_mex.obj
 0002:00000be4       ??_C@_05PCMOAPL@int16?$AA@ 0000000180038be4     sfc_mex:sfc_mex.obj
 0002:00000bec       ??_C@_05BOGOCLFF@uint8?$AA@ 0000000180038bec     sfc_mex:sfc_mex.obj
 0002:00000bf4       ??_C@_04DCGBOBJJ@int8?$AA@ 0000000180038bf4     sfc_mex:sfc_mex.obj
 0002:00000bfc       ??_C@_04KBDJOJNB@?$FL?$CFd?$FN?$AA@ 0000000180038bfc     sfc_mex:sfc_mex.obj
 0002:00000c08       ??_C@_0CD@NFPEPNBJ@Cannot?5add?5field?5?$CFs?5to?5struct?5?$CFs@ 0000000180038c08     sfc_mex:sfc_mex.obj
 0002:00000c30       ??_C@_0CF@PLDCCEBG@Cannot?5get?5field?5?$CFs?5from?5struct?5@ 0000000180038c30     sfc_mex:sfc_mex.obj
 0002:00000c58       ??_C@_0CO@MFJLJCHI@Struct?5array?5?8?$CFs?8?5does?5not?5have?5@ 0000000180038c58     sfc_mex:sfc_mex.obj
 0002:00000c88       ??_C@_0DF@IPGEGIDM@Object?5?8?$CFs?8?5is?5not?5a?5struct?3?5can@ 0000000180038c88     sfc_mex:sfc_mex.obj
 0002:00000cc0       ??_C@_0BL@KEKJNNL@MATLAB?5expression?5?8?$CFs?8?5?$CFs?4?$AA@ 0000000180038cc0     sfc_mex:sfc_mex.obj
 0002:00000ce0       ??_C@_0GH@JOEOEBFA@Size?5mismatch?5for?5?8?$CFs?8?5on?5dimens@ 0000000180038ce0     sfc_mex:sfc_mex.obj
 0002:00000d48       ??_C@_04IAGNFIBA@size?$AA@ 0000000180038d48     sfc_mex:sfc_mex.obj
 0002:00000d50       ??_C@_0DN@DNLDLJNN@is?5not?5of?5the?5correct?5class?3?5exp@ 0000000180038d50     sfc_mex:sfc_mex.obj
 0002:00000d90       ??_C@_06POLMGHPK@isreal?$AA@ 0000000180038d90     sfc_mex:sfc_mex.obj
 0002:00000d98       ??_C@_0CC@EDDDCJDC@is?5not?5of?5the?5correct?5complexnes@ 0000000180038d98     sfc_mex:sfc_mex.obj
 0002:00000dc0       ??_C@_0CB@POBCEEOP@is?5not?5of?5the?5correct?5sparseness@ 0000000180038dc0     sfc_mex:sfc_mex.obj
 0002:00000de8       ??_C@_0CC@JOFDGEBC@is?5not?5of?5the?5correct?5numerictyp@ 0000000180038de8     sfc_mex:sfc_mex.obj
 0002:00000e10       ??_C@_07MIMONDDE@isequal?$AA@ 0000000180038e10     sfc_mex:sfc_mex.obj
 0002:00000e18       ??_C@_0M@NAPEIPJI@numerictype?$AA@ 0000000180038e18     sfc_mex:sfc_mex.obj
 0002:00000e28       ??_C@_0BN@IMIABIKK@is?5not?5of?5the?5correct?5fimath?$AA@ 0000000180038e28     sfc_mex:sfc_mex.obj
 0002:00000e48       ??_C@_06LJOKAFHF@fimath?$AA@ 0000000180038e48     sfc_mex:sfc_mex.obj
 0002:00000e50       ??_C@_0EP@IAFBLFNF@Stateflow?5Internal?5Error?3?5?6Error@ 0000000180038e50     sfc_mex:sfc_mex.obj
 0002:00000ea0       ??_C@_02GFKODMMF@sf?$AA@   0000000180038ea0     sfc_mex:sfc_mex.obj
 0002:00000ea8       ??_C@_08MJJBNONC@mxDecode?$AA@ 0000000180038ea8     sfc_mex:sfc_mex.obj
 0002:00000ec0       ??_C@_0GH@OOBFJADG@Simulation?5stopped?5due?5to?5out?5of@ 0000000180038ec0     sfc_mex:sfc_mex.obj
 0002:00000f30       ??_C@_0HC@JODLBNFO@Simulation?5stopped?5due?5to?5size?5m@ 0000000180038f30     sfc_mex:sfc_mex.obj
 0002:00000fb0       ??_C@_0HC@PPOAOPGB@Simulation?5stopped?5due?5to?5size?5m@ 0000000180038fb0     sfc_mex:sfc_mex.obj
 0002:00001030       ??_C@_0JM@OFMOAAGL@Simulation?5stopped?5due?5to?5size?5m@ 0000000180039030     sfc_mex:sfc_mex.obj
 0002:000010d0       ??_C@_0KC@ODCGHMPH@Simulation?5stopped?5due?5to?5size?5o@ 00000001800390d0     sfc_mex:sfc_mex.obj
 0002:00001180       ??_C@_0GO@BKNPNGBP@Subscripted?5assignment?5dimension@ 0000000180039180     sfc_mex:sfc_mex.obj
 0002:000011f0       ??_C@_0DJ@MEDANBMA@Enable?5debugging?5to?5pinpoint?5the@ 00000001800391f0     sfc_mex:sfc_mex.obj
 0002:0000122c       ??_C@_01CLKCMJKC@?5?$AA@   000000018003922c     sfc_mex:sfc_mex.obj
 0002:00001230       ??_C@_0BAO@DDKKHLGF@Matrix?$CImatrix?$CJ?5subscript?5turned?5@ 0000000180039230     sfc_mex:sfc_mex.obj
 0002:00001340       ??_C@_0BAO@MGKOAKHL@Vector?$CIvector?$CJ?5subscript?5turned?5@ 0000000180039340     sfc_mex:sfc_mex.obj
 0002:00001450       ??_C@_0FA@KAHDAHHI@Cannot?5determine?5the?5exact?5numbe@ 0000000180039450     sfc_mex:sfc_mex.obj
 0002:000014a0       ??_C@_0FC@HJKNPCCF@Negative?5value?5detected?4?5Enable?5@ 00000001800394a0     sfc_mex:sfc_mex.obj
 0002:000014f8       ??_C@_0DK@JJKHINMK@Overflow?5detected?4?5Enable?5debugg@ 00000001800394f8     sfc_mex:sfc_mex.obj
 0002:00001540       ??_C@_0EA@POIJMBCP@Divide?5by?5zero?5detected?4?5Enable?5@ 0000000180039540     sfc_mex:sfc_mex.obj
 0002:00001580       ??_C@_0EK@CFEMECLL@Nonconforming?5enum?5value?5detecte@ 0000000180039580     sfc_mex:sfc_mex.obj
 0002:000015d0       ??_C@_0EE@BPGAOMO@Size?5mismatch?5for?5MATLAB?5express@ 00000001800395d0     sfc_mex:sfc_mex.obj
 0002:00001620       ??_C@_0EJ@KLNPHOFG@Dimension?5of?5fixed?5size?5one?5?$CI1?$CJ?5@ 0000000180039620     sfc_mex:sfc_mex.obj
 0002:00001670       ??_C@_07JFPGMOK@fprintf?$AA@ 0000000180039670     sfc_mex:sfc_mex.obj
 0002:00001680       ??_C@_0FE@EHCFPDEG@In?5MATLAB?5expression?5?8?$CFs?8?0?5field@ 0000000180039680     sfc_mex:sfc_mex.obj
 0002:000016d8       ??_C@_0DE@IJIFCHLH@In?5MATLAB?5expression?5?8?$CFs?8?0?5field@ 00000001800396d8     sfc_mex:sfc_mex.obj
 0002:00001710       ??_C@_0FK@JKPMKGDE@MATLAB?5expression?5?8?$CFs?8?5does?5not?5@ 0000000180039710     sfc_mex:sfc_mex.obj
 0002:0000176c       ??_C@_06PBJBIPGK@struct?$AA@ 000000018003976c     sfc_mex:sfc_mex.obj
 0002:00001778       ??_C@_0O@NFNPPCGN@isfimathlocal?$AA@ 0000000180039778     sfc_mex:sfc_mex.obj
 0002:00001788       ??_C@_0M@MLCGNPLD@embedded?4fi?$AA@ 0000000180039788     sfc_mex:sfc_mex.obj
 0002:00001798       ??_C@_0M@EGMNDJHO@?$CFs?5?$DN?5?$CF?415g?6?$AA@ 0000000180039798     sfc_mex:sfc_mex.obj
 0002:000017a4       ??_C@_03OFAPEBGM@?$CFs?6?$AA@ 00000001800397a4     sfc_mex:sfc_mex.obj
 0002:000017a8       ??_C@_0CL@LLBJDFID@failed?5sf_assertion?5in?5?$CFs?5at?5lin@ 00000001800397a8     sfc_mex:sfc_mex.obj
 0002:000017e0       ??_C@_0EJ@MIHEOKKA@?8?$CFs?8?3?5Array?5with?5number?5of?5dimen@ 00000001800397e0     sfc_mex:sfc_mex.obj
 0002:00001830       ??_C@_09JCLLFAHO@sfc_mex?4c?$AA@ 0000000180039830     sfc_mex:sfc_mex.obj
 0002:00001840       ??_C@_0O@FCFMOEOA@aNumDims?5?$DO?$DN?50?$AA@ 0000000180039840     sfc_mex:sfc_mex.obj
 0002:00001850       ??_C@_0CK@KDIMGCCA@?8?$CFs?8?3?5Sparse?5matrices?5are?5not?5su@ 0000000180039850     sfc_mex:sfc_mex.obj
 0002:00001880       ??_C@_0CI@KBLJAMNB@MATLAB?5expression?5?8?$CFs?8?5is?5not?5nu@ 0000000180039880     sfc_mex:sfc_mex.obj
 0002:000018a8       ??_C@_0P@LCMMCGDM@aSrcMx?5?$CB?$DN?5NULL?$AA@ 00000001800398a8     sfc_mex:sfc_mex.obj
 0002:000018c0       ??_C@_0EI@HJNNACGI@Eval?5of?5MATLAB?5expression?5?8?$CFs?8?5i@ 00000001800398c0     sfc_mex:sfc_mex.obj
 0002:00001908       ??_C@_0DM@BJICAGGK@Stateflow?5currently?5only?5support@ 0000000180039908     sfc_mex:sfc_mex.obj
 0002:00001944       ??_C@_05LAPONLG@false?$AA@ 0000000180039944     sfc_mex:sfc_mex.obj
 0002:0000194c       ??_C@_03LHCJEHON@nan?$AA@  000000018003994c     sfc_mex:sfc_mex.obj
 0002:00001950       ??_C@_04BHIIPFEC@base?$AA@ 0000000180039950     sfc_mex:sfc_mex.obj
 0002:00001958       ??_C@_06PLMANNP@evalin?$AA@ 0000000180039958     sfc_mex:sfc_mex.obj
 0002:00001960       ??_C@_06GFECGKEO@caller?$AA@ 0000000180039960     sfc_mex:sfc_mex.obj
 0002:00001968       ??_C@_0CM@LOMLNLMC@Invalid?5workspace?5type?5for?5sf_ma@ 0000000180039968     sfc_mex:sfc_mex.obj
 0002:00001994       ??_C@_01GBGANLPD@0?$AA@    0000000180039994     sfc_mex:sfc_mex.obj
 0002:00001998       ??_C@_06FJKEMHGD@global?$AA@ 0000000180039998     sfc_mex:sfc_mex.obj
 0002:000019a0       ??_C@_08KHPDDPHG@getfield?$AA@ 00000001800399a0     sfc_mex:sfc_mex.obj
 0002:000019ac       ??_C@_05LPIJGKJ@Value?$AA@ 00000001800399ac     sfc_mex:sfc_mex.obj
 0002:000019b8       ??_C@_0BH@HNIMIIFD@Unknown?5workspace?5type?$AA@ 00000001800399b8     sfc_mex:sfc_mex.obj
 0002:000019d0       ??_C@_0DA@IPMLFPJI@MATLAB?5expression?5?8?$CFs?8?5could?5not@ 00000001800399d0     sfc_mex:sfc_mex.obj
 0002:00001a00       ??_C@_0EB@HHPLBHBA@Parameter?5value?5out?5of?5bounds?4?5?$CF@ 0000000180039a00     sfc_mex:sfc_mex.obj
 0002:00001a50       __mask@@NegDouble@         0000000180039a50     sfc_mex:sfc_mex.obj
 0002:00001a60       ??_C@_0CB@DBMOOMDL@Unsupported?5class?5type?5?$CFs?5for?5?$CFs@ 0000000180039a60     sfc_mex:sfc_mex.obj
 0002:00001a88       ??_C@_0BI@OPNKAIOC@mxIsComplex?$CImxArrayPtr?$CJ?$AA@ 0000000180039a88     sfc_mex:sfc_mex.obj
 0002:00001aa0       ??_C@_0GA@OFLPCMBM@Stateflow?5Runtime?5Warning?3?5Loss?5@ 0000000180039aa0     sfc_mex:sfc_mex.obj
 0002:00001b00       __real@3810000000000000    0000000180039b00     sfc_mex:sfc_mex.obj
 0002:00001b08       __real@47efffffe0000000    0000000180039b08     sfc_mex:sfc_mex.obj
 0002:00001b10       __real@c060000000000000    0000000180039b10     sfc_mex:sfc_mex.obj
 0002:00001b18       __real@405fc00000000000    0000000180039b18     sfc_mex:sfc_mex.obj
 0002:00001b20       __real@406fe00000000000    0000000180039b20     sfc_mex:sfc_mex.obj
 0002:00001b28       __real@c0e0000000000000    0000000180039b28     sfc_mex:sfc_mex.obj
 0002:00001b30       __real@40dfffc000000000    0000000180039b30     sfc_mex:sfc_mex.obj
 0002:00001b38       __real@40efffe000000000    0000000180039b38     sfc_mex:sfc_mex.obj
 0002:00001b40       __real@c1e0000000000000    0000000180039b40     sfc_mex:sfc_mex.obj
 0002:00001b48       __real@41dfffffffc00000    0000000180039b48     sfc_mex:sfc_mex.obj
 0002:00001b50       __real@41efffffffe00000    0000000180039b50     sfc_mex:sfc_mex.obj
 0002:00001b58       ??_C@_0DO@JIJMNCAH@Class?5mismatch?5for?5variable?5?8?$CFs?8@ 0000000180039b58     sfc_mex:sfc_mex.obj
 0002:00001b98       ??_C@_03BBKEAIF@?$DP?$DP?$DP?$AA@ 0000000180039b98     sfc_mex:sfc_mex.obj
 0002:00001ba0       ??_C@_0DE@HICLJLJO@Assignment?5of?5complex?5data?5to?5no@ 0000000180039ba0     sfc_mex:sfc_mex.obj
 0002:00001bd8       ??_C@_0CF@NHFFCIEB@MATLAB?5function?5?8?$CFs?8?5returned?5NU@ 0000000180039bd8     sfc_mex:sfc_mex.obj
 0002:00001c00       ??_C@_0GP@JPKMBIEI@Array?5bounds?5error?5in?5MATLAB?5exp@ 0000000180039c00     sfc_mex:sfc_mex.obj
 0002:00001c70       ??_C@_0P@FLJFOPHI@pIndex?$FLi?$FN?5?$DO?$DN?50?$AA@ 0000000180039c70     sfc_mex:sfc_mex.obj
 0002:00001c80       ??_C@_0DI@IGEABFHB@MATLAB?5expression?5?8?$CFs?8?5has?5?$CFd?5di@ 0000000180039c80     sfc_mex:sfc_mex.obj
 0002:00001cb8       ??_C@_0L@EFLJKPA@mxArrayPtr?$AA@ 0000000180039cb8     sfc_mex:sfc_mex.obj
 0002:00001cc8       ??_C@_0CK@FHKKOEPH@numDims?5?$DO?$DN?50?5?$CG?$CG?5numDims?5?$DM?$DN?5MAX_D@ 0000000180039cc8     sfc_mex:sfc_mex.obj
 0002:00001d00       ??_C@_0EM@MPIDLJBF@MATLAB?5expression?5?8?$CFs?8?5subscript@ 0000000180039d00     sfc_mex:sfc_mex.obj
 0002:00001d4c       ??_C@_04IGKKBJEE@?$DN?$CFg?$DL?$AA@ 0000000180039d4c     sfc_mex:sfc_mex.obj
 0002:00001d54       ??_C@_01PKGAHCOL@?$CJ?$AA@ 0000000180039d54     sfc_mex:sfc_mex.obj
 0002:00001d58       ??_C@_03LEIBKMN@?0?$CFd?$AA@ 0000000180039d58     sfc_mex:sfc_mex.obj
 0002:00001d5c       ??_C@_03IECKINJK@?$CI?$CFd?$AA@ 0000000180039d5c     sfc_mex:sfc_mex.obj
 0002:00001d60       ??_C@_0FB@HKJNNBFK@Stateflow?5ml?5type?5data?5?8?$CFs?8?5subs@ 0000000180039d60     sfc_mex:sfc_mex.obj
 0002:00001db8       ??_C@_0CN@HPHHCDPK@Stateflow?5ml?5type?5data?5?8?$CFs?8?5is?5n@ 0000000180039db8     sfc_mex:sfc_mex.obj
 0002:00001de8       ??_C@_0CG@JIOBALFE@Stateflow?5ml?5type?5data?5?8?$CFs?8?5is?5e@ 0000000180039de8     sfc_mex:sfc_mex.obj
 0002:00001e10       ??_C@_0BD@GAHDCPBG@mxArrayPtr?5?$CB?$DN?5NULL?$AA@ 0000000180039e10     sfc_mex:sfc_mex.obj
 0002:00001e28       ??_C@_0CF@HCINMAFF@result?5?$DN?5mxCreateDoubleScalar?$CIva@ 0000000180039e28     sfc_mex:sfc_mex.obj
 0002:00001e50       ??_C@_0BF@GAJKLFOH@fixpt_lower_mx_array?$AA@ 0000000180039e50     sfc_mex:sfc_mex.obj
 0002:00001e68       ??_C@_02FINOOIBE@Cg?$AA@   0000000180039e68     sfc_mex:sfc_mex.obj
 0002:00001e70       ??_C@_09GIFEIFFL@sfprivate?$AA@ 0000000180039e70     sfc_mex:sfc_sf.obj
 0002:00001e80       ??_C@_0CC@JDELABLI@get_machine_and_chart_file_numbe@ 0000000180039e80     sfc_mex:sfc_sf.obj
 0002:00001ea8       ??_C@_0BO@JCKKMPIB@get_sfun_block_specialization?$AA@ 0000000180039ea8     sfc_mex:sfc_sf.obj
 0002:00001ed0       ??_C@_0FP@OGBKADON@The?5chart?5name?5?4?4?4?$CFs?5is?5not?5pres@ 0000000180039ed0     sfc_mex:sfc_sf.obj
 0002:00001f30       ??_C@_0FM@KEMGDKHM@The?5chart?5name?5?$CFs?5is?5not?5present@ 0000000180039f30     sfc_mex:sfc_sf.obj
 0002:00001f90       ??_C@_0BD@NMFAPBEK@mdlInitializeSizes?$AA@ 0000000180039f90     sfc_mex:sfc_sf.obj
 0002:00001fa4       ??_C@_06EJFCAODB@sfc_sf?$AA@ 0000000180039fa4     sfc_mex:sfc_sf.obj
 0002:00001fb0       ??_C@_0BJ@PBIFPMMD@mdlInitializeSampleTimes?$AA@ 0000000180039fb0     sfc_mex:sfc_sf.obj
 0002:00001fd0       ??_C@_0FI@CPPGBPPK@Stateflow?5Internal?5Error?3?5?6Error@ 0000000180039fd0     sfc_mex:sfc_sf.obj
 0002:00002028       ??_C@_0CN@GACCLMJH@preload_infomatman_for_rtw_optim@ 000000018003a028     sfc_mex:sfc_sf.obj
 0002:00002058       ??_C@_07CFINJGKH@Private?$AA@ 000000018003a058     sfc_mex:sfc_sf.obj
 0002:00002060       ??_C@_0GC@KEKNFKIJ@Stateflow?5Internal?5Error?3?5?6rtw_o@ 000000018003a060     sfc_mex:sfc_sf.obj
 0002:000020d0       ??_C@_0EK@MLFDFPLJ@Stateflow?5Internal?5Error?3?5?6Inter@ 000000018003a0d0     sfc_mex:sfc_sf.obj
 0002:00002120       ??_C@_0BG@PNKGMGHF@rtw_optimization_info?$AA@ 000000018003a120     sfc_mex:sfc_sf.obj
 0002:00002138       ??_C@_0BA@PHPHFLPF@chart_inlinable?$AA@ 000000018003a138     sfc_mex:sfc_sf.obj
 0002:00002150       ??_C@_0MB@KGDKCEKF@Stateflow?5Internal?5Error?3?5?6Numbe@ 000000018003a150     sfc_mex:sfc_sf.obj
 0002:00002220       ??_C@_0GN@DNCJEGHD@Stateflow?5Internal?5Error?3?5?6Error@ 000000018003a220     sfc_mex:sfc_sf.obj
 0002:00002290       ??_C@_0CA@GOKFFBBO@outputEventsWithMultipleCallers?$AA@ 000000018003a290     sfc_mex:sfc_sf.obj
 0002:000022b0       ??_C@_0LH@NDHODBLK@Stateflow?5Internal?5Error?3?5?6Numbe@ 000000018003a2b0     sfc_mex:sfc_sf.obj
 0002:00002368       ??_C@_0BB@GEEDBOGK@reusable_outputs?$AA@ 000000018003a368     sfc_mex:sfc_sf.obj
 0002:00002380       ??_C@_0II@FEBCOBGA@Stateflow?5Internal?5Error?3?5?6Numbe@ 000000018003a380     sfc_mex:sfc_sf.obj
 0002:00002408       ??_C@_0BG@HMMHPAKE@expressionable_inputs?$AA@ 000000018003a408     sfc_mex:sfc_sf.obj
 0002:00002420       ??_C@_0BB@MBBOKNEL@listen_for_ctrlc?$AA@ 000000018003a420     sfc_mex:sfc_sf.obj
 0002:00002434       ??_C@_03LOANPFAI@mex?$AA@  000000018003a434     sfc_mex:sfc_sf.obj
 0002:00002438       ??_C@_07HLHKBCBI@sfdebug?$AA@ 000000018003a438     sfc_mex:sfc_sf.obj
 0002:00002440       ??_C@_07MFNNEMOJ@drawnow?$AA@ 000000018003a440     sfc_mex:sfc_sf.obj
 0002:00002448       __real@3fd3333333333333    000000018003a448     sfc_mex:sfc_sf.obj
 0002:00002450       ??_C@_0DG@OJBAPEMA@Internal?5Error?3?5paramsIndex?5?$DN?5?$CFd@ 000000018003a450     sfc_mex:sfc_sf.obj
 0002:00002490       ??_C@_0BAI@GPDPHGCD@Cannot?5broadcast?5function?5call?5o@ 000000018003a490     sfc_mex:sfc_sf.obj
 0002:000025a0       ??_C@_0BBC@NGKHEJAF@Cannot?5enable?1disable?5function?5c@ 000000018003a5a0     sfc_mex:sfc_sf.obj
 0002:000026b8       ??_C@_08HDNBGBNP@bitWidth?$AA@ 000000018003a6b8     sfc_mex:sfc_sf.obj
 0002:000026c8       ??_C@_0BG@MDDFDLDC@resolveToSignalObject?$AA@ 000000018003a6c8     sfc_mex:sfc_sf.obj
 0002:000026e0       ??_C@_07KHBFOCMF@varName?$AA@ 000000018003a6e0     sfc_mex:sfc_sf.obj
 0002:000026e8       ??_C@_09LHPHPAOE@isComplex?$AA@ 000000018003a6e8     sfc_mex:sfc_sf.obj
 0002:000026f8       ??_C@_0CM@OAMAJMIG@Failed?5to?5register?5type?5?8?$CFs?8?5wit@ 000000018003a6f8     sfc_mex:sfc_sf.obj
 0002:00002728       ??_C@_08MLIGMCAH@typeSize?$AA@ 000000018003a728     sfc_mex:sfc_sf.obj
 0002:00002738       ??_C@_0BI@OFLHAMB@vector_of_void_pointers?$AA@ 000000018003a738     sfc_mex:sfc_sf.obj
 0002:00002750       ??_C@_04NBAGBPGE@bias?$AA@ 000000018003a750     sfc_mex:sfc_sf.obj
 0002:00002758       ??_C@_08EGJNFMPO@exponent?$AA@ 000000018003a758     sfc_mex:sfc_sf.obj
 0002:00002764       ??_C@_05LAHHKLJI@slope?$AA@ 000000018003a764     sfc_mex:sfc_sf.obj
 0002:00002770       ??_C@_0L@EMMELFNN@wordLength?$AA@ 000000018003a770     sfc_mex:sfc_sf.obj
 0002:00002780       ??_C@_08EJEJGLGA@isSigned?$AA@ 000000018003a780     sfc_mex:sfc_sf.obj
 0002:0000278c       ??_C@_05LFJLPLPG@fixpt?$AA@ 000000018003a78c     sfc_mex:sfc_sf.obj
 0002:00002798       ??_C@_07GOBOHMJA@boolean?$AA@ 000000018003a798     sfc_mex:sfc_sf.obj
 0002:000027a0       ??_C@_04GPMDFGEJ@type?$AA@ 000000018003a7a0     sfc_mex:sfc_sf.obj
 0002:000027a8       ??_C@_0O@EIPJLOAA@extModeUpload?$AA@ 000000018003a7a8     sfc_mex:sfc_sf.obj
 0002:000027b8       __real@43e0000000000000    000000018003a7b8     sfc_mex:sfc_sf.obj
 0002:000027c0       ??_C@_03PLHFFLIH@ptr?$AA@  000000018003a7c0     sfc_mex:sfc_sf.obj
 0002:000027c8       ??_C@_0BC@HMCIKMPA@requiredStackSize?$AA@ 000000018003a7c8     sfc_mex:sfc_sf.obj
 0002:000027e0       ??_C@_0CB@OCGIMAKA@RegisterMachineParentedDataDwork@ 000000018003a7e0     sfc_mex:sfc_sf.obj
 0002:00002808       ??_C@_0BD@LFPAKDFC@machineDataVarInfo?$AA@ 000000018003a808     sfc_mex:sfc_sf.obj
 0002:00002820       ??_C@_09GAJBGLOB@dworkInfo?$AA@ 000000018003a820     sfc_mex:sfc_sf.obj
 0002:00002830       sf_uint_bits_log2          000000018003a830     sfc_debug:sfcdebug.obj
 0002:00002850       ??_C@_04GKMJMOBJ@disp?$AA@ 000000018003a850     sfc_debug:sfcdebug.obj
 0002:00002858       ??_C@_0DJ@GEKCDEED@Runtime?5size?5mismatch?5for?5dimens@ 000000018003a858     sfc_debug:sfcdebug.obj
 0002:00002898       ??_C@_0N@IHFJDIPG@load_machine?$AA@ 000000018003a898     sfc_debug:sfcdebug.obj
 0002:000028a8       ??_C@_0P@NOFOFJMO@ScriptCacheGet?$AA@ 000000018003a8a8     sfc_debug:sfcdebug.obj
 0002:000028b8       ??_C@_0P@HCIIHGKN@simulationTime?$AA@ 000000018003a8b8     sfc_debug:sfcdebug.obj
 0002:000028c8       ??_C@_06MBJIKMHL@isSend?$AA@ 000000018003a8c8     sfc_debug:sfcdebug.obj
 0002:000028d0       ??_C@_0BC@HKLNGIIJ@messagePortNumber?$AA@ 000000018003a8d0     sfc_debug:sfcdebug.obj
 0002:000028e8       ??_C@_07KGNNMFDL@chartId?$AA@ 000000018003a8e8     sfc_debug:sfcdebug.obj
 0002:000028f0       ??_C@_0BD@LPIHANBP@State?5Entry?5Action?$AA@ 000000018003a8f0     sfc_debug:sfcdebug.obj
 0002:00002908       ??_C@_0BE@EDAKPKIF@State?5During?5Action?$AA@ 000000018003a908     sfc_debug:sfcdebug.obj
 0002:00002920       ??_C@_0BC@FKIGLKJE@State?5Exit?5Action?$AA@ 000000018003a920     sfc_debug:sfcdebug.obj
 0002:00002934       ??_C@_04CGFJFPFD@none?$AA@ 000000018003a934     sfc_debug:sfcdebug.obj
 0002:00002940       ??_C@_0BD@JMJALEKH@Transition?5Trigger?$AA@ 000000018003a940     sfc_debug:sfcdebug.obj
 0002:00002958       ??_C@_0BO@JIGLNAHF@Transition?5Guarding?5Condition?$AA@ 000000018003a958     sfc_debug:sfcdebug.obj
 0002:00002978       ??_C@_0BB@ODEGBFLN@Condition?5Action?$AA@ 000000018003a978     sfc_debug:sfcdebug.obj
 0002:00002990       ??_C@_0BC@EPJNNAPA@Transition?5Action?$AA@ 000000018003a990     sfc_debug:sfcdebug.obj
 0002:000029a8       ??_C@_0DI@JGHJOLLJ@INTERNAL?5ERROR?4?5Failed?5assertion@ 000000018003a9a8     sfc_debug:sfcdebug.obj
 0002:000029e0       ??_C@_01EEMJAFIK@?6?$AA@   000000018003a9e0     sfc_debug:sfcdebug.obj
 0002:000029e8       ??_C@_0P@HHNBJNJA@context_string?$AA@ 000000018003a9e8     sfc_debug:sfcdebug.obj
 0002:000029f8       ??_C@_0BN@PMGOFJAJ@shouldAlwaysHonorBreakpoints?$AA@ 000000018003a9f8     sfc_debug:sfcdebug.obj
 0002:00002a18       ??_C@_0DL@EPKGPGLC@?$CImachine?9?$DOdataCompInfo?4fixedPoin@ 000000018003aa18     sfc_debug:sfcdebug.obj
 0002:00002a58       ??_C@_0L@GJHMCDGO@sfcdebug?4c?$AA@ 000000018003aa58     sfc_debug:sfcdebug.obj
 0002:00002a68       ??_C@_0DE@CBCLKIAM@?$CImachine?9?$DOdataCompInfo?4isComplex@ 000000018003aa68     sfc_debug:sfcdebug.obj
 0002:00002aa0       ??_C@_0DP@MDOJBFKE@?$CIinstance?9?$DOdataCompInfo?4fixedPoi@ 000000018003aaa0     sfc_debug:sfcdebug.obj
 0002:00002ae0       ??_C@_0DM@KFHGIBMB@?$CIinstance?9?$DOdataCompInfo?4fixedPoi@ 000000018003aae0     sfc_debug:sfcdebug.obj
 0002:00002b20       ??_C@_0DF@IIPJPBAH@?$CIinstance?9?$DOdataCompInfo?4isComple@ 000000018003ab20     sfc_debug:sfcdebug.obj
 0002:00002b58       ??_C@_0DA@OMEPAHNH@?$CIchart?9?$DOdata?4outputDataFlags?$CJ?4le@ 000000018003ab58     sfc_debug:sfcdebug.obj
 0002:00002b88       ??_C@_0CP@JPBDBJBK@?$CIchart?9?$DOdata?4inputDataFlags?$CJ?4len@ 000000018003ab88     sfc_debug:sfcdebug.obj
 0002:00002bb8       ??_C@_03KGJNKAJD@lic?$AA@  000000018003abb8     sfc_debug:sfcdebug.obj
 0002:00002bbc       ??_C@_04PNMLDJAE@ense?$AA@ 000000018003abbc     sfc_debug:sfcdebug.obj
 0002:00002bc8       ??_C@_0L@ONMHLBPB@?$CFs?$CFs?$CFslbox?$AA@ 000000018003abc8     sfc_debug:sfcdebug.obj
 0002:00002bd4       ??_C@_04CLOJJEIM@fixe?$AA@ 000000018003abd4     sfc_debug:sfcdebug.obj
 0002:00002bdc       ??_C@_05CBHOIFCP@t_too?$AA@ 000000018003abdc     sfc_debug:sfcdebug.obj
 0002:00002be4       ??_C@_06MGFNEDEJ@d_poin?$AA@ 000000018003abe4     sfc_debug:sfcdebug.obj
 0002:00002bec       ??_C@_04HDOCAJNK@?$CFs?$CFs?$AA@ 000000018003abec     sfc_debug:sfcdebug.obj
 0002:00002bf4       ??_C@_04BJBBOLDM@chec?$AA@ 000000018003abf4     sfc_debug:sfcdebug.obj
 0002:00002bfc       ??_C@_04KNBDLPKC@kout?$AA@ 000000018003abfc     sfc_debug:sfcdebug.obj
 0002:00002c08       ??_C@_0BA@FKECJMCE@active_instance?$AA@ 000000018003ac08     sfc_debug:sfcdebug.obj
 0002:00002c18       ??_C@_0DD@MJFCMKPO@transCnt?5?$DN?$DN?5instance?9?$DOcvToolIds?4@ 000000018003ac18     sfc_debug:sfcdebug.obj
 0002:00002c50       ??_C@_0CO@MONEMJEL@stateCnt?5?$DN?$DN?5instance?9?$DOcvToolIds?4@ 000000018003ac50     sfc_debug:sfcdebug.obj
 0002:00002c80       ??_C@_0O@ELHBEDAD@init_debugger?$AA@ 000000018003ac80     sfc_debug:sfcdebug.obj
 0002:00002c90       ??_C@_0L@PKOFOKNN@break_here?$AA@ 000000018003ac90     sfc_debug:sfcdebug.obj
 0002:00002ca0       ??_C@_0BH@KBPHNGCH@script?4activeMachineId?$AA@ 000000018003aca0     sfc_debug:sfcdebug.obj
 0002:00002cb8       ??_C@_03KCHOJKKI@set?$AA@  000000018003acb8     sfc_debug:sfcdebug.obj
 0002:00002cc0       ??_C@_0DD@PKMAPHBF@?$CImachine?9?$DOdata?4watchFlags?$CJ?4lengt@ 000000018003acc0     sfc_debug:sfcdebug.obj
 0002:00002d00       ??_C@_0FE@KLPHIMDI@?$CIchart?9?$DOdata?4watchFlags?$CJ?4length?$DO@ 000000018003ad00     sfc_debug:sfcdebug.obj
 0002:00002d58       ??_C@_0BO@GFBPGEIL@bufferSizeGet?5?$DN?$DN?5totalSizeGet?$AA@ 000000018003ad58     sfc_debug:sfcdebug.obj
 0002:00002d78       ??_C@_0BO@BEEPOEDP@bufferSizeSet?5?$DN?$DN?5totalSizeSet?$AA@ 000000018003ad78     sfc_debug:sfcdebug.obj
 0002:00002d98       ??_C@_0BG@NNAKOPEK@get_script_line_count?$AA@ 000000018003ad98     sfc_debug:sfcdebug.obj
 0002:00002db0       ??_C@_0BJ@GADAHKGG@temporal_threshold_error?$AA@ 000000018003adb0     sfc_debug:sfcdebug.obj
 0002:00002dd0       ??_C@_0BK@KABIOMCC@transition_conflict_error?$AA@ 000000018003add0     sfc_debug:sfcdebug.obj
 0002:00002df0       ??_C@_0BK@HLPANOPJ@state_inconsistency_error?$AA@ 000000018003adf0     sfc_debug:sfcdebug.obj
 0002:00002e10       ??_C@_0BA@PCEGODO@cycle_detection?$AA@ 000000018003ae10     sfc_debug:sfcdebug.obj
 0002:00002e20       ??_C@_0CP@HMOGACCG@Simulation?5stopped?5due?5to?5out?5of@ 000000018003ae20     sfc_debug:sfcdebug.obj
 0002:00002e50       ??_C@_0BD@LFFFHIJG@array_bounds_error?$AA@ 000000018003ae50     sfc_debug:sfcdebug.obj
 0002:00002e68       ??_C@_0O@IENBAMNA@runtime_error?$AA@ 000000018003ae68     sfc_debug:sfcdebug.obj
 0002:00002e78       ??_C@_0CC@EDKHOOPE@Call?5to?5MATLAB?5function?5aborted?3@ 000000018003ae78     sfc_debug:sfcdebug.obj
 0002:00002ea0       ??_C@_0DJ@JBGHLJFL@Simulation?5stopped?5due?5to?5size?5m@ 000000018003aea0     sfc_debug:sfcdebug.obj
 0002:00002ee0       ??_C@_0DJ@EAKPCDBG@Simulation?5stopped?5due?5to?5size?5m@ 000000018003aee0     sfc_debug:sfcdebug.obj
 0002:00002f20       ??_C@_0GD@BJCLDBKO@Simulation?5stopped?5due?5to?5size?5m@ 000000018003af20     sfc_debug:sfcdebug.obj
 0002:00002f90       ??_C@_0GJ@OHCOIONE@Simulation?5stopped?5due?5to?5size?5o@ 000000018003af90     sfc_debug:sfcdebug.obj
 0002:00003000       ??_C@_0DF@BOMHHCNB@Subscripted?5assignment?5dimension@ 000000018003b000     sfc_debug:sfcdebug.obj
 0002:00003040       ??_C@_0NG@BOPFGKBO@Matrix?$CImatrix?$CJ?5subscript?5turned?5@ 000000018003b040     sfc_debug:sfcdebug.obj
 0002:00003120       ??_C@_0HE@FPEPCMDA@Matrix?$CImatrix?$CJ?5subscript?5turned?5@ 000000018003b120     sfc_debug:sfcdebug.obj
 0002:000031a0       ??_C@_0NG@MLJIHJIH@Vector?$CIvector?$CJ?5subscript?5turned?5@ 000000018003b1a0     sfc_debug:sfcdebug.obj
 0002:00003280       ??_C@_0HE@BHPDCNDF@Vector?$CIvector?$CJ?5subscript?5turned?5@ 000000018003b280     sfc_debug:sfcdebug.obj
 0002:000032f8       ??_C@_0BL@HKADOJK@Unknown?5runtime?5error?3?5?$CFs?4?$AA@ 000000018003b2f8     sfc_debug:sfcdebug.obj
 0002:00003318       ??_C@_0P@FIEIFKHH@dataName?$CB?$DNNULL?$AA@ 000000018003b318     sfc_debug:sfcdebug.obj
 0002:00003328       ??_C@_0BC@JKFOPCCM@non_integer_error?$AA@ 000000018003b328     sfc_debug:sfcdebug.obj
 0002:00003340       ??_C@_09MMCAMPEC@nan_error?$AA@ 000000018003b340     sfc_debug:sfcdebug.obj
 0002:00003350       ??_C@_0P@KGNBONIG@negative_error?$AA@ 000000018003b350     sfc_debug:sfcdebug.obj
 0002:00003360       ??_C@_0DA@OEGHOJFO@Simulation?5stopped?5due?5to?5divide@ 000000018003b360     sfc_debug:sfcdebug.obj
 0002:00003390       ??_C@_0P@DAGNNBKM@overflow_error?$AA@ 000000018003b390     sfc_debug:sfcdebug.obj
 0002:000033a0       ??_C@_0BF@IEPBJJM@divide_by_zero_error?$AA@ 000000018003b3a0     sfc_debug:sfcdebug.obj
 0002:000033b8       ??_C@_0BC@CNIFONOF@unsafe_enum_error?$AA@ 000000018003b3b8     sfc_debug:sfcdebug.obj
 0002:000033d0       ??_C@_0BA@GLGJGIFO@data_loss_error?$AA@ 000000018003b3d0     sfc_debug:sfcdebug.obj
 0002:000033e0       ??_C@_0BB@LFNCDKMF@data_range_error?$AA@ 000000018003b3e0     sfc_debug:sfcdebug.obj
 0002:00003400       ??_C@_0FA@OJFHKNAF@Simulation?5stopped?5because?5a?5dat@ 000000018003b400     sfc_debug:sfcdebug.obj
 0002:00003450       ??_C@_0BI@LLOJJCOG@read_before_write_error?$AA@ 000000018003b450     sfc_debug:sfcdebug.obj
 0002:00003468       __real@4059000000000000    000000018003b468     sfc_debug:sfcdebug.obj
 0002:00003470       ??_C@_0EL@LHLCBPON@objectType?$DN?$DNEVENT_OBJECT?5?$CG?$CG?5obje@ 000000018003b470     sfc_debug:sfcdebug.obj
 0002:000034c0       ??_C@_0CK@BGKNIJPH@Simulation?5stopped?5due?5to?5infini@ 000000018003b4c0     sfc_debug:sfcdebug.obj
 0002:000034f0       ??_C@_0BC@OGHOEIO@draw_message_post?$AA@ 000000018003b4f0     sfc_debug:sfcdebug.obj
 0002:00003510       ??_C@_0EC@EKMLJIIP@strlen?$CItargetName?$CJ?$DMsizeof?$CIdebugI@ 000000018003b510     sfc_debug:sfcdebug.obj
 0002:00003560       ??_C@_0EE@LPPEFNLK@strlen?$CImachineName?$CJ?$DMsizeof?$CIdebug@ 000000018003b560     sfc_debug:sfcdebug.obj
 0002:000035a8       ??_C@_0BO@OEBODAF@charts?9?$DOlength?5?$DM?5charts?9?$DOsize?$AA@ 000000018003b5a8     sfc_debug:sfcdebug.obj
 0002:000035c8       ??_C@_0P@NDNBPAGO@charts?9?$DOsize?$DO0?$AA@ 000000018003b5c8     sfc_debug:sfcdebug.obj
 0002:000035d8       ??_C@_09DACGJFPO@terminate?$AA@ 000000018003b5d8     sfc_debug:sfcdebug.obj
 0002:000035e8       ??_C@_0BH@BOIPOAMD@currentoptionalinteger?$AA@ 000000018003b5e8     sfc_debug:sfc_api.obj
 0002:00003600       ??_C@_0BI@KDFLIHKN@currentstatementcontext?$AA@ 000000018003b600     sfc_debug:sfc_api.obj
 0002:00003618       ??_C@_0BF@CJJCNHOP@currentstatementinfo?$AA@ 000000018003b618     sfc_debug:sfc_api.obj
 0002:00003630       ??_C@_0BA@EEHAMBBL@currentcoverage?$AA@ 000000018003b630     sfc_debug:sfc_api.obj
 0002:00003640       ??_C@_0BD@CPIGBEHM@currentmachinename?$AA@ 000000018003b640     sfc_debug:sfc_api.obj
 0002:00003658       ??_C@_0BF@MPNFKHIK@currentmachinenumber?$AA@ 000000018003b658     sfc_debug:sfc_api.obj
 0002:00003670       ??_C@_0BB@EAGFPGEG@currentmachineid?$AA@ 000000018003b670     sfc_debug:sfc_api.obj
 0002:00003688       ??_C@_0P@LDEJFJKJ@simulationtime?$AA@ 000000018003b688     sfc_debug:sfc_api.obj
 0002:00003698       ??_C@_0P@CKMPNBM@currenttagtype?$AA@ 000000018003b698     sfc_debug:sfc_api.obj
 0002:000036a8       ??_C@_0BH@EMAALFDO@currentactiveeventtype?$AA@ 000000018003b6a8     sfc_debug:sfc_api.obj
 0002:000036c0       ??_C@_0BF@BIDFPCPF@currentactiveeventid?$AA@ 000000018003b6c0     sfc_debug:sfc_api.obj
 0002:000036d8       ??_C@_0BA@LAPNNELA@currentobjectid?$AA@ 000000018003b6d8     sfc_debug:sfc_api.obj
 0002:000036e8       ??_C@_0BB@LLJHHKEI@currenteventtype?$AA@ 000000018003b6e8     sfc_debug:sfc_api.obj
 0002:00003700       ??_C@_0BC@BDADCDEL@currentobjecttype?$AA@ 000000018003b700     sfc_debug:sfc_api.obj
 0002:00003718       ??_C@_0BH@HDHFFKCN@currentisminortimestep?$AA@ 000000018003b718     sfc_debug:sfc_api.obj
 0002:00003730       ??_C@_0BG@PKFJEKLL@currentinstancehandle?$AA@ 000000018003b730     sfc_debug:sfc_api.obj
 0002:00003748       ??_C@_0BG@GJFHKFBJ@currentinstancenumber?$AA@ 000000018003b748     sfc_debug:sfc_api.obj
 0002:00003760       ??_C@_0BD@DKAMMHEE@currentchartnumber?$AA@ 000000018003b760     sfc_debug:sfc_api.obj
 0002:00003778       ??_C@_0P@EANFOHCD@currentchartid?$AA@ 000000018003b778     sfc_debug:sfc_api.obj
 0002:00003788       ??_C@_0CC@JILMFDHL@extract_message_post_receive_inf@ 000000018003b788     sfc_debug:sfc_api.obj
 0002:000037ac       ??_C@_06IMFOKBKF@assign?$AA@ 000000018003b7ac     sfc_debug:sfc_api.obj
 0002:000037b8       ??_C@_0BC@CMFMGKCG@set_script_cv_ids?$AA@ 000000018003b7b8     sfc_debug:sfc_api.obj
 0002:000037d0       ??_C@_0BE@ONNFKBAC@set_instance_cv_ids?$AA@ 000000018003b7d0     sfc_debug:sfc_api.obj
 0002:000037e8       ??_C@_0BE@CDIKCKCD@get_instance_handle?$AA@ 000000018003b7e8     sfc_debug:sfc_api.obj
 0002:00003800       ??_C@_0BE@GPEMFILK@break_between_times?$AA@ 000000018003b800     sfc_debug:sfc_api.obj
 0002:00003818       ??_C@_0O@KGONFDDG@active_states?$AA@ 000000018003b818     sfc_debug:sfc_api.obj
 0002:00003828       ??_C@_0BC@LHALNGBC@state_consistency?$AA@ 000000018003b828     sfc_debug:sfc_api.obj
 0002:00003840       ??_C@_0BE@JNDELHDH@transition_conflict?$AA@ 000000018003b840     sfc_debug:sfc_api.obj
 0002:00003858       ??_C@_0L@ECJAFPAF@data_range?$AA@ 000000018003b858     sfc_debug:sfc_api.obj
 0002:00003868       ??_C@_0O@NAKDKJME@select_charts?$AA@ 000000018003b868     sfc_debug:sfc_api.obj
 0002:00003878       ??_C@_0N@KLDBDGD@select_chart?$AA@ 000000018003b878     sfc_debug:sfc_api.obj
 0002:00003888       ??_C@_0O@NJPMKBAC@set_animation?$AA@ 000000018003b888     sfc_debug:sfc_api.obj
 0002:00003898       ??_C@_09FLOFKLFE@set_watch?$AA@ 000000018003b898     sfc_debug:sfc_api.obj
 0002:000038a8       ??_C@_0O@ECMAEPOC@get_script_id?$AA@ 000000018003b8a8     sfc_debug:sfc_api.obj
 0002:000038b8       ??_C@_0BJ@KFGPCNG@query_script_breakpoints?$AA@ 000000018003b8b8     sfc_debug:sfc_api.obj
 0002:000038d8       ??_C@_0BJ@CAAHLJNF@clear_script_breakpoints?$AA@ 000000018003b8d8     sfc_debug:sfc_api.obj
 0002:000038f8       ??_C@_0BH@BAILBHDP@add_script_breakpoints?$AA@ 000000018003b8f8     sfc_debug:sfc_api.obj
 0002:00003910       ??_C@_0BH@KAKDDELG@set_script_breakpoints?$AA@ 000000018003b910     sfc_debug:sfc_api.obj
 0002:00003928       ??_C@_0BE@GAGDJPKA@set_eml_breakpoints?$AA@ 000000018003b928     sfc_debug:sfc_api.obj
 0002:00003940       ??_C@_0BA@NHOBHLLJ@set_breakpoints?$AA@ 000000018003b940     sfc_debug:sfc_api.obj
 0002:00003950       ??_C@_0BF@GOGOODJG@break_on_state_entry?$AA@ 000000018003b950     sfc_debug:sfc_api.obj
 0002:00003968       ??_C@_0BJ@FPOJDFBP@break_on_event_broadcast?$AA@ 000000018003b968     sfc_debug:sfc_api.obj
 0002:00003988       ??_C@_0BF@FJBBAFJ@break_on_chart_entry?$AA@ 000000018003b988     sfc_debug:sfc_api.obj
 0002:000039a0       ??_C@_0N@MHHEHLAI@browse_trace?$AA@ 000000018003b9a0     sfc_debug:sfc_api.obj
 0002:000039b0       ??_C@_0BB@JEAJMJMI@consistency_info?$AA@ 000000018003b9b0     sfc_debug:sfc_api.obj
 0002:000039c4       ??_C@_04MLCEENPJ@whos?$AA@ 000000018003b9c4     sfc_debug:sfc_api.obj
 0002:000039d0       ??_C@_0L@LNIDAIN@watch_data?$AA@ 000000018003b9d0     sfc_debug:sfc_api.obj
 0002:000039e0       ??_C@_0M@JEJMEFEG@browse_data?$AA@ 000000018003b9e0     sfc_debug:sfc_api.obj
 0002:000039ec       ??_C@_03HNAFFKGA@get?$AA@  000000018003b9ec     sfc_debug:sfc_api.obj
 0002:000039f0       ??_C@_05LBOHBHFK@close?$AA@ 000000018003b9f0     sfc_debug:sfc_api.obj
 0002:000039f8       ??_C@_0BM@ICDFOOIE@set_disable_all_breakpoints?$AA@ 000000018003b9f8     sfc_debug:sfc_api.obj
 0002:00003a18       ??_C@_0BP@IBIALPGH@disable_all_breakpoints_and_go?$AA@ 000000018003ba18     sfc_debug:sfc_api.obj
 0002:00003a38       ??_C@_0BJ@BOMFHJBD@is_array_bounds_detected?$AA@ 000000018003ba38     sfc_debug:sfc_api.obj
 0002:00003a58       ??_C@_0BC@LKOOEAAH@is_cycle_detected?$AA@ 000000018003ba58     sfc_debug:sfc_api.obj
 0002:00003a70       ??_C@_0P@NIBPNIDJ@stop_debugging?$AA@ 000000018003ba70     sfc_debug:sfc_api.obj
 0002:00003a80       ??_C@_05ELPHFHOI@break?$AA@ 000000018003ba80     sfc_debug:sfc_api.obj
 0002:00003a88       ??_C@_06PLELHCEK@resume?$AA@ 000000018003ba88     sfc_debug:sfc_api.obj
 0002:00003a90       ??_C@_08OKABEMKO@step_out?$AA@ 000000018003ba90     sfc_debug:sfc_api.obj
 0002:00003aa0       ??_C@_09CDNMPCHO@step_over?$AA@ 000000018003baa0     sfc_debug:sfc_api.obj
 0002:00003aac       ??_C@_02KPEDIMCA@go?$AA@   000000018003baac     sfc_debug:sfc_api.obj
 0002:00003ab0       ??_C@_0P@MMCMIGPN@debugger_alive?$AA@ 000000018003bab0     sfc_debug:sfc_api.obj
 0002:00003ac0       ??_C@_0N@GHFBLJDM@machine_load?$AA@ 000000018003bac0     sfc_debug:sfc_api.obj
 0002:00003ad0       ??_C@_0O@GIBFCMLF@chart_visible?$AA@ 000000018003bad0     sfc_debug:sfc_api.obj
 0002:00003ef0       ??_C@_05JEMLEKKA@found?$AA@ 000000018003bef0     sfc_debug:sfc_api.obj
 0002:00003ef8       ??_C@_09KFNMLIAN@sfc_api?4c?$AA@ 000000018003bef8     sfc_debug:sfc_api.obj
 0002:00003f08       ??_C@_0N@PFBMDOLG@sf_debug_api?$AA@ 000000018003bf08     sfc_debug:sfc_api.obj
 0002:00003f18       ??_C@_07KEAHHHLK@nrhs?$DN?$DN3?$AA@ 000000018003bf18     sfc_debug:sfc_api.obj
 0002:00003f20       ??_C@_0BC@HOOMKBNL@mxIsChar?$CIprhs?$FL0?$FN?$CJ?$AA@ 000000018003bf20     sfc_debug:sfc_api.obj
 0002:00003f38       ??_C@_0BF@NGLAGMHA@mxIsNumeric?$CIprhs?$FL0?$FN?$CJ?$AA@ 000000018003bf38     sfc_debug:sfc_api.obj
 0002:00003f50       ??_C@_07IEIELKNG@nrhs?$DO?$DN1?$AA@ 000000018003bf50     sfc_debug:sfc_api.obj
 0002:00003f58       ??_C@_07LNBMEGPL@nrhs?$DN?$DN2?$AA@ 000000018003bf58     sfc_debug:sfc_api.obj
 0002:00003f60       ??_C@_0BD@DPNMCCEH@nrhs?$DN?$DN1?5?$HM?$HM?5nrhs?$DN?$DN3?$AA@ 000000018003bf60     sfc_debug:sfc_api.obj
 0002:00003f78       ??_C@_09FKOBHCEN@nrhs?5?$DN?$DN?52?$AA@ 000000018003bf78     sfc_debug:sfc_api.obj
 0002:00003f88       ??_C@_09EMKMAIDO@nrhs?5?$DM?$DN?51?$AA@ 000000018003bf88     sfc_debug:sfc_api.obj
 0002:00003f98       ??_C@_07OLEGOBHN@nrhs?$DN?$DN4?$AA@ 000000018003bf98     sfc_debug:sfc_api.obj
 0002:00003fa0       ??_C@_07PCFNNADM@nrhs?$DN?$DN5?$AA@ 000000018003bfa0     sfc_debug:sfc_api.obj
 0002:00003fa8       ??_C@_07JGDBBFDI@nrhs?$DN?$DN1?$AA@ 000000018003bfa8     sfc_debug:sfc_api.obj
 0002:00003fb0       ??_C@_07KBNAPCKL@nlhs?$DN?$DN1?$AA@ 000000018003bfb0     sfc_debug:sfc_api.obj
 0002:00003fb8       ??_C@_08PAMHJLPB@statusOk?$AA@ 000000018003bfb8     sfc_debug:sfc_api.obj
 0002:00003fc8       ??_C@_07NJHAIDPP@nrhs?$DN?$DN6?$AA@ 000000018003bfc8     sfc_debug:sfc_api.obj
 0002:00003fd0       ??_C@_0L@EMNHGDGL@nlhs?$DN?$DNnrhs?$AA@ 000000018003bfd0     sfc_debug:sfc_api.obj
 0002:00003fe0       ??_C@_0P@BLJCAHMG@select_objects?$AA@ 000000018003bfe0     sfc_debug:sfdb_animation.obj
 0002:00003ff0       ??_C@_06CFKBOPCI@states?$AA@ 000000018003bff0     sfc_debug:sfdb_animation.obj
 0002:00003ff8       ??_C@_0P@KHIIFDEG@instanceHandle?$AA@ 000000018003bff8     sfc_debug:sfdb_animation.obj
 0002:00004008       ??_C@_0P@DEIGLMOE@instanceNumber?$AA@ 000000018003c008     sfc_debug:sfdb_animation.obj
 0002:00004018       ??_C@_0N@HACOJJON@instanceName?$AA@ 000000018003c018     sfc_debug:sfdb_animation.obj
 0002:00004028       ??_C@_0M@BFNIOHPP@chartNumber?$AA@ 000000018003c028     sfc_debug:sfdb_animation.obj
 0002:00004038       ??_C@_09KMHJEGJ@chartName?$AA@ 000000018003c038     sfc_debug:sfdb_animation.obj
 0002:00004044       ??_C@_06OOECHJN@charts?$AA@ 000000018003c044     sfc_debug:sfdb_animation.obj
 0002:00004050       ??_C@_0O@LOMGGENK@machineNumber?$AA@ 000000018003c050     sfc_debug:sfdb_animation.obj
 0002:00004060       ??_C@_09OOJCKABH@machineId?$AA@ 000000018003c060     sfc_debug:sfdb_animation.obj
 0002:00004070       ??_C@_0M@OCOCCFP@machineName?$AA@ 000000018003c070     sfc_debug:sfdb_animation.obj
 0002:00004080       ??_C@_0CN@CCJEMGOM@?$CIinstance?9?$DOsm?4statePack?$CJ?4length?$DO@ 000000018003c080     sfc_debug:sfdb_animation.obj
 0002:000040b0       ??_C@_0DC@DKAJIDPA@?$CIinstance?9?$DOsm?4transitionPack?$CJ?4le@ 000000018003c0b0     sfc_debug:sfdb_animation.obj
 0002:000040e8       ??_C@_0BB@EGGLBLCL@sfdb_animation?4c?$AA@ 000000018003c0e8     sfc_debug:sfdb_animation.obj
 0002:00004100       ??_C@_0BB@GDGPIGLB@cv_model_enabled?$AA@ 000000018003c100     sfc_debug:cv_sfinterface.obj
 0002:00004118       ??_C@_09DDDNMFIJ@get_param?$AA@ 000000018003c118     sfc_debug:cv_sfinterface.obj
 0002:00004128       ??_C@_0L@BODNDPN@CoverageId?$AA@ 000000018003c128     sfc_debug:cv_sfinterface.obj
 0002:00004138       __real@4008000000000000    000000018003c138     sfc_debug:cv_sfinterface.obj
 0002:00004140       ??_C@_05IEGMLJMJ@exist?$AA@ 000000018003c140     sfc_debug:cv_sfinterface.obj
 0002:00004148       ??_C@_02DDEKINOE@cv?$AA@   000000018003c148     sfc_debug:cv_sfinterface.obj
 0002:00004150       __real@4082c00000000000    000000018003c150     sfc_debug:cv_sfinterface.obj
 0002:00004158       ??_C@_0O@HGNEKHDK@MatlabVersion?$AA@ 000000018003c158     sfc_debug:cv_sfinterface.obj
 0002:00004168       ??_C@_0M@IIAIMKFO@status?5?$DN?$DN?50?$AA@ 000000018003c168     sfc_debug:cv_sfinterface.obj
 0002:00004178       ??_C@_0BB@ENEMAMMG@cv_sfinterface?4c?$AA@ 000000018003c178     sfc_debug:cv_sfinterface.obj
 0002:00004190       ??_C@_0CC@JMPFGLON@mxGetNumberOfElements?$CIplhs?$FL3?$FN?$CJ?$DN?$DN@ 000000018003c190     sfc_debug:cv_sfinterface.obj
 0002:000041b8       ??_C@_0P@MCDOIOOF@plhs?$FL3?$FN?5?$CB?$DNNULL?$AA@ 000000018003c1b8     sfc_debug:cv_sfinterface.obj
 0002:000041c8       ??_C@_0P@HAMLCBNF@len?$DM?$DNdataCount?$AA@ 000000018003c1c8     sfc_debug:cv_sfinterface.obj
 0002:000041d8       ??_C@_0BA@FJOAHKLL@len?$DN?$DNtransCount?$AA@ 000000018003c1d8     sfc_debug:cv_sfinterface.obj
 0002:000041e8       ??_C@_0BA@JELAJLGI@len?$DN?$DNstateCount?$AA@ 000000018003c1e8     sfc_debug:cv_sfinterface.obj
 0002:000041f8       ??_C@_0BC@NEFBEIHN@InitChartInstance?$AA@ 000000018003c1f8     sfc_debug:cv_sfinterface.obj
 0002:0000420c       ??_C@_04MMALOABH@cvsf?$AA@ 000000018003c20c     sfc_debug:cv_sfinterface.obj
 0002:00004218       ??_C@_0L@GIEKKEHF@InitScript?$AA@ 000000018003c218     sfc_debug:cv_sfinterface.obj
 0002:00004228       ??_C@_08DNDOONPK@sigrange?$AA@ 000000018003c228     sfc_debug:cv_sfinterface.obj
 0002:00004238       ??_C@_0O@KGBGEHIN@MetricEnabled?$AA@ 000000018003c238     sfc_debug:cv_sfinterface.obj
 0002:00004248       ??_C@_0BC@NKPEPJDJ@chart?9?$DOchartId?$CB?$DN0?$AA@ 000000018003c248     sfc_debug:cv_sfinterface.obj
 0002:0000425c       ??_C@_02GMHACPFF@?$CFu?$AA@ 000000018003c25c     sfc_debug:sfdb_data_browse.obj
 0002:00004260       ??_C@_02NJPGOMH@?$CFf?$AA@ 000000018003c260     sfc_debug:sfdb_data_browse.obj
 0002:00004268       ??_C@_0BD@PCGIEHBF@sfdb_data_browse?4c?$AA@ 000000018003c268     sfc_debug:sfdb_data_browse.obj
 0002:00004280       __real@c2a2309ce53fffcd    000000018003c280     sfc_debug:sfdb_data_browse.obj
 0002:00004288       ??_C@_0CK@JKBFHDPL@result?5?$DN?5mxCreateDoubleMatrix?$CI1?0@ 000000018003c288     sfc_debug:sfdb_data_browse.obj
 0002:000042b8       ??_C@_0DK@FJDNFCNK@result?5?$DN?5mxCreateDoubleMatrix?$CI1?0@ 000000018003c2b8     sfc_debug:sfdb_data_browse.obj
 0002:000042f8       ??_C@_0DL@OAKPHGJG@result?5?$DN?5mxCreateDoubleMatrix?$CI1?0@ 000000018003c2f8     sfc_debug:sfdb_data_browse.obj
 0002:00004338       ??_C@_0N@MNGHGLAH@isFixedPoint?$AA@ 000000018003c338     sfc_debug:sfdb_data_browse.obj
 0002:00004348       ??_C@_06DLEPGFEF@format?$AA@ 000000018003c348     sfc_debug:sfdb_data_browse.obj
 0002:00004350       ??_C@_05MFEJDJP@value?$AA@ 000000018003c350     sfc_debug:sfdb_data_browse.obj
 0002:00004358       ??_C@_05DCCHDMEJ@scope?$AA@ 000000018003c358     sfc_debug:sfdb_data_browse.obj
 0002:00004360       ??_C@_02EGCJHIOB@id?$AA@   000000018003c360     sfc_debug:sfdb_data_browse.obj
 0002:00004364       ??_C@_04PJOLNDGD@data?$AA@ 000000018003c364     sfc_debug:sfdb_data_browse.obj
 0002:0000436c       ??_C@_06LIBBAANI@len?$DN?$DN1?$AA@ 000000018003c36c     sfc_debug:sfdb_handle_management.obj
 0002:00004378       ??_C@_0BJ@IEEBKHME@sfdb_handle_management?4c?$AA@ 000000018003c378     sfc_debug:sfdb_handle_management.obj
 0002:00004394       ??_C@_06NCGDPKCC@handle?$AA@ 000000018003c394     sfc_debug:sfdb_handle_management.obj
 0002:000043a0       ??_C@_0BP@NAIIDBEE@parentObjectType?$DN?$DNCHART_OBJECT?$AA@ 000000018003c3a0     sfc_debug:sfdb_handle_management.obj
 0002:000043c0       ??_C@_0BD@JOOOIBOE@get_machine_option?$AA@ 000000018003c3c0     sfc_debug:sfdb_handle_management.obj
 0002:000043d8       ??_C@_0P@KGLBOIAN@get_machine_id?$AA@ 000000018003c3d8     sfc_debug:sfdb_handle_management.obj
 0002:000043e8       ??_C@_0N@OBHOGINE@get_chart_id?$AA@ 000000018003c3e8     sfc_debug:sfdb_handle_management.obj
 0002:000043f8       ??_C@_0BD@DICPGEAM@register_sfunction?$AA@ 000000018003c3f8     sfc_debug:sfdb_handle_management.obj
 0002:00004410       ??_C@_0BF@FENDCECP@get_chart_visibility?$AA@ 000000018003c410     sfc_debug:sfdb_handle_management.obj
 0002:00004428       ??_C@_0BM@FDGIEMLG@objectProperties?9?$DOlength?$DN?$DN0?$AA@ 000000018003c428     sfc_debug:sfdb_handle_management.obj
 0002:00004448       ??_C@_0CE@KBPIEDGG@?$CI?$CI?$CKobjectProperties?$CJ?$CJ?4length?$DOnum@ 000000018003c448     sfc_debug:sfdb_handle_management.obj
 0002:00004470       ??_C@_0CA@HFGDFECP@len?5?$DN?$DN?5objectProperties?9?$DOlength?$AA@ 000000018003c470     sfc_debug:sfdb_handle_management.obj
 0002:00004490       ??_C@_0P@BHPLCHGJ@get_object_ids?$AA@ 000000018003c490     sfc_debug:sfdb_handle_management.obj
 0002:000044a0       ??_C@_0BK@IFFOLHLE@objectProperties?9?$DOsize?$DN?$DN0?$AA@ 000000018003c4a0     sfc_debug:sfdb_handle_management.obj
 0002:000044c0       ??_C@_0BO@GFLPGHHM@len?5?$DO?$DN?5objectProperties?9?$DOsize?$AA@ 000000018003c4c0     sfc_debug:sfdb_handle_management.obj
 0002:000044e0       ??_C@_05GFHEIIDD@event?$AA@ 000000018003c4e0     sfc_debug:sfdb_handle_management.obj
 0002:000044e8       ??_C@_0M@BFOKCNLA@debug?4watch?$AA@ 000000018003c4e8     sfc_debug:sfdb_handle_management.obj
 0002:000044f8       ??_C@_0CE@OILCPIFA@machine?4debug?4disableAllBreakpoi@ 000000018003c4f8     sfc_debug:sfdb_handle_management.obj
 0002:00004520       ??_C@_0DA@JMDEGBBH@machine?4debug?4runTimeCheck?4state@ 000000018003c520     sfc_debug:sfdb_handle_management.obj
 0002:00004550       ??_C@_0CP@IPHIMGFA@machine?4debug?4runTimeCheck?4trans@ 000000018003c550     sfc_debug:sfdb_handle_management.obj
 0002:00004580       ??_C@_0CL@LENOAAKD@machine?4debug?4runTimeCheck?4dataR@ 000000018003c580     sfc_debug:sfdb_handle_management.obj
 0002:000045b0       ??_C@_0CK@MBMAMLGE@machine?4debug?4runTimeCheck?4cycle@ 000000018003c5b0     sfc_debug:sfdb_handle_management.obj
 0002:000045e0       ??_C@_0CA@EGLALCO@machine?4debug?4animation?4enabled?$AA@ 000000018003c5e0     sfc_debug:sfdb_handle_management.obj
 0002:00004600       ??_C@_0L@KGLELNDP@transition?$AA@ 000000018003c600     sfc_debug:sfdb_handle_management.obj
 0002:0000460c       ??_C@_06JKPEPHBG@dst?4id?$AA@ 000000018003c60c     sfc_debug:sfdb_handle_management.obj
 0002:00004614       ??_C@_05HDBKIDE@state?$AA@ 000000018003c614     sfc_debug:sfdb_handle_management.obj
 0002:00004620       ??_C@_0EG@MFIKDIJB@strlen?$CImachineName?$CJ?5?$DM?5sizeof?$CIdeb@ 000000018003c620     sfc_debug:sfdb_handle_management.obj
 0002:00004668       ??_C@_0BM@DEONCIBN@stackPtr?5?$DN?$DN?5symScope?9?$DOstack?$AA@ 000000018003c668     sfc_debug:sfdb_symbol_scope.obj
 0002:00004688       ??_C@_0BE@PIKAOBFK@sfdb_symbol_scope?4c?$AA@ 000000018003c688     sfc_debug:sfdb_symbol_scope.obj
 0002:000046a0       ??_C@_0BP@MJGDIBPE@symScope?9?$DOcurrentScope?5?$CB?$DN?5NULL?$AA@ 000000018003c6a0     sfc_debug:sfdb_symbol_scope.obj
 0002:000046c0       ??_C@_0BP@OCHHKFJA@symScope?9?$DOcurrentScope?5?$DN?$DN?5NULL?$AA@ 000000018003c6c0     sfc_debug:sfdb_symbol_scope.obj
 0002:000046e0       ??_C@_0BM@KCIKANPA@symScope?9?$DOstack?5?$DN?$DN?5stackPtr?$AA@ 000000018003c6e0     sfc_debug:sfdb_symbol_scope.obj
 0002:00004700       ??_C@_0DK@NCABFGD@symScope?9?$DOcurrentScope?5?$CB?$DN?5NULL?5?$CG@ 000000018003c700     sfc_debug:sfdb_symbol_scope.obj
 0002:00004740       ??_C@_0DL@LDAGNOEE@currScope?9?$DOsymbolTable?4count?5?$DM?5c@ 000000018003c740     sfc_debug:sfdb_symbol_scope.obj
 0002:00004780       ??_C@_0BK@PHCKFGOO@numDims?5?$DM?$DN?5MAX_DIMENSIONS?$AA@ 000000018003c780     sfc_debug:sfdb_symbol_scope.obj
 0002:000047a0       ??_C@_0EE@CLCFNFKP@Warning?3?5Can?8t?5display?5value?4?5Nu@ 000000018003c7a0     sfc_debug:sfdb_symbol_scope.obj
 0002:000047e8       ??_C@_0BB@NPDHFBEP@valuePtr?5?$CB?$DN?5NULL?$AA@ 000000018003c7e8     sfc_debug:sfdb_symbol_scope.obj
 0002:00004800       ??_C@_0O@CHHKIHJE@chart?5?$CB?$DN?5NULL?$AA@ 000000018003c800     sfc_debug:sfdb_symbol_scope.obj
 0002:00004810       ??_C@_0CB@PFGINMAC@dataInfo?5?$CG?$CG?5data?5?$CG?$CG?5st?5?$CG?$CG?5i?5?$DO?$DN?50@ 000000018003c810     sfc_debug:sfdb_symbol_scope.obj
 0002:00004840       ??_C@_0PC@ENOLANEC@Cannot?5change?5value?5of?5?8?$CFs?8?5at?5d@ 000000018003c840     sfc_debug:sfdb_symbol_scope.obj
 0002:00004934       ??_C@_02PINLEBJB@fi?$AA@   000000018003c934     sfc_debug:sfdb_symbol_scope.obj
 0002:00004938       ??_C@_06FDANFAAP@sim2fi?$AA@ 000000018003c938     sfc_debug:sfdb_symbol_scope.obj
 0002:00004940       ??_C@_0N@PGGMJAFA@Out?5of?5Scope?$AA@ 000000018003c940     sfc_debug:sfdb_symbol_scope.obj
 0002:00004950       ??_C@_0BF@KFJKGDMO@Unrecognized?5symbol?4?$AA@ 000000018003c950     sfc_debug:sfdb_symbol_scope.obj
 0002:00004968       ??_C@_0L@INJGJGAM@?5?$CIcomplex?$CJ?$AA@ 000000018003c968     sfc_debug:sfdb_symbol_scope.obj
 0002:00004978       ??_C@_0O@MHGLJPE@fixpt?5?$CI?$CFs?5?$CFs?$CJ?$AA@ 000000018003c978     sfc_debug:sfdb_symbol_scope.obj
 0002:00004988       ??_C@_08FFKICJMO@?$CFs?$CL?$CF?416g?$AA@ 000000018003c988     sfc_debug:sfdb_symbol_scope.obj
 0002:00004994       ??_C@_02EPPPECEI@SI?$AA@   000000018003c994     sfc_debug:sfdb_symbol_scope.obj
 0002:00004998       ??_C@_09LKFGHFHF@?$CFs?$CI2?$FO?$CFd?$CJ?$CK?$AA@ 000000018003c998     sfc_debug:sfdb_symbol_scope.obj
 0002:000049a4       ??_C@_06KJECHFDK@?$CF?416g?$CK?$AA@ 000000018003c9a4     sfc_debug:sfdb_symbol_scope.obj
 0002:000049ac       ??_C@_02IJPJFKDF@ml?$AA@   000000018003c9ac     sfc_debug:sfdb_symbol_scope.obj
 0002:000049b0       ??_C@_0O@NJOJHIHO@logical?5array?$AA@ 000000018003c9b0     sfc_debug:sfdb_symbol_scope.obj
 0002:000049c0       ??_C@_0L@MDMKKENH@char?5array?$AA@ 000000018003c9c0     sfc_debug:sfdb_symbol_scope.obj
 0002:000049d0       ??_C@_0N@DGCGENML@uint32?5array?$AA@ 000000018003c9d0     sfc_debug:sfdb_symbol_scope.obj
 0002:000049e0       ??_C@_0M@OFFMACLB@int32?5array?$AA@ 000000018003c9e0     sfc_debug:sfdb_symbol_scope.obj
 0002:000049f0       ??_C@_0N@JMJKGLLH@uint16?5array?$AA@ 000000018003c9f0     sfc_debug:sfdb_symbol_scope.obj
 0002:00004a00       ??_C@_0M@EPOACEMN@int16?5array?$AA@ 000000018003ca00     sfc_debug:sfdb_symbol_scope.obj
 0002:00004a10       ??_C@_0M@NOMKNEGI@uint8?5array?$AA@ 000000018003ca10     sfc_debug:sfdb_symbol_scope.obj
 0002:00004a20       ??_C@_0L@HCHBFFAP@int8?5array?$AA@ 000000018003ca20     sfc_debug:sfdb_symbol_scope.obj
 0002:00004a30       ??_C@_0N@KIFCNMIF@single?5array?$AA@ 000000018003ca30     sfc_debug:sfdb_symbol_scope.obj
 0002:00004a40       ??_C@_0N@OFOFFBCM@double?5array?$AA@ 000000018003ca40     sfc_debug:sfdb_symbol_scope.obj
 0002:00004a50       ??_C@_04BIAHPGJI@?$CFdx1?$AA@ 000000018003ca50     sfc_debug:sfdb_symbol_scope.obj
 0002:00004a58       ??_C@_04CADIJHHA@?$CFd?9D?$AA@ 000000018003ca58     sfc_debug:sfdb_symbol_scope.obj
 0002:00004a60       ??_C@_05JIPKJPMI@?$CFs?$CFdx?$AA@ 000000018003ca60     sfc_debug:sfdb_symbol_scope.obj
 0002:00004a68       ??_C@_0BH@GLACFBLP@?5?$CIvariable?5sized?3?5MAX?5?$AA@ 000000018003ca68     sfc_debug:sfdb_symbol_scope.obj
 0002:00004a80       ??_C@_07CIFAGBMG@unknown?$AA@ 000000018003ca80     sfc_debug:sfdb_symbol_scope.obj
 0002:00004a88       ??_C@_05ENKANFLO@class?$AA@ 000000018003ca88     sfc_debug:sfdb_symbol_scope.obj
 0002:00004a90       ??_C@_05FBJAGGIG@bytes?$AA@ 000000018003ca90     sfc_debug:sfdb_symbol_scope.obj
 0002:00004a98       ??_C@_04MEMAJGDJ@name?$AA@ 000000018003ca98     sfc_debug:sfdb_symbol_scope.obj
 0002:00004aa0       ??_C@_0CF@NELOECCL@coverageVector?9?$DOlength?$DOcoverageI@ 000000018003caa0     sfc_debug:sfdb_coverage.obj
 0002:00004ac8       ??_C@_0BA@CBMBNBFB@sfdb_coverage?4c?$AA@ 000000018003cac8     sfc_debug:sfdb_coverage.obj
 0002:00004ad8       ??_C@_0DN@FAEHHEAM@?$CIscript?9?$DObm?4breakpoints?$CJ?4length?$DO@ 000000018003cad8     sfc_debug:sfdb_breakpoints.obj
 0002:00004b18       ??_C@_0BD@BABBLJFB@sfdb_breakpoints?4c?$AA@ 000000018003cb18     sfc_debug:sfdb_breakpoints.obj
 0002:00004b30       ??_C@_0P@IGHKOFID@get_script_bps?$AA@ 000000018003cb30     sfc_debug:sfdb_breakpoints.obj
 0002:00004b40       ??_C@_0BA@ICOJJJDD@get_all_scripts?$AA@ 000000018003cb40     sfc_debug:sfdb_breakpoints.obj
 0002:00004b50       ??_C@_0EI@EDDFBGGP@?$CIunsigned?5int?$CJ?$CImxGetM?$CIplhs?$FL0?$FN?$CJ?5?$CK@ 000000018003cb50     sfc_debug:sfdb_breakpoints.obj
 0002:00004b98       ??_C@_0BE@PNADEEOB@get_eml_line_counts?$AA@ 000000018003cb98     sfc_debug:sfdb_breakpoints.obj
 0002:00004bb0       ??_C@_0CC@JPCLBDPC@mxGetNumberOfElements?$CIplhs?$FL0?$FN?$CJ?$DN?$DN@ 000000018003cbb0     sfc_debug:sfdb_breakpoints.obj
 0002:00004bd8       ??_C@_0P@EHJHKHLL@get_global_bps?$AA@ 000000018003cbd8     sfc_debug:sfdb_breakpoints.obj
 0002:00004be8       ??_C@_0CE@NADCJCF@?$CIchart?9?$DObm?4chart?$FLtagType?$FN?$CJ?4lengt@ 000000018003cbe8     sfc_debug:sfdb_breakpoints.obj
 0002:00004c10       ??_C@_0CP@JOFCMAIP@?$CIchart?9?$DObm?4state?$FLtagType?$FN?$CJ?4lengt@ 000000018003cc10     sfc_debug:sfdb_breakpoints.obj
 0002:00004c40       ??_C@_0DE@GNPGALGC@?$CIchart?9?$DObm?4transition?$FLtagType?$FN?$CJ?4@ 000000018003cc40     sfc_debug:sfdb_breakpoints.obj
 0002:00004c78       ??_C@_0DB@PCFIPMMH@?$CImachine?9?$DObm?4event?$FLtagType?$FN?$CJ?4len@ 000000018003cc78     sfc_debug:sfdb_breakpoints.obj
 0002:00004cb0       ??_C@_0CP@FENPPAOI@?$CIchart?9?$DObm?4event?$FLtagType?$FN?$CJ?4lengt@ 000000018003ccb0     sfc_debug:sfdb_breakpoints.obj
 0002:00004ce0       ??_C@_0CH@EKAIFOIL@numCols?5?$DN?$DN?5TOTAL_EVENT_BREAKPOIN@ 000000018003cce0     sfc_debug:sfdb_breakpoints.obj
 0002:00004d08       ??_C@_0CA@BECONEOF@numRows?5?$DN?$DN?5machine?9?$DOevent?4count?$AA@ 000000018003cd08     sfc_debug:sfdb_breakpoints.obj
 0002:00004d28       ??_C@_07HCEBIAFG@get_bps?$AA@ 000000018003cd28     sfc_debug:sfdb_breakpoints.obj
 0002:00004d30       ??_C@_0BI@LFGGAIIJ@?$CIbps?$CJ?4length?$DObreakPoint?$AA@ 000000018003cd30     sfc_debug:sfdb_breakpoints.obj
 0002:00004d48       ??_C@_0N@CNOINHPD@numCols?5?$DN?$DN?51?$AA@ 000000018003cd48     sfc_debug:sfdb_breakpoints.obj
 0002:00004d58       ??_C@_0M@NNPJEEAE@get_eml_bps?$AA@ 000000018003cd58     sfc_debug:sfdb_breakpoints.obj
 0002:00004d68       ??_C@_0BO@CDPAPHEM@numRows?5?$DN?$DN?5chart?9?$DOevent?4count?$AA@ 000000018003cd68     sfc_debug:sfdb_breakpoints.obj
 0002:00004d88       ??_C@_0CM@FFJFHNEO@numCols?5?$DN?$DN?5TOTAL_TRANSITION_BREA@ 000000018003cd88     sfc_debug:sfdb_breakpoints.obj
 0002:00004db8       ??_C@_0CD@IOIMPEBN@numRows?5?$DN?$DN?5chart?9?$DOtransition?4cou@ 000000018003cdb8     sfc_debug:sfdb_breakpoints.obj
 0002:00004de0       ??_C@_0CH@JEIBGOOJ@numCols?5?$DN?$DN?5TOTAL_STATE_BREAKPOIN@ 000000018003cde0     sfc_debug:sfdb_breakpoints.obj
 0002:00004e08       ??_C@_0BO@BIKNFPLB@numRows?5?$DN?$DN?5chart?9?$DOstate?4count?$AA@ 000000018003ce08     sfc_debug:sfdb_breakpoints.obj
 0002:00004e28       ??_C@_0CH@BNLENKGD@numCols?5?$DN?$DN?5TOTAL_CHART_BREAKPOIN@ 000000018003ce28     sfc_debug:sfdb_breakpoints.obj
 0002:00004e50       ??_C@_0N@MEFFBAFI@numRows?5?$DN?$DN?51?$AA@ 000000018003ce50     sfc_debug:sfdb_breakpoints.obj
 0002:00004e60       ??_C@_0BJ@BLHBHILO@sfdb_state_consistency?4c?$AA@ 000000018003ce60     sfc_debug:sfdb_state_consistency.obj
 0002:00004e80       ??_C@_09LHFAMEGK@errorType?$AA@ 000000018003ce80     sfc_debug:sfdb_state_consistency.obj
 0002:00004e90       ??_C@_08DLAIKNBK@objectId?$AA@ 000000018003ce90     sfc_debug:sfdb_state_consistency.obj
 0002:00004ea0       ??_C@_0L@GODCDFEF@objectType?$AA@ 000000018003cea0     sfc_debug:sfdb_state_consistency.obj
 0002:00004eb0       ??_C@_0L@CCGENCKP@errorStack?$AA@ 000000018003ceb0     sfc_debug:sfdb_state_consistency.obj
 0002:00004ec0       ??_C@_0O@PPHMCEKO@cycleDetected?$AA@ 000000018003cec0     sfc_debug:sfdb_call_stack.obj
 0002:00004ed0       ??_C@_0N@MGKMJLEK@cycleStarted?$AA@ 000000018003ced0     sfc_debug:sfdb_call_stack.obj
 0002:00004ee0       ??_C@_07BNCILGOA@tagType?$AA@ 000000018003cee0     sfc_debug:sfdb_call_stack.obj
 0002:00004ee8       ??_C@_0L@POKIGEMP@eventScope?$AA@ 000000018003cee8     sfc_debug:sfdb_call_stack.obj
 0002:00004ef8       ??_C@_0M@LKJJPLIC@traceVector?$AA@ 000000018003cef8     sfc_debug:sfdb_call_stack.obj
 0002:00004f10       ??_C@_0EC@MGCLADPL@?$CIinstance?9?$DOcycleDetection?4transi@ 000000018003cf10     sfc_debug:sfdb_cycle_detection.obj
 0002:00004f58       ??_C@_0BH@ELCAAKDD@sfdb_cycle_detection?4c?$AA@ 000000018003cf58     sfc_debug:sfdb_cycle_detection.obj
 0002:00004f70       ??_C@_0O@PICIAFIK@newNode?$CB?$DNNULL?$AA@ 000000018003cf70     sfc_debug:sfdb_cycle_detection.obj
 0002:00004f80       _pDefaultRawDllMain        000000018003cf80     MSVCRT:crtdll.obj
 0002:00004f80       _pRawDllMain               000000018003cf80     MSVCRT:crtdll.obj
 0002:00004f98       ?ProcessDetach@NativeDll@<CrtImplementationDetails>@@0IB 000000018003cf98     MSVCRT:tncleanup.obj
 0002:00004f9c       ?ProcessAttach@NativeDll@<CrtImplementationDetails>@@0IB 000000018003cf9c     MSVCRT:tncleanup.obj
 0002:00004fa0       ?ThreadAttach@NativeDll@<CrtImplementationDetails>@@0IB 000000018003cfa0     MSVCRT:tncleanup.obj
 0002:00004fa4       ?ThreadDetach@NativeDll@<CrtImplementationDetails>@@0IB 000000018003cfa4     MSVCRT:tncleanup.obj
 0002:00004fa8       ?ProcessVerifier@NativeDll@<CrtImplementationDetails>@@0IB 000000018003cfa8     MSVCRT:tncleanup.obj
 0002:00004fb0       __rtc_iaa                  000000018003cfb0     MSVCRT:_initsect_.obj
 0002:00004fb8       __rtc_izz                  000000018003cfb8     MSVCRT:_initsect_.obj
 0002:00004fc0       __rtc_taa                  000000018003cfc0     MSVCRT:_initsect_.obj
 0002:00004fc8       __rtc_tzz                  000000018003cfc8     MSVCRT:_initsect_.obj
 0002:00008f64       __IMPORT_DESCRIPTOR_libmx  0000000180040f64     libmx:libmx.dll
 0002:00008f78       __IMPORT_DESCRIPTOR_libmex 0000000180040f78     libmex:libmex.dll
 0002:00008f8c       __IMPORT_DESCRIPTOR_libfixedpoint 0000000180040f8c     libfixedpoint:libfixedpoint.dll
 0002:00008fa0       __IMPORT_DESCRIPTOR_libut  0000000180040fa0     libut:libut.dll
 0002:00008fb4       __IMPORT_DESCRIPTOR_libemlrt 0000000180040fb4     libemlrt:libemlrt.dll
 0002:00008fc8       __IMPORT_DESCRIPTOR_MSVCR100 0000000180040fc8     MSVCRT:MSVCR100.dll
 0002:00008fdc       __IMPORT_DESCRIPTOR_KERNEL32 0000000180040fdc     kernel32:KERNEL32.dll
 0002:00008ff0       __NULL_IMPORT_DESCRIPTOR   0000000180040ff0     libmx:libmx.dll
 0003:00000b30       DYNAMIC_DIMENSION          0000000180042b30     openloop_DE_sfun_registry.obj
 0003:00001820       emlrtContextGlobal         0000000180043820     sfc_mex:sfc_mex.obj
 0003:000018c0       _fltused                   00000001800438c0     MSVCRT:dllsupp.obj
 0003:000018c8       __security_cookie          00000001800438c8     MSVCRT:gs_cookie.obj
 0003:000018d0       __security_cookie_complement 00000001800438d0     MSVCRT:gs_cookie.obj
 0003:000018e0       __native_dllmain_reason    00000001800438e0     MSVCRT:natstart.obj
 0003:000018e4       __native_vcclrit_reason    00000001800438e4     MSVCRT:natstart.obj
 0003:00002b18       emlrtRootTLSGlobal         0000000180044b18     sfc_mex:sfc_mex.obj
 0003:00002e08       sSFDebuggerInitialized     0000000180044e08     sfc_debug:sfcdebug.obj
 0003:00003ee0       ?__type_info_root_node@@3U__type_info_node@@A 0000000180045ee0     MSVCRT:tncleanup.obj
 0003:00003ef0       _openloop_DEMachineNumber_ 0000000180045ef0     <common>
 0003:00003ef8       _sfTime_                   0000000180045ef8     <common>
 0003:00003f00       gSfComplexDataTypeOffsets  0000000180045f00     <common>
 0003:00003f60       gSfDataTypeOffsets         0000000180045f60     <common>
 0003:00003fa8       gMaskBits                  0000000180045fa8     <common>
 0003:00003fb0       __native_startup_state     0000000180045fb0     <common>
 0003:00003fb8       __native_startup_lock      0000000180045fb8     <common>
 0003:00003fc0       __onexitend                0000000180045fc0     <common>
 0003:00003fc8       __onexitbegin              0000000180045fc8     <common>
 0003:00003fd0       __dyn_tls_init_callback    0000000180045fd0     <common>

 entry point at        0001:00036454

 Static symbols

 0001:00000fe0       get_sim_state_c2_openloop_DE 0000000180001fe0 f   c2_openloop_DE.obj
 0001:00001180       sf_get_sim_state_info_c2_openloop_DE 0000000180002180 f   c2_openloop_DE.obj
 0001:00001360       set_sim_state_c2_openloop_DE 0000000180002360 f   c2_openloop_DE.obj
 0001:00001440       c2_update_debugger_state_c2_openloop_DE 0000000180002440 f   c2_openloop_DE.obj
 0001:00001450       c2_emlrt_marshallIn        0000000180002450 f   c2_openloop_DE.obj
 0001:000014c0       c2_b_emlrt_marshallIn      00000001800024c0 f   c2_openloop_DE.obj
 0001:00001550       c2_e_emlrt_marshallIn      0000000180002550 f   c2_openloop_DE.obj
 0001:000015b0       c2_f_emlrt_marshallIn      00000001800025b0 f   c2_openloop_DE.obj
 0001:000016b0       mdlProcessParameters_c2_openloop_DE 00000001800026b0 f   c2_openloop_DE.obj
 0001:00001770       initialize_params_c2_openloop_DE 0000000180002770 f   c2_openloop_DE.obj
 0001:000019a0       mdlSetWorkWidths_c2_openloop_DE 00000001800029a0 f   c2_openloop_DE.obj
 0001:00002040       sf_get_instance_specialization 0000000180003040 f   c2_openloop_DE.obj
 0001:00002050       mdlStart_c2_openloop_DE    0000000180003050 f   c2_openloop_DE.obj
 0001:00002250       init_dsm_address_info      0000000180003250 f   c2_openloop_DE.obj
 0001:00002260       chart_debug_initialization 0000000180003260 f   c2_openloop_DE.obj
 0001:00002ee0       init_script_number_translation 0000000180003ee0 f   c2_openloop_DE.obj
 0001:00002ef0       c2_sf_marshallOut          0000000180003ef0 f   c2_openloop_DE.obj
 0001:00002fa0       c2_sf_marshallIn           0000000180003fa0 f   c2_openloop_DE.obj
 0001:00003040       c2_b_sf_marshallOut        0000000180004040 f   c2_openloop_DE.obj
 0001:00003180       c2_b_sf_marshallIn         0000000180004180 f   c2_openloop_DE.obj
 0001:00003250       c2_c_emlrt_marshallIn      0000000180004250 f   c2_openloop_DE.obj
 0001:00003330       c2_c_sf_marshallOut        0000000180004330 f   c2_openloop_DE.obj
 0001:00003460       sf_opaque_initialize_c2_openloop_DE 0000000180004460 f   c2_openloop_DE.obj
 0001:000034a0       initialize_c2_openloop_DE  00000001800044a0 f   c2_openloop_DE.obj
 0001:000034f0       sf_opaque_enable_c2_openloop_DE 00000001800044f0 f   c2_openloop_DE.obj
 0001:00003510       enable_c2_openloop_DE      0000000180004510 f   c2_openloop_DE.obj
 0001:00003540       sf_opaque_disable_c2_openloop_DE 0000000180004540 f   c2_openloop_DE.obj
 0001:00003560       disable_c2_openloop_DE     0000000180004560 f   c2_openloop_DE.obj
 0001:00003590       sf_opaque_gateway_c2_openloop_DE 0000000180004590 f   c2_openloop_DE.obj
 0001:000035b0       sf_c2_openloop_DE          00000001800045b0 f   c2_openloop_DE.obj
 0001:00004300       sf_opaque_get_sim_state_c2_openloop_DE 0000000180005300 f   c2_openloop_DE.obj
 0001:00004320       sf_opaque_set_sim_state_c2_openloop_DE 0000000180005320 f   c2_openloop_DE.obj
 0001:00004350       sf_opaque_terminate_c2_openloop_DE 0000000180005350 f   c2_openloop_DE.obj
 0001:000043d0       finalize_c2_openloop_DE    00000001800053d0 f   c2_openloop_DE.obj
 0001:000043e0       sf_opaque_init_subchart_simstructs 00000001800053e0 f   c2_openloop_DE.obj
 0001:00004400       initSimStructsc2_openloop_DE 0000000180005400 f   c2_openloop_DE.obj
 0001:00004410       mdlRTW_c2_openloop_DE      0000000180005410 f   c2_openloop_DE.obj
 0001:00006000       _ssFatalError              0000000180007000 f   openloop_DE_sfun_registry.obj
 0001:000090b0       ProcessMexSfunctionCmdLineCall 000000018000a0b0 f   openloop_DE_sfun_registry.obj
 0001:000091a0       mdlGetTimeOfNextVarHit     000000018000a1a0 f   openloop_DE_sfun_registry.obj
 0001:000091f0       _ProcessMexSfunctionCmdLineCall 000000018000a1f0 f   openloop_DE_sfun_registry.obj
 0001:00009940       _CreateSimStruct           000000018000a940 f   openloop_DE_sfun_registry.obj
 0001:00009ad0       _RegNumInputPortsCB        000000018000aad0 f   openloop_DE_sfun_registry.obj
 0001:00009b50       _RegNumOutputPortsCB       000000018000ab50 f   openloop_DE_sfun_registry.obj
 0001:00009c30       sf_machine_load_sfunction_ptrs 000000018000ac30 f   openloop_DE_sfun_registry.obj
 0001:0000a560       getThreadLocalStorage      000000018000b560 f   sfc_mex:sfc_mex.obj
 0001:0000a5a0       releaseThreadLocalStorage  000000018000b5a0 f   sfc_mex:sfc_mex.obj
 0001:0000a5b0       SNPRINTF_WRAPPER           000000018000b5b0 f   sfc_mex:sfc_mex.obj
 0001:0000a5d0       convert_dims_to_string     000000018000b5d0 f   sfc_mex:sfc_mex.obj
 0001:0000a7f0       is_real_T_equal_to_double  000000018000b7f0 f   sfc_mex:sfc_mex.obj
 0001:0000a810       is_real32_T_equal_to_double 000000018000b810 f   sfc_mex:sfc_mex.obj
 0001:0000a820       is_mxLogical_equal_to_double 000000018000b820 f   sfc_mex:sfc_mex.obj
 0001:0000a840       is_int8_T_equal_to_double  000000018000b840 f   sfc_mex:sfc_mex.obj
 0001:0000a860       is_uint8_T_equal_to_double 000000018000b860 f   sfc_mex:sfc_mex.obj
 0001:0000a880       is_int16_T_equal_to_double 000000018000b880 f   sfc_mex:sfc_mex.obj
 0001:0000a8a0       is_uint16_T_equal_to_double 000000018000b8a0 f   sfc_mex:sfc_mex.obj
 0001:0000a8c0       is_int32_T_equal_to_double 000000018000b8c0 f   sfc_mex:sfc_mex.obj
 0001:0000a8e0       is_uint32_T_equal_to_double 000000018000b8e0 f   sfc_mex:sfc_mex.obj
 0001:0000a900       is_char_T_equal_to_double  000000018000b900 f   sfc_mex:sfc_mex.obj
 0001:0000a920       sf_zero_numeric_value      000000018000b920 f   sfc_mex:sfc_mex.obj
 0001:0000a950       sf_error_append_debugger_context_if_available 000000018000b950 f   sfc_mex:sfc_mex.obj
 0001:0000aa20       sf_mex_get_error_message_for_write 000000018000ba20 f   sfc_mex:sfc_mex.obj
 0001:0000aa50       replace_single_quotes_by_doubled_quotes 000000018000ba50 f   sfc_mex:sfc_mex.obj
 0001:0000ac90       sf_mex_get_formatted_error_string 000000018000bc90 f   sfc_mex:sfc_mex.obj
 0001:0000b210       sf_mex_destroy_array       000000018000c210 f   sfc_mex:sfc_mex.obj
 0001:0000b5a0       sfrtAddSize                000000018000c5a0 f   sfc_mex:sfc_mex.obj
 0001:0000b660       sfrtGenSizeString          000000018000c660 f   sfc_mex:sfc_mex.obj
 0001:0000b6d0       sfIsProperVector           000000018000c6d0 f   sfc_mex:sfc_mex.obj
 0001:0000b700       sfIsRowVector              000000018000c700 f   sfc_mex:sfc_mex.obj
 0001:0000b840       sf_ExtractMessageId        000000018000c840 f   sfc_mex:sfc_mex.obj
 0001:0000bb20       sf_mex_err                 000000018000cb20 f   sfc_mex:sfc_mex.obj
 0001:0000bbd0       sf_error_dimension_out_of_bound 000000018000cbd0 f   sfc_mex:sfc_mex.obj
 0001:0000bc90       sf_mex_check_and_set_actual_dimensions 000000018000cc90 f   sfc_mex:sfc_mex.obj
 0001:0000be70       sf_mex_check_complex       000000018000ce70 f   sfc_mex:sfc_mex.obj
 0001:0000bf00       sf_mex_check_sparse        000000018000cf00 f   sfc_mex:sfc_mex.obj
 0001:0000bf60       sf_mex_check_numerictype   000000018000cf60 f   sfc_mex:sfc_mex.obj
 0001:0000c0f0       sf_mex_check_fimath        000000018000d0f0 f   sfc_mex:sfc_mex.obj
 0001:0000cca0       size_mismatch_error        000000018000dca0 f   sfc_mex:sfc_mex.obj
 0001:0000d740       check_array_dimensions     000000018000e740 f   sfc_mex:sfc_mex.obj
 0001:0000d7b0       check_input_mxarray        000000018000e7b0 f   sfc_mex:sfc_mex.obj
 0001:0000def0       sf_numeric_value_to_double 000000018000eef0 f   sfc_mex:sfc_mex.obj
 0001:0000df40       ml_generic_out_of_bounds_check 000000018000ef40 f   sfc_mex:sfc_mex.obj
 0001:0000e110       ml_get_element_value_from_array 000000018000f110 f   sfc_mex:sfc_mex.obj
 0001:0000e4b0       _ml_generic_castability_check 000000018000f4b0 f   sfc_mex:sfc_mex.obj
 0001:0000f210       ml_generic_castability_check 0000000180010210 f   sfc_mex:sfc_mex.obj
 0001:0000f2b0       ml_check_mx_array_for_single_castability 00000001800102b0 f   sfc_mex:sfc_mex.obj
 0001:0000f350       ml_check_mx_array_for_logical_castability 0000000180010350 f   sfc_mex:sfc_mex.obj
 0001:0000f3f0       ml_check_mx_array_for_int8_castability 00000001800103f0 f   sfc_mex:sfc_mex.obj
 0001:0000f4a0       ml_check_mx_array_for_uint8_castability 00000001800104a0 f   sfc_mex:sfc_mex.obj
 0001:0000f500       ml_check_mx_array_for_int16_castability 0000000180010500 f   sfc_mex:sfc_mex.obj
 0001:0000f560       ml_check_mx_array_for_uint16_castability 0000000180010560 f   sfc_mex:sfc_mex.obj
 0001:0000f5c0       ml_check_mx_array_for_int32_castability 00000001800105c0 f   sfc_mex:sfc_mex.obj
 0001:0000f620       ml_check_mx_array_for_uint32_castability 0000000180010620 f   sfc_mex:sfc_mex.obj
 0001:0000f680       ml_check_mx_array_for_castability 0000000180010680 f   sfc_mex:sfc_mex.obj
 0001:0000ffb0       set_data_value             0000000180010fb0 f   sfc_mex:sfc_mex.obj
 0001:00010320       get_data_value             0000000180011320 f   sfc_mex:sfc_mex.obj
 0001:00010430       get_next_element_address   0000000180011430 f   sfc_mex:sfc_mex.obj
 0001:00010500       sf_normalize_index         0000000180011500 f   sfc_mex:sfc_mex.obj
 0001:00010890       ml_array_index_bound_check 0000000180011890 f   sfc_mex:sfc_mex.obj
 0001:000113b0       mx_value                   00000001800123b0 f   sfc_mex:sfc_mex.obj
 0001:00011400       sf_create_numeric_array    0000000180012400 f   sfc_mex:sfc_mex.obj
 0001:000114a0       sf_mex_assign_to_mx_array  00000001800124a0 f   sfc_mex:sfc_mex.obj
 0001:000117f0       assign_from_mx_array       00000001800127f0 f   sfc_mex:sfc_mex.obj
 0001:00012020       sf_mex_import_v            0000000180013020 f   sfc_mex:sfc_mex.obj
 0001:00012720       get_machine_and_chart_file_number 0000000180013720 f   sfc_mex:sfc_sf.obj
 0001:00012810       get_sfun_block_specialization 0000000180013810 f   sfc_mex:sfc_sf.obj
 0001:000128c0       call_sf_machine_global_method_dispatcher 00000001800138c0 f   sfc_mex:sfc_sf.obj
 0001:00012b10       mdl_zeroCrossings_processing 0000000180013b10 f   sfc_mex:sfc_sf.obj
 0001:00012be0       mdl_derivatives_processing 0000000180013be0 f   sfc_mex:sfc_sf.obj
 0001:00012ea0       mdl_outputs_continuous_legacy 0000000180013ea0 f   sfc_mex:sfc_sf.obj
 0001:00012f20       mdl_outputs_processing     0000000180013f20 f   sfc_mex:sfc_sf.obj
 0001:00013190       mdl_enable_processing      0000000180014190 f   sfc_mex:sfc_sf.obj
 0001:00013260       mdl_disable_processing     0000000180014260 f   sfc_mex:sfc_sf.obj
 0001:00013fd0       sf_call_output_fcn_enable_disable 0000000180014fd0 f   sfc_mex:sfc_sf.obj
 0001:00014250       set_dwork_information_from_mx_array 0000000180015250 f   sfc_mex:sfc_sf.obj
 0001:00014b10       ptr2mxStruct               0000000180015b10 f   sfc_mex:sfc_sf.obj
 0001:00014e20       SNPRINTF_WRAPPER           0000000180015e20 f   sfc_debug:sfcdebug.obj
 0001:00014e40       sf_debug_chart_instance_initialized_quick 0000000180015e40 f   sfc_debug:sfcdebug.obj
 0001:00014e50       sf_debug_chart_instance_initialized 0000000180015e50 f   sfc_debug:sfcdebug.obj
 0001:00014ff0       sfrtAddSize                0000000180015ff0 f   sfc_debug:sfcdebug.obj
 0001:000150b0       sfrtGenSizeString          00000001800160b0 f   sfc_debug:sfcdebug.obj
 0001:000157c0       fill_single_message_info   00000001800167c0 f   sfc_debug:sfcdebug.obj
 0001:00015980       sf_debug_sim_status_listener 0000000180016980 f   sfc_debug:sfcdebug.obj
 0001:00015ef0       sf_debug_form_mask_bits    0000000180016ef0 f   sfc_debug:sfcdebug.obj
 0001:00015f30       sf_debug_form_sf_data_type_offsets 0000000180016f30 f   sfc_debug:sfcdebug.obj
 0001:00015ff0       sf_debug_free_all          0000000180016ff0 f   sfc_debug:sfcdebug.obj
 0001:000161a0       sf_debug_append_debugger_context 00000001800171a0 f   sfc_debug:sfcdebug.obj
 0001:00016340       sf_debug_update_always_honor_breakpoints 0000000180017340 f   sfc_debug:sfcdebug.obj
 0001:00016510       local_strdup               0000000180017510 f   sfc_debug:sfcdebug.obj
 0001:000173f0       sf_debug_em_terminate      00000001800183f0 f   sfc_debug:sfcdebug.obj
 0001:00017430       sf_debug_push_eml_function 0000000180018430 f   sfc_debug:sfcdebug.obj
 0001:000174d0       sf_debug_pop_eml_function  00000001800184d0 f   sfc_debug:sfcdebug.obj
 0001:000181d0       sf_debug_get_machine_number_from_id_or_name 00000001800191d0 f   sfc_debug:sfcdebug.obj
 0001:00018320       sf_debug_get_chart_number_from_id 0000000180019320 f   sfc_debug:sfcdebug.obj
 0001:000190c0       sf_debug_transfer_control_to_debugger_GUI 000000018001a0c0 f   sfc_debug:sfcdebug.obj
 0001:0001a050       sf_debug_scripts_rehash    000000018001b050 f   sfc_debug:sfcdebug.obj
 0001:0001a290       sf_debug_get_script_line_count 000000018001b290 f   sfc_debug:sfcdebug.obj
 0001:0001abc0       cv_eml_state_cvId          000000018001bbc0 f   sfc_debug:sfcdebug.obj
 0001:0001ac30       cv_eml_trans_cvId          000000018001bc30 f   sfc_debug:sfcdebug.obj
 0001:0001bfc0       sf_debug_data_array_bounds_error 000000018001cfc0 f   sfc_debug:sfcdebug.obj
 0001:0001c3f0       eml_debug_runtime_error_doclink 000000018001d3f0 f   sfc_debug:sfcdebug.obj
 0001:0001c550       sf_debug_runtime_error     000000018001d550 f   sfc_debug:sfcdebug.obj
 0001:0001c5c0       sf_debug_matlab_error      000000018001d5c0 f   sfc_debug:sfcdebug.obj
 0001:0001cf00       sf_debug_data_value_error  000000018001df00 f   sfc_debug:sfcdebug.obj
 0001:0001d800       sf_debug_data_loss_error   000000018001e800 f   sfc_debug:sfcdebug.obj
 0001:0001e790       call_cv_range_check        000000018001f790 f   sfc_debug:sfcdebug.obj
 0001:0001ef60       sf_debug_invoke_cycle_detection_code 000000018001ff60 f   sfc_debug:sfcdebug.obj
 0001:0001fde0       sf_reset_debug_info_struct 0000000180020de0 f   sfc_debug:sfcdebug.obj
 0001:00020640       cv_script_cvId             0000000180021640 f   sfc_debug:sfcdebug.obj
 0001:000213a0       sfc_api_chart_visible      00000001800223a0 f   sfc_debug:sfc_api.obj
 0001:00021420       sfc_api_active_instance    0000000180022420 f   sfc_debug:sfc_api.obj
 0001:000214a0       sfc_api_machine_load       00000001800224a0 f   sfc_debug:sfc_api.obj
 0001:00021570       sfc_api_debugger_alive     0000000180022570 f   sfc_debug:sfc_api.obj
 0001:00021580       sfc_api_go                 0000000180022580 f   sfc_debug:sfc_api.obj
 0001:00021590       sfc_api_step_over          0000000180022590 f   sfc_debug:sfc_api.obj
 0001:000215a0       sfc_api_step_out           00000001800225a0 f   sfc_debug:sfc_api.obj
 0001:000215b0       sfc_api_resume             00000001800225b0 f   sfc_debug:sfc_api.obj
 0001:000215c0       sfc_api_break              00000001800225c0 f   sfc_debug:sfc_api.obj
 0001:000215d0       sfc_api_stop_debugging     00000001800225d0 f   sfc_debug:sfc_api.obj
 0001:00021620       sfc_api_is_cycle_detected  0000000180022620 f   sfc_debug:sfc_api.obj
 0001:00021670       sfc_api_is_array_bounds_detected 0000000180022670 f   sfc_debug:sfc_api.obj
 0001:000216c0       sfc_api_set_disable_all_breakpoints 00000001800226c0 f   sfc_debug:sfc_api.obj
 0001:00021730       sfc_api_disable_all_breakpoints_and_go 0000000180022730 f   sfc_debug:sfc_api.obj
 0001:00021740       sfc_api_close              0000000180022740 f   sfc_debug:sfc_api.obj
 0001:00021750       sfc_api_browse_data        0000000180022750 f   sfc_debug:sfc_api.obj
 0001:000217c0       sfc_api_watch_data         00000001800227c0 f   sfc_debug:sfc_api.obj
 0001:000218c0       sfc_api_extract_message_post_receive_info 00000001800228c0 f   sfc_debug:sfc_api.obj
 0001:000218e0       sfc_api_assign_data        00000001800228e0 f   sfc_debug:sfc_api.obj
 0001:00021980       sfc_api_whos               0000000180022980 f   sfc_debug:sfc_api.obj
 0001:00021a10       sfc_api_get_consistency_info 0000000180022a10 f   sfc_debug:sfc_api.obj
 0001:00021a20       sfc_api_browse_trace       0000000180022a20 f   sfc_debug:sfc_api.obj
 0001:00021a30       sfc_api_break_on_chart_entry 0000000180022a30 f   sfc_debug:sfc_api.obj
 0001:00021a50       sfc_api_break_on_event_broadcast 0000000180022a50 f   sfc_debug:sfc_api.obj
 0001:00021a70       sfc_api_break_on_state_entry 0000000180022a70 f   sfc_debug:sfc_api.obj
 0001:00021a90       sfc_api_set_watch          0000000180022a90 f   sfc_debug:sfc_api.obj
 0001:00021b30       sfc_api_set_breakpoints    0000000180022b30 f   sfc_debug:sfc_api.obj
 0001:00021bd0       sfc_api_set_eml_breakpoints 0000000180022bd0 f   sfc_debug:sfc_api.obj
 0001:00021c50       sfc_api_set_script_breakpoints 0000000180022c50 f   sfc_debug:sfc_api.obj
 0001:00021ca0       sfc_api_add_script_breakpoints 0000000180022ca0 f   sfc_debug:sfc_api.obj
 0001:00021cf0       sfc_api_clear_script_breakpoints 0000000180022cf0 f   sfc_debug:sfc_api.obj
 0001:00021d40       sfc_api_query_script_breakpoints 0000000180022d40 f   sfc_debug:sfc_api.obj
 0001:00021da0       sfc_api_get_script_id      0000000180022da0 f   sfc_debug:sfc_api.obj
 0001:00021e60       sfc_api_get_active_states  0000000180022e60 f   sfc_debug:sfc_api.obj
 0001:00021ee0       sfc_api_break_between_times 0000000180022ee0 f   sfc_debug:sfc_api.obj
 0001:00021f40       sfc_api_get_instance_handle 0000000180022f40 f   sfc_debug:sfc_api.obj
 0001:00021ff0       sfc_api_set_animation      0000000180022ff0 f   sfc_debug:sfc_api.obj
 0001:00022040       sfc_api_select_chart       0000000180023040 f   sfc_debug:sfc_api.obj
 0001:000220a0       sfc_api_select_charts      00000001800230a0 f   sfc_debug:sfc_api.obj
 0001:000220d0       sfc_api_cycle_detection_check 00000001800230d0 f   sfc_debug:sfc_api.obj
 0001:00022120       sfc_api_data_range_check   0000000180023120 f   sfc_debug:sfc_api.obj
 0001:00022170       sfc_api_transition_conflict_check 0000000180023170 f   sfc_debug:sfc_api.obj
 0001:000221c0       sfc_api_state_consistency_check 00000001800231c0 f   sfc_debug:sfc_api.obj
 0001:00022210       sfc_api_set_instance_cv_ids 0000000180023210 f   sfc_debug:sfc_api.obj
 0001:00022320       sfc_api_set_script_cv_ids  0000000180023320 f   sfc_debug:sfc_api.obj
 0001:000223d0       sfc_api_get_current_machine_id 00000001800233d0 f   sfc_debug:sfc_api.obj
 0001:00022400       sfc_api_get_current_machine_number 0000000180023400 f   sfc_debug:sfc_api.obj
 0001:00022430       sfc_api_get_current_chart_number 0000000180023430 f   sfc_debug:sfc_api.obj
 0001:00022460       sfc_api_get_current_instance_number 0000000180023460 f   sfc_debug:sfc_api.obj
 0001:00022490       sfc_api_get_current_instance_handle 0000000180023490 f   sfc_debug:sfc_api.obj
 0001:000224b0       sfc_api_get_current_is_minor_time_step 00000001800234b0 f   sfc_debug:sfc_api.obj
 0001:000224e0       sfc_api_get_current_machine_name 00000001800234e0 f   sfc_debug:sfc_api.obj
 0001:00022500       sfc_api_get_current_chart_id 0000000180023500 f   sfc_debug:sfc_api.obj
 0001:00022530       sfc_api_get_current_object_type 0000000180023530 f   sfc_debug:sfc_api.obj
 0001:00022560       sfc_api_get_current_event_type 0000000180023560 f   sfc_debug:sfc_api.obj
 0001:00022590       sfc_api_get_current_object_id 0000000180023590 f   sfc_debug:sfc_api.obj
 0001:000225c0       sfc_get_current_active_event_type 00000001800235c0 f   sfc_debug:sfc_api.obj
 0001:000225f0       sfc_api_get_current_active_event_id 00000001800235f0 f   sfc_debug:sfc_api.obj
 0001:00022620       sfc_api_get_current_simulation_time 0000000180023620 f   sfc_debug:sfc_api.obj
 0001:00022640       sfc_get_current_tag_type   0000000180023640 f   sfc_debug:sfc_api.obj
 0001:00022670       sfc_get_current_coverage_percentage 0000000180023670 f   sfc_debug:sfc_api.obj
 0001:00022690       sfc_get_current_statement_context 0000000180023690 f   sfc_debug:sfc_api.obj
 0001:000226b0       sfc_get_current_optional_integer 00000001800236b0 f   sfc_debug:sfc_api.obj
 0001:000226e0       sfc_get_current_statement_info 00000001800236e0 f   sfc_debug:sfc_api.obj
 0001:00022780       sfc_api_get                0000000180023780 f   sfc_debug:sfc_api.obj
 0001:000233f0       sf_debug_sm_fill_state_activity_data 00000001800243f0 f   sfc_debug:sfdb_animation.obj
 0001:00025cf0       void_ptr_stack_vector_free_total 0000000180026cf0 f   sfc_debug:sfdb_data_browse.obj
 0001:00025d80       sf_debug_st_terminate_machine 0000000180026d80 f   sfc_debug:sfdb_data_browse.obj
 0001:00025dc0       sf_debug_st_terminate_instance 0000000180026dc0 f   sfc_debug:sfdb_data_browse.obj
 0001:00026170       push_on_to_void_ptr_stack  0000000180027170 f   sfc_debug:sfdb_data_browse.obj
 0001:00026300       pop_from_void_ptr_stack    0000000180027300 f   sfc_debug:sfdb_data_browse.obj
 0001:00026430       sf_debug_st_get_data_value 0000000180027430 f   sfc_debug:sfdb_data_browse.obj
 0001:000269c0       mx_value                   00000001800279c0 f   sfc_debug:sfdb_data_browse.obj
 0001:00026a00       sf_debug_st_fill_data_struct 0000000180027a00 f   sfc_debug:sfdb_data_browse.obj
 0001:00026d40       data_type_format_strings   0000000180027d40 f   sfc_debug:sfdb_data_browse.obj
 0001:00026df0       sf_debug_st_fill_data      0000000180027df0 f   sfc_debug:sfdb_data_browse.obj
 0001:00027b40       sf_debug_hm_get_simulink_handle 0000000180028b40 f   sfc_debug:sfdb_handle_management.obj
 0001:00028640       sf_debug_hm_initialize_globals 0000000180029640 f   sfc_debug:sfdb_handle_management.obj
 0001:00028740       sf_debug_hm_get_machine_debug_flag 0000000180029740 f   sfc_debug:sfdb_handle_management.obj
 0001:000288b0       sf_debug_hm_get_machine_id 00000001800298b0 f   sfc_debug:sfdb_handle_management.obj
 0001:000289d0       sf_debug_hm_get_chart_id   00000001800299d0 f   sfc_debug:sfdb_handle_management.obj
 0001:00028b70       sf_debug_hm_register_executing_SFunction 0000000180029b70 f   sfc_debug:sfdb_handle_management.obj
 0001:00028f00       sf_debug_hm_form_object_boolean_properties 0000000180029f00 f   sfc_debug:sfdb_handle_management.obj
 0001:000291d0       sf_debug_hm_form_object_properties 000000018002a1d0 f   sfc_debug:sfdb_handle_management.obj
 0001:00029410       sf_debug_hm_terminate_charts 000000018002a410 f   sfc_debug:sfdb_handle_management.obj
 0001:00029b70       sf_debug_hm_terminate_machines 000000018002ab70 f   sfc_debug:sfdb_handle_management.obj
 0001:0002b770       sf_debug_ss_copy_dimension 000000018002c770 f   sfc_debug:sfdb_symbol_scope.obj
 0001:0002b830       sf_debug_ss_get_number_elements 000000018002c830 f   sfc_debug:sfdb_symbol_scope.obj
 0001:0002b850       sf_debug_ss_fill_data_struct 000000018002c850 f   sfc_debug:sfdb_symbol_scope.obj
 0001:0002bba0       sf_debug_ss_reset_data_info 000000018002cba0 f   sfc_debug:sfdb_symbol_scope.obj
 0001:0002bc00       sf_debug_fill_data_info_by_symbol_scope_entry 000000018002cc00 f   sfc_debug:sfdb_symbol_scope.obj
 0001:0002bcc0       sf_debug_fill_data_info_by_data_vector 000000018002ccc0 f   sfc_debug:sfdb_symbol_scope.obj
 0001:0002bf10       get_data_info_helper       000000018002cf10 f   sfc_debug:sfdb_symbol_scope.obj
 0001:0002c010       sf_debug_ss_get_data_info  000000018002d010 f   sfc_debug:sfdb_symbol_scope.obj
 0001:0002c240       sf_debug_select_mex_function 000000018002d240 f   sfc_debug:sfdb_symbol_scope.obj
 0001:0002c270       sf_debug_is_dyn_matrix_initialized 000000018002d270 f   sfc_debug:sfdb_symbol_scope.obj
 0001:0002c290       sf_debug_ss_set_data_value_try 000000018002d290 f   sfc_debug:sfdb_symbol_scope.obj
 0001:0002c460       sf_debug_ss_get_data_value 000000018002d460 f   sfc_debug:sfdb_symbol_scope.obj
 0001:0002cbd0       sf_debug_ss_data_bytes_string 000000018002dbd0 f   sfc_debug:sfdb_symbol_scope.obj
 0001:0002cc80       sf_debug_ss_data_class_string 000000018002dc80 f   sfc_debug:sfdb_symbol_scope.obj
 0001:0002d010       sf_debug_ss_data_size_string 000000018002e010 f   sfc_debug:sfdb_symbol_scope.obj
 0001:0002d0f0       sf_debug_ss_data_create_data_info_struct 000000018002e0f0 f   sfc_debug:sfdb_symbol_scope.obj
 0001:0002d3c0       sf_debug_ss_data_create_name_value_pair 000000018002e3c0 f   sfc_debug:sfdb_symbol_scope.obj
 0001:0002d460       sf_debug_ss_data_get_whos_info 000000018002e460 f   sfc_debug:sfdb_symbol_scope.obj
 0001:0002d470       same_named_data_in_data_array 000000018002e470 f   sfc_debug:sfdb_symbol_scope.obj
 0001:0002ed00       sf_debug_cc_terminate_chart 000000018002fd00 f   sfc_debug:sfdb_coverage.obj
 0001:0002f0a0       sf_debug_cc_terminate_instance 00000001800300a0 f   sfc_debug:sfdb_coverage.obj
 0001:0002fc90       sf_debug_cc_mark_object_if_needed 0000000180030c90 f   sfc_debug:sfdb_coverage.obj
 0001:00030590       sf_debug_bm_initialize_eml 0000000180031590 f   sfc_debug:sfdb_breakpoints.obj
 0001:000316d0       sf_debug_bm_map_debug_tag_to_breakpoint_tag 00000001800326d0 f   sfc_debug:sfdb_breakpoints.obj
 0001:000317b0       sf_debug_bm_is_a_eml_breakpoint_impl 00000001800327b0 f   sfc_debug:sfdb_breakpoints.obj
 0001:000332f0       sf_debug_sc_push_on_error_stack 00000001800342f0 f   sfc_debug:sfdb_state_consistency.obj
 0001:00033420       sf_debug_sc_reset_error_stack 0000000180034420 f   sfc_debug:sfdb_state_consistency.obj
 0001:000335b0       sf_debug_sc_is_state_inconsistent 00000001800345b0 f   sfc_debug:sfdb_state_consistency.obj
 0001:000338b0       sf_debug_sc_fill_consistency_info 00000001800348b0 f   sfc_debug:sfdb_state_consistency.obj
 0001:00033e90       void_assertion_fcn         0000000180034e90 f   sfc_debug:sfdb_call_stack.obj
 0001:00034410       sf_debug_tm_fill_local_trace 0000000180035410 f   sfc_debug:sfdb_call_stack.obj
 0001:000349e0       sf_debug_cd_terminate_instance 00000001800359e0 f   sfc_debug:sfdb_cycle_detection.obj
 0001:00034a40       sf_debug_cd_free_checksum_stack 0000000180035a40 f   sfc_debug:sfdb_cycle_detection.obj
 0001:00034a90       sf_debug_cd_reset_pack_strings 0000000180035a90 f   sfc_debug:sfdb_cycle_detection.obj
 0001:00035150       md5file_clear              0000000180036150 f   sfc_debug:ckmd5.obj
 0001:00035180       Encode                     0000000180036180 f   sfc_debug:ckmd5.obj
 0001:000351d0       Decode                     00000001800361d0 f   sfc_debug:ckmd5.obj
 0001:00035270       MD5Transform               0000000180036270 f   sfc_debug:ckmd5.obj
 0001:00035ac0       md5file_addn               0000000180036ac0 f   sfc_debug:ckmd5.obj
 0001:00035b90       md5file_hash               0000000180036b90 f   sfc_debug:ckmd5.obj
 0001:0003605c       pre_c_init                 000000018003705c f   MSVCRT:crtdll.obj
 0001:00036318       __DllMainCRTStartup        0000000180037318 f   MSVCRT:crtdll.obj
 0001:00036a20       __DllMainCRTStartup$filt$0 0000000180037a20 f   MSVCRT:crtdll.obj
 0001:00036a50       __DllMainCRTStartup$fin$1  0000000180037a50 f   MSVCRT:crtdll.obj
 0001:00036a6a       _onexit$fin$0              0000000180037a6a f   MSVCRT:atonexit.obj
 0001:00036a90       _IsNonwritableInCurrentImage$filt$0 0000000180037a90 f   MSVCRT:pesect.obj
